:020000040800F2
:100000000000012021E100080BE100080DE10008DB
:100010000FE1000811E1000813E1000800000000F2
:1000200000000000000000000000000015E10008D2
:1000300017E100080000000019E100081BE10008BA
:1000400071E1000871E1000871E1000871E1000848
:1000500071E1000871E1000871E1000871E1000838
:1000600071E1000871E1000871E1000871E1000828
:1000700071E1000871E1000871E1000871E1000818
:1000800071E1000871E1000871E1000871E1000808
:100090000000000071E1000871E1000871E1000852
:1000A00071E1000871E1000871E1000871E10008E8
:1000B00071E1000871E1000871E1000871E10008D8
:1000C00071E1000871E1000871E1000871E10008C8
:1000D000BD3600080D67000871E1000871E10008F5
:1000E00071E1000825C9000871E1000871E100080C
:1000F00071E10008000000000000000071E100084C
:1001000071E1000871E10008B9C8000871E1000858
:1001100071E1000871E1000871E1000871E1000877
:1001200071E1000871E1000871E1000871E1000867
:0801300071E1000871E1000813
:1001380010B5054C237833B9044B13B10448AFF319
:1001480000800123237010BDB002002000000000D1
:10015800E413010808B5034B1BB103490348AFF387
:10016800008008BD00000000B4020020E41301086C
:1001780010F8012B11F8013B012A28BF9A42F7D049
:10018800D01A7047034613F8012B002AFBD1181A1E
:100198000138704781F0004102E000BF83F000435E
:1001A80030B54FEA41044FEA430594EA050F08BF0A
:1001B80090EA020F1FBF54EA000C55EA020C7FEACE
:1001C800645C7FEA655C00F0E2804FEA5454D4EB4B
:1001D8005555B8BF6D420CDD2C4480EA020281EA15
:1001E800030382EA000083EA010180EA020281EA4D
:1001F8000303362D88BF30BD11F0004F4FEA01319F
:100208004FF4801C4CEA113102D0404261EB4101AD
:1002180013F0004F4FEA03334CEA133302D0524233
:1002280063EB430394EA050F00F0A780A4F10104EF
:10023800D5F1200E0DDB02FA0EFC22FA05F2801829
:1002480041F1000103FA0EF2801843FA05F359410F
:100258000EE0A5F120050EF1200E012A03FA0EFC8E
:1002680028BF4CF0020C43FA05F3C01851EBE371B8
:1002780001F0004507D54FF0000EDCF1000C7EEBD5
:1002880000006EEB0101B1F5801F1BD3B1F5001F13
:100298000CD349085FEA30004FEA3C0C04F1010432
:1002A8004FEA445212F5800F80F09A80BCF1004F5B
:1002B80008BF5FEA500C50F1000041EB045141EADD
:1002C800050130BD5FEA4C0C404141EB0101013CA6
:1002D80028BFB1F5801FE9D291F0000F04BF014695
:1002E8000020B1FA81F308BF2033A3F10B03B3F167
:1002F80020020CDA0C3208DD02F1140CC2F10C02F7
:1003080001FA0CF021FA02F10CE002F11402D8BF54
:10031800C2F1200C01FA02F120FA0CFCDCBF41EA20
:100328000C019040E41AA2BF01EB0451294330BDEF
:100338006FEA04041F3C1CDA0C340EDC04F11404CC
:10034800C4F1200220FA04F001FA02F340EA0300A3
:1003580021FA04F345EA030130BDC4F10C04C4F1E9
:10036800200220FA02F001FA04F340EA03002946C9
:1003780030BD21FA04F0294630BD94F0000F83F413
:10038800801306BF81F480110134013D4EE77FEAF6
:10039800645C18BF7FEA655C29D094EA050F08BF42
:1003A80090EA020F05D054EA000C04BF1946104623
:1003B80030BD91EA030F1EBF0021002030BD5FEA67
:1003C800545C05D14000494128BF41F0004130BD8F
:1003D80014F580043CBF01F5801130BD01F00045E3
:1003E80045F0FE4141F470014FF0000030BD7FEA56
:1003F800645C1ABF194610467FEA655C1CBF0B4651
:10040800024650EA013406BF52EA033591EA030F67
:1004180041F4002130BD00BF90F0000F04BF00215F
:10042800704730B54FF4806404F132044FF0000592
:100438004FF0000150E700BF90F0000F04BF00210B
:10044800704730B54FF4806404F1320410F0004571
:1004580048BF40424FF000013EE700BF42004FEA6C
:10046800E2014FEA31014FEA02701FBF12F07F43E9
:1004780093F07F4F81F06051704732F07F4208BFA0
:10048800704793F07F4F04BF41F40021704730B5A7
:100498004FF4607401F0004521F000411CE700BFF3
:1004A80050EA010208BF704730B54FF000050AE076
:1004B80050EA010208BF704730B511F0004502D577
:1004C800404261EB41014FF4806404F132045FEA79
:1004D800915C3FF4D8AE4FF003025FEADC0C18BF22
:1004E80003325FEADC0C18BF033202EBDC02C2F114
:1004F800200300FA03FC20FA02F001FA03FE40EAA6
:100508000E0021FA02F11444BDE600BF70B54FF0A9
:10051800FF0C4CF4E06C1CEA11541DBF1CEA135587
:1005280094EA0C0F95EA0C0F00F0DEF82C4481EAEF
:10053800030621EA4C5123EA4C5350EA013518BF0F
:1005480052EA033541F4801143F4801338D0A0FBFC
:1005580002CE4FF00005E1FB02E506F00042E0FBA9
:1005680003E54FF00006E1FB03569CF0000F18BFAF
:100578004EF0010EA4F1FF04B6F5007F64F5407457
:1005880004D25FEA4E0E6D4146EB060642EAC621EA
:1005980041EA55514FEAC52040EA5E504FEACE2E57
:1005A800B4F1FD0C88BFBCF5E06F1ED8BEF1004F5A
:1005B80008BF5FEA500E50F1000041EB045170BDD6
:1005C80006F0004646EA010140EA020081EA03011A
:1005D800B4EB5C04C2BFD4EB0C0541EA045170BD16
:1005E80041F480114FF0000E013C00F3AB8014F190
:1005F800360FDEBF002001F0004170BDC4F10004D9
:10060800203C35DA0C341BDC04F11404C4F1200559
:1006180000FA05F320FA04F001FA05F240EA0200B4
:1006280001F0004221F0004110EBD37021FA04F6EA
:1006380042EB06015EEA430E08BF20EAD37070BDA4
:10064800C4F10C04C4F1200500FA04F320FA05F003
:1006580001FA04F240EA020001F0004110EBD37005
:1006680041F100015EEA430E08BF20EAD37070BD75
:10067800C4F1200500FA05F24EEA020E20FA04F34E
:1006880001FA05F243EA020321FA04F001F00041FD
:1006980021FA04F220EA020000EBD3705EEA430E6E
:1006A80008BF20EAD37070BD94F0000F0FD101F09D
:1006B8000046400041EB010111F4801F08BF013CD6
:1006C800F7D041EA060195F0000F18BF704703F014
:1006D8000046520043EB030313F4801F08BF013D9B
:1006E800F7D043EA0603704794EA0C0F0CEA135557
:1006F80018BF95EA0C0F0CD050EA410618BF52EA11
:100708004306D1D181EA030101F000414FF0000016
:1007180070BD50EA410606BF1046194652EA430624
:1007280019D094EA0C0F02D150EA013613D195EA98
:100738000C0F05D152EA03361CBF104619460AD1E0
:1007480081EA030101F0004141F0FE4141F47001EA
:100758004FF0000070BD41F0FE4141F4780170BDDA
:1007680070B54FF0FF0C4CF4E06C1CEA11541DBF3F
:100778001CEA135594EA0C0F95EA0C0F00F0A7F841
:10078800A4EB050481EA030E52EA03354FEA01316E
:1007980000F088804FEA03334FF0805545EA131381
:1007A80043EA12634FEA022245EA111545EA106549
:1007B8004FEA00260EF000419D4208BF964244F1E0
:1007C800FD0404F5407402D25B084FEA3202B61AFF
:1007D80065EB03055B084FEA32024FF480104FF4D3
:1007E800002CB6EB020E75EB030E22BFB61A754647
:1007F80040EA0C005B084FEA3202B6EB020E75EBDA
:10080800030E22BFB61A754640EA5C005B084FEA41
:100818003202B6EB020E75EB030E22BFB61A75460E
:1008280040EA9C005B084FEA3202B6EB020E75EB19
:10083800030E22BFB61A754640EADC0055EA060EDA
:1008480018D04FEA051545EA16754FEA06164FEA1D
:10085800C30343EA52734FEAC2025FEA1C1CC0D1C9
:1008680011F4801F0BD141EA00014FF000004FF056
:10087800004CB6E711F4801F04BF01430020B4F117
:10088800FD0C88BFBCF5E06F3FF6AFAEB5EB030CCF
:1008980004BFB6EB020C5FEA500C50F1000041EBCC
:1008A800045170BD0EF0004E4EEA113114EB5C0499
:1008B800C2BFD4EB0C0541EA045170BD41F480116C
:1008C8004FF0000E013C90E645EA060E8DE60CEA74
:1008D800135594EA0C0F08BF95EA0C0F3FF43BAF91
:1008E80094EA0C0F0AD150EA01347FF434AF95EA48
:1008F8000C0F7FF425AF104619462CE795EA0C0F2C
:1009080006D152EA03353FF4FDAE1046194622E7F8
:1009180050EA410618BF52EA43067FF4C5AE50EAD2
:1009280041047FF40DAF52EA43057FF4EBAE12E7C2
:100938004A0011D212F5001211D20DD56FF4787356
:10094800B3EB62520ED44FEAC12343F0004343EAAB
:10095800505323FA02F070474FF00000704750EAF6
:10096800013002D14FF0FF3070474FF00000704760
:1009780080F0004002E000BF81F0004142001FBF4C
:100988005FEA410392EA030F7FEA226C7FEA236C55
:100998006AD04FEA1262D2EB1363C1BFD21841404A
:1009A80048404140B8BF5B42192B88BF704710F0E0
:1009B800004F40F4000020F07F4018BF404211F083
:1009C800004F41F4000121F07F4118BF494292EAEB
:1009D800030F3FD0A2F1010241FA03FC10EB0C0017
:1009E800C3F1200301FA03F100F0004302D54942A4
:1009F80060EB4000B0F5000F13D3B0F1807F06D351
:100A080040084FEA310102F10102FE2A51D2B1F148
:100A1800004F40EBC25008BF20F0010040EA03003D
:100A28007047490040EB0000013A28BFB0F5000FBD
:100A3800EDD2B0FA80FCACF1080CB2EB0C0200FA73
:100A48000CF0AABF00EBC25052421843BCBFD040C2
:100A58001843704792F0000F81F4000106BF80F43C
:100A680000000132013BB5E74FEA41037FEA226CFF
:100A780018BF7FEA236C21D092EA030F04D092F0CA
:100A8800000F08BF0846704790EA010F1CBF0020FE
:100A9800704712F07F4F04D1400028BF40F000405B
:100AA800704712F100723CBF00F50000704700F07B
:100AB800004343F0FE4040F4000070477FEA2262A2
:100AC80016BF08467FEA23630146420206BF5FEA73
:100AD800412390EA010F40F4800070474FF0000373
:100AE80004E000BF10F0004348BF40425FEA000C3A
:100AF80008BF704743F0964301464FF000001CE0E2
:100B080050EA010208BF70474FF000030AE000BF37
:100B180050EA010208BF704711F0004302D5404275
:100B280061EB41015FEA010C02BF844601460020E7
:100B380043F0B64308BFA3F18053A3F50003BCFA02
:100B48008CF2083AA3EBC25310DB01FA02FC6344AF
:100B580000FA02FCC2F12002BCF1004F20FA02F2B6
:100B680043EB020008BF20F00100704702F12002A9
:100B780001FA02FCC2F1200250EA4C0021FA02F20A
:100B880043EB020008BF20EADC7070474FF0FF0C0F
:100B98001CEAD0521EBF1CEAD15392EA0C0F93EA0A
:100BA8000C0F6FD01A4480EA010C400218BF5FEAAC
:100BB80041211ED04FF0006343EA501043EA51111F
:100BC800A0FB01310CF00040B1F5000F3EBF490019
:100BD80041EAD3715B0040EA010062F17F02FD2A1D
:100BE8001DD8B3F1004F40EBC25008BF20F0010000
:100BF800704790F0000F0CF0004C08BF49024CEA17
:100C0800502040EA51207F3AC2BFD2F1FF0340EAA8
:100C1800C250704740F400004FF00003013A5DDC19
:100C280012F1190FDCBF00F000407047C2F100025A
:100C3800410021FA02F1C2F1200200FA02FC5FEA47
:100C4800310040F1000053EA4C0308BF20EADC7091
:100C5800704792F0000F00F0004C02BF400010F403
:100C6800000F013AF9D040EA0C0093F0000F01F0B0
:100C7800004C02BF490011F4000F013BF9D041EAD2
:100C88000C018FE70CEAD15392EA0C0F18BF93EAD4
:100C98000C0F0AD030F0004C18BF31F0004CD8D1FE
:100CA80080EA010000F00040704790F0000F17BF85
:100CB80090F0004F084691F0000F91F0004F14D0CB
:100CC80092EA0C0F01D142020FD193EA0C0F03D123
:100CD8004B0218BF084608D180EA010000F0004026
:100CE80040F0FE4040F40000704740F0FE4040F401
:100CF800400070474FF0FF0C1CEAD0521EBF1CEAA0
:100D0800D15392EA0C0F93EA0C0F69D0A2EB0302BD
:100D180080EA010C49024FEA402037D04FF0805357
:100D280043EA111143EA10130CF000408B4238BF1C
:100D38005B0042F17D024FF4000C8B4224BF5B1A2A
:100D480040EA0C00B3EB510F24BFA3EB510340EA78
:100D58005C00B3EB910F24BFA3EB910340EA9C0026
:100D6800B3EBD10F24BFA3EBD10340EADC001B0196
:100D780018BF5FEA1C1CE0D1FD2A3FF650AF8B423A
:100D880040EBC25008BF20F0010070470CF0004C47
:100D98004CEA50207F32C2BFD2F1FF0340EAC25072
:100DA800704740F400004FF00003013A37E792F033
:100DB800000F00F0004C02BF400010F4000F013A91
:100DC800F9D040EA0C0093F0000F01F0004C02BF8C
:100DD800490011F4000F013BF9D041EA0C0195E7F5
:100DE8000CEAD15392EA0C0F08D142027FF47DAF8E
:100DF80093EA0C0F7FF470AF084676E793EA0C0F7E
:100E080004D14B023FF44CAF08466EE730F0004C7B
:100E180018BF31F0004CCAD130F000427FF45CAF0B
:100E280031F000437FF43CAF5FE700BF4FF0FF3C79
:100E380006E000BF4FF0010C02E000BF4FF0010CCC
:100E48004DF804CD4FEA40024FEA41037FEA226C95
:100E580018BF7FEA236C11D001B052EA530C18BFB7
:100E680090EA010F58BFB2EB030088BFC81738BF1C
:100E78006FEAE17018BF40F0010070477FEA226C0A
:100E880002D15FEA402C05D17FEA236CE4D15FEA06
:100E9800412CE1D05DF8040B704700BF844608463A
:100EA8006146FFE70FB5FFF7C9FF002848BF10F1FB
:100EB800000F0FBD4DF808EDFFF7F4FF0CBF012040
:100EC80000205DF808FB00BF4DF808EDFFF7EAFFCA
:100ED80034BF012000205DF808FB00BF4DF808ED85
:100EE800FFF7E0FF94BF012000205DF808FB00BF7A
:100EF8004DF808EDFFF7D2FF94BF012000205DF800
:100F080008FB00BF4DF808EDFFF7C8FF34BF01200C
:100F180000205DF808FB00BF4FEA40024FEA41039A
:100F28007FEA226C02D15FEA402C08D17FEA236C69
:100F380002D15FEA412C02D14FF0000070474FF018
:100F4800010070474FEA4002B2F1FE4F0FD34FF055
:100F58009E03B3EB12620DD94FEA002343F000431E
:100F680010F0004F23FA02F018BF404270474FF0CC
:100F78000000704712F1610F01D1420205D110F053
:100F8800004008BF6FF0004070474FF00000704706
:100F980042000ED2B2F1FE4F0BD34FF09E03B3EBDB
:100FA800126209D44FEA002343F0004323FA02F007
:100FB80070474FF00000704712F1610F01D14202F3
:100FC80002D14FF0FF3070474FF00000704700BF6C
:100FD8000022427082700122C270B1FA81F10222AD
:100FE80049090271032201704271704743788B42AC
:100FF8001FD0012941700AD0022910D0C1B901239C
:10100800C37081700223037103234371704703780F
:1010180043B1012383700223C3700023F3E70378ED
:10102800002BF6D0022383700023C3700123EAE764
:10103800FEE7704782B00B88ADF800304B88ADF8FA
:1010480002308B88ADF80430CB88ADF80630023911
:10105800431C053013F8012F0DF1080C0CEB42026C
:10106800834232F8082C21F8022FF3D102B07047DE
:1010780010B50C461146FFF7B9FF2146BDE81040F0
:10108800FFF7D8BF0A4B10B54FF07F32C0E92323D2
:101098004FF47F43A0F89430FF2380F8963004463D
:1010A800983000F073FD002384F8A43010BD00BF11
:1010B800FFFF7F0070B51146154604461E4600F036
:1010C800DBFC294604F1140000F0D6FC294604F1A3
:1010D800280000F0D1FC294604F13C0000F0CCFCCB
:1010E800294604F1500000F0C7FC294604F16400C9
:1010F80000F0C2FC294604F1780000F0BDFC4FF472
:10110800FA7332464FF4FA6104F1980000F024FDB6
:101118002046FFF7B7FF002384F8A5304FF47F433C
:10112800A4F8A63070BD704700F0ADBC143000F0D4
:10113800AABC08B5503000F0B0FC292100F1140316
:101148000246B3FBF1F313F0FF0002D1101E18BFE3
:10115800012008BD08B5643000F09FFC292100F18A
:1011680014030246B3FBF1F313F0FF0002D1101E83
:1011780018BF012008BD90F8903013B990F98C0081
:10118800704790F98D00704790F8903013B990F936
:101198008E00704790F98F00704710B504460BF029
:1011A800E3FC38B104F13C0000F071FC012838BFC1
:1011B8000120C0B210BD783000F071BC783000F06A
:1011C80076BC10B5044600F038FC04F1140000F0B9
:1011D80034FC04F1280000F030FC04F13C0000F07D
:1011E8002CFC04F1500000F034FC04F1640000F021
:1011F80030FC04F17800BDE8104000F030BC7F28D6
:1012080007D0002807DA10F1800F06D04042C0B29C
:10121800704700207047012070477F20704710B149
:10122800404240B270477F2070477F280FD010F1AE
:10123800310F0EDA10F1780F0DDB7830FE2340B253
:10124800584323304623B0FBF3F0C0B27047FF2069
:101258007047FE20704700207047012805DD40F2E6
:10126800FE73984203DC80B270470120704740F259
:10127800FF707047A0F57870C0EBC02040F2AE73E5
:1012880090FBF3F000F58060FFF7E7BFFFF7F2BFD0
:10129800032812DD0C2812DD0F2812DD122812DDBA
:1012A800162812DD192812DD1C2812DD1F2812DD70
:1012B8002128CCBFFF20062070470020704701205E
:1012C80070470220704708207047032070470720A6
:1012D80070470420704705207047000005289ABF12
:1012E800014B185CFF2070474014010805289ABF7D
:1012F800014B185CFF207047461401087F2803D073
:10130800002803DAC0B2704700207047FF207047FA
:101318007F2811D010F1320F10DA884210DD401A00
:101328006423C1F1FF21584301F57F01CE313130EB
:1013380090FBF1F0C0B27047FF20704764207047FF
:1013480000207047014B4840185C70474C14010856
:1013580052B110B4054C0A4411F8013B58408A4276
:10136800205CF9D110BC7047704700BF4C140108CD
:10137800392808D822280ED9094B2338C0B2C340CF
:1013880003F0010070475F2807D0613819288CBF27
:10139800002001207047002070470120704700BFDF
:1013A80001EC7F00F8B50246451E461D00245F2764
:1013B80015F8010FFF2804BF0134E4B2FFF7D8FF86
:1013C80000B92F70AE42F3D1062C04D119B10B68C5
:1013D80013608B88938000239371F8BD2DE9F8433F
:1013E800DFF83490471E441D012500264FF02808D9
:1013F80017F8011F08480FF092FF034610B1A0EB41
:101408000903DBB2A3FB05329E19A742A5FB0853CB
:10141800EED13046BDE8F8834C15010810B5417986
:10142800A1F13000C3B2092B07D80523B0FBF3F3B1
:1014380003EB8303C01AC0B210BD044C20460FF062
:101448006EFF0028F1D0001BC0B2EEE74C15010872
:10145800F0B5094B094F821D2826B1FBF3F4272C60
:1014680094BF3D5D302502F8015D824203FB1411F3
:10147800B3FBF6F3F1D1F0BD00801A064C15010854
:1014880070B50446FEF77EFE82B20023551E98B260
:10149800A84214FA83F104DA265C302E03F1010322
:1014A800F5D0121A01322046BDE870400FF006BF91
:1014B8002DE9F04F0D4699B0164600211A461F46F1
:1014C80080460FF015FF00212A2201A800910FF095
:1014D8000FFFDFF8CC90DFF8CCA0DFF8CCB005EB3D
:1014E8004606AE4211D16846FEF74CFE30B100F117
:1014F80060030DEB0300002300F8613C6946404699
:101508000FF056FF19B0BDE8F08F35F9020B47F61A
:10151800FF739842E7D0002812DC59460CA80FF058
:1015280047FF6846FEF72EFE04460CA8FEF72AFE83
:101538000444A742D5D30CA968460FF0E1FED0E7D2
:10154800B0F57A7F0BDA0CA980B20EF06EF80CA811
:10155800FFF796FF51460CA80FF0D2FEE1E764238F
:101568000CA93230B0FBF3F080B20EF05EF80CA894
:10157800FFF786FF0CA8FEF705FE00F15F036B443A
:1015880000F160010DEB010013F8302C00F8302C4D
:101598002E2203F8302C002300F82F3C4946DAE7C6
:1015A8003A1401083514010830140108F0B589B05F
:1015B8006D4600242F468E1CE1B28A4204D8394673
:1015C800FFF776FF09B0F0BD36F8241025F8021BA6
:1015D8000134F1E742F210736421B0FBF3F203FB2C
:1015E8001200B0FBF1F301FB130000EB023000EB3B
:1015F800831080B27047020B00F03F0342F2107173
:1016080001FB0233C0F38510642202FB00307047EF
:101618002DE9F04142F2107388B0B1FBF3F603FBF9
:1016280016141F49DFF87C8005460FF0C1FE694695
:10163800F0B20DF0D7FF6846FFF722FF694628464B
:101648000FF05EFE414628460FF05AFE64276946B1
:10165800B4FBF7F6F0B20DF0C5FF6846FFF710FFD0
:10166800694628460FF04CFE07FB164441462846BB
:101678000FF046FE6946E0B20DF0B4FF9DF8013068
:101688008DF800309DF802308DF80130694600234E
:1016980028468DF802300FF033FE08B0BDE8F0811F
:1016A800012601083E14010870B50E4600210546C2
:1016B80014460FF01DFE00239AB2944200D870BD64
:1016C800F25C002AFBD0EA540133F5E770B50E4608
:1016D80014460021013205460FF00AFE00239AB293
:1016E800944200D870BDF25C002AFBD0EA54013362
:1016F800F5E730B50023044698B2904201D30120A3
:1017080005E0E55CC85C1DB9B0FA80F0400930BD61
:101718000028FCD0854203F10103EDD00020F6E754
:10172800914206D19DF900008342CCBF00200120E0
:101738007047022909D0022A05D0012905D0531E75
:1017480058425841704701207047002070477D2358
:10175800438043F2390309B2C360002301808180CA
:10176800C380037270470000C2680449044B01FB40
:10177800023323F00043C360980F7047FD43030012
:10178800C39E260010B50129044680791AD804287A
:1017980001D80130A071012AE07917D8042801D8AE
:1017A8000130E07191424AD8914245D3012930D1A4
:1017B800012A2ED1A279E3799A4228D322D96FF04F
:1017C8007C0310E00028E6D00138E3E708B10138CF
:1017D800E0710229E6D1022AE6D19DF90820934258
:1017E8000BDDB4F9003062881A4412B27C2A28DD75
:1017F8007D2262800022227227E01BDA23885B4266
:101808001BB2F0E72046FFF7AFFF0028D7D07D23B3
:10181800E9E7B4F90400B4F900302288B4F90210F9
:10182800002804DB7C29DEDD524213B2DBE77C3181
:10183800D9DBF9E70023D6E76FF04A03D3E74B2358
:10184800D1E712F17C0F02DB6280A38010BD4FF656
:10185800837262800122CEE702680449044B01FBCF
:10186800023323F000430360180C7047FD43030064
:10187800C39E2600F0B5002597B001608580044618
:101888005622294668460FF033FD0126E27DAA421A
:1018980009D80023802104F1B800A37517B0BDE86A
:1018A800F0400FF025BD2046FFF7D6FFE7797B1BF8
:1018B800002190FBF3F202FB1300C0B2EC460A468B
:1018C800CBB29F4223D800230022277B1146D0B2F7
:1018D800874227D80029D9D1A279033A012A04EBF3
:1018E800050105D925B191F9172012BB012BCDD9D6
:1018F8000B76A26852F82310583305F10E026B4498
:10190800013544F8221003F8586CEDB2BEE71CF814
:1019180001EBBEF1000F03D18242D5D00132D2B221
:101928000131CDE72069805C0132984208BF01216E
:10193800CDE7501E8342DBDB01329342D8DCA5E7BA
:101948002DE9F047154696B0013D01600271044645
:101958004371EDB25622002168460FF0C9FC0027FA
:10196800022D84BF4FF0010900253E464FF0010AC1
:1019780094F807809CBF4FF00309B8FBF9F8E27DA3
:10198800B24209D80023802104F1B800A37516B02B
:10199800BDE8F0470FF0ACBC2046FFF75DFFA8EBB1
:1019A8000603002190FBF3F202FB1300C0B2EC46E1
:1019B8000A46CBB2434506D21CF801EBBEF1000F34
:1019C8002AD1824226D1434528BF434603FB095109
:1019D800002094F80CE001F0FF018446C2B296455D
:1019E8001CD8BCF1000FCAD116B1FFB9012BC6D95A
:1019F800A2191F461176A26852F8211006F10E02AC
:101A0800013644F8221003F158026A44F6B202F88B
:101A180058ACB4E70132D2B20131CAE72269125C8C
:101A280001308A4208BF4FF0010CD7E77A1E934273
:101A3800DEDB7A1C9342DBDCA1E7D0E901236421D9
:101A4800D31AC36082604B43418AB3FBF1F303743A
:101A58007047D0E90123D31AC0E9022370474368CD
:101A68002BB1C26864214A43B2FBF3F2D3B20374C8
:101A78000023C360436070470023C0E902334182FA
:101A88004360037470474368013343607047007CC8
:101A9800704743680B4443607047C068704711B192
:101AA800C3680133C3604368013343607047007CF7
:101AB80070470023038083700372704703460078E1
:101AC80010B100221A707047587810B100225A706D
:101AD8007047987810B100229A707047187A08B148
:101AE80000221A7270470170704701707047817048
:101AF80070478170426070474068704700234360B8
:101B0800038170470A2310B50446838001F0BAFFA9
:101B18002368E0809B6820469847208110BD038990
:101B280070B504469BB1858845B1013DADB285804D
:101B38006DB903681B68BDE87040184701F0A2FF43
:101B4800E388C01A238980B2834201D2258170BDFF
:101B5800236820465B68EEE72DE9F041044610460D
:101B68001D4616468846FEF7B9FF074606EB0800ED
:101B7800FEF7B4FF01463846FFF7BCF86560206001
:101B88002846FEF7AFFFA060BDE8F08110B5044617
:101B98004068FEF7A7FFA06010BD000010B502293D
:101BA800044680EAE070A0EBE47068D15AB9002CD2
:101BB800ACBF7F233F239842A8BF1846002C01DA08
:101BC80040F0400010BD012A1AD1632805DC40000E
:101BD800002CF7DA40F48070F4E740F2F5439842BD
:101BE8000CDCFEF77BFF5749FEF7D0FF0EF03CFAFE
:101BF800FFF7CEF9400040F00100E9E7FF20E7E7F2
:101C0800022A40F09C80632805DC8000002CD9DA89
:101C180040F40070D6E7B0F57A7F0CDAFEF75EFF85
:101C28004849FEF7B3FF0EF01FFAFFF7B1F980003D
:101C380040F00100EAE742F20F7398420CD8FEF731
:101C48004DFF4149FEF7A2FF0EF00EFAFFF7A0F98B
:101C5800800040F00200D9E73C4B98420CD8FEF7D0
:101C68003DFF3B49FEF792FF0EF0FEF9FFF790F9B2
:101C7800800040F00300C9E740F2FF10C6E70329DF
:101C88005DD1012A1BD1B0F57A7F05DA4000002C1E
:101C980098DA40F4006095E7B0F5205F0CDAFEF7BB
:101CA8001DFF2849FEF772FF0EF0DEF9FFF770F905
:101CB800400040F00100EAE740F2FF70E7E7022A3F
:101CC8003DD1B0F57A7F06DA8000002CBFF67AAFF6
:101CD80040F4805076E742F20F7398420CDCFEF72E
:101CE800FDFE1849FEF752FF0EF0BEF9FFF750F956
:101CF800800040F00100E8E7164B98420CD8FEF748
:101D0800EDFE1149FEF742FF0EF0AEF9FFF740F97C
:101D1800800040F00200D8E7B0F57A2F0CD2FEF729
:101D2800DDFE0B49FEF732FF0EF09EF9FFF730F9A2
:101D3800800040F00300C8E740F6FF70C5E70020C8
:101D480040E700BFCDCCCC3D0AD7233C17F00100BB
:101D58006F12833A9F8601000023036070470000DA
:101D680038B5084B09291B7828BF09218B4204463E
:101D78000D4602D10023036038BD01F077FE2571BE
:101D88002060F9E7CC020020036810B504460BB9BF
:101D9800002010BD01F06AFE2368C01A40F2EE234D
:101DA8009842F5D90023054A2360127823799A428C
:101DB800EED0034A0120D377EBE700BFCC02002026
:101DC80028030020FF2343710023017183710381DD
:101DD8008372704738B5037904460D465BB1417983
:101DE800A94208D041B101290AD00023A371657125
:101DF80055B1012D0FD038BD03689B689847F4E7AB
:101E080003680021DB68F9E723689B680121204605
:101E18009847A071EFE723682946DB68F7E72DE9C3
:101E2800F04F077CC37B857CC67C90F815E090F862
:101E3800208090F80EC0BF000C4647EA931703F0C5
:101E48003F01437C03F0010247EA822705F00F02B5
:101E5800D20142EA530206F07F031B0143EA15133D
:101E6800057D89B06D0045EAD6150EF00306059389
:101E780045EA4623867D009306F01F05AD0145EA35
:101E88009E03C57D90F819E00193ED0045EA5613CD
:101E9800057E02930EF0070645EA0623857E039326
:101EA80005F03F06760146EADE03C67E90F81CE0A0
:101EB8000493B60046EA95160EF0010546EA852613
:101EC800457F069205F00F0B4FEACB1B4BEA5E0BE2
:101ED80090F81EE00EF07F0A4FEA0A1A4AEA151A2D
:101EE800C57F6D0045EADE1508F0030E45EA4E256C
:101EF80090F821E00EF01F094FEA891949EA98097C
:101F0800490190F82280407B41EADC010CF0070C83
:101F180040EA0C204FEAC80848EA5E180791FFF724
:101F2800A9F9079920800846FFF7A4F96080384688
:101F3800FFF7A0F9069AA0801046FFF79BF9059BCA
:101F4800E0801846FFF796F920810098FFF792F98C
:101F580060810198FFF78EF9A0810298FFF78AF94E
:101F6800E0810398FFF786F920820498FFF782F949
:101F780060823046FFF77EF9A0825846FFF77AF96B
:101F8800E0825046FFF776F920832846FFF772F97A
:101F980060834846FFF76EF9A0834046FFF76AF969
:101FA8004FF48063E0832384638409B0BDE8F08F35
:101FB8002DE9F04104460F4601F064FD4FF0010899
:101FC8000546236820461B689847064650B9A37AF9
:101FD800012B1FD12389ED1A40F6C4139D42C8BFB7
:101FE800A07217E0236820465B689847A37AA3B9D4
:101FF8000F2814D1A4F80A80E37AE2180133DBB27F
:10200800182B1073E3720AD939462046FFF707FFE9
:102018000023A3723046BDE8F081012BECD0258166
:10202800CFE7827922B14379012B01D8FFF7C0BFEE
:10203800002070477047704770470020704770470E
:10204800002070470020704770470020704700202C
:1020580070474FF0B04382B0DA6C0243DA64DB6C4D
:1020680003400193019B02B070474FF0B04382B028
:102078009A6D02439A659B6D03400193019B02B0E0
:1020880070474FF0B04382B01A6E02431A661B6E57
:1020980003400193019B02B0704750E8003F43F0B2
:1020A800800340E80032002AF7D1704750E8003F2B
:1020B80023F0200340E80032002AF7D1704750E8A7
:1020C800003F23F0400340E80032002AF7D1704770
:1020D80050E8003F23F0800340E80032002AF7D19F
:1020E800704770470288044B5140C9B233F8113029
:1020F80083EA122303807047044301089AB110B49D
:10210800B0F800C0084C0A4411F8013B83EA0C03FC
:10211800DBB2914234F8133083EA1C2CA0F800C0DB
:10212800F2D110BC704770470443010837B54FF629
:10213800FF730446ADF806304518AC4203D1BDF82C
:10214800060003B030BD14F8011B0DF10600FFF7BF
:10215800C9FFF2E700207047074B1B784BB9074BC4
:102168001888074B1B8880B29BB2C01A18BF012081
:1021780070470020704700BF08000020883D0020FD
:10218800863D0020704700000649074A0B881288E0
:102198000133C3F3080392B29A421EBF034AD054D4
:1021A8000B807047803300207E3300207E31002072
:1021B8000023A0F87032A0F86E3270470023A0F810
:1021C8005C32A0F85A3270473A4B5A6A037A92B294
:1021D80063B18389D31A9BB2B3F5FA7F84BF002316
:1021E8000372837A4F2B84BF00230372037A8281A0
:1021F800082B0FD8DFE803F0050E0E0E0E0E0F1792
:102208002200EE2901D0C82904D101238372417527
:10221800062303727047837A5A1C034482725975E5
:1022280041720723F5E7827A531C0244DBB28372BA
:102238005175427A9A42EDD20823EAE7837A5A1C0A
:10224800034482725975C37D162B04D1012380F88B
:1022580065300923DDE74369174A03F0FF239342FA
:1022680003D1012380F86730F3E7144A93421CD165
:10227800837E102B19D1C37E022B08D0052B0DD0DD
:10228800012BE6D1027EEE2A08BF80F86A30037E71
:10229800EE2BDED1012380F86B30DAE7012380F8DA
:1022A8006830037F80F86930D3E7012380F866300F
:1022B800CFE700BF0044014000C8002800C8003232
:1022C800044B1888044B1B8880B29BB2C01A18BFF5
:1022D80001207047803300207E3300200278024BB3
:1022E80051405B5C03707047842F0108FF23037023
:1022F800704700BF7047B0F86E32B0F870229B1A72
:1023080098B21B0444BF00F5006080B2003818BFC3
:1023180001207047A0F11400EDE7B0F87022B0F882
:102328006E12914203461FBF8118013291F8740260
:10233800B3F872121ABF0A40A3F87022002070473F
:10234800A0F11400E9E770B50B7803704B7843707F
:102358000B78FD2B05460C4638D18B788370CB78EB
:10236800C3700B7903714B7943718B7983718B68D7
:10237800C3718B68C3F30F2303728B7A43720A26E7
:10238800627804F10C01A8190FF01AF86378B4F810
:102398000C213344981CEA545A1CB4F80C1192B21C
:1023A800090AA954A278D20780B20ED504F588721A
:1023B800054404F58E7452F8041B45F8041BA24228
:1023C800F9D112782A700F3398B270BD00238B7040
:1023D8000B7983704B79C3708B7903718B68437168
:1023E8000626CDE738B54A78352A0D46044601F168
:1023F8000C010AD80EF0E4FF68780021C0F136021B
:102408002044BDE838400EF073BF403551F8043B16
:1024180040F8043BA942F9D10B88038038BD38B590
:102428004A781B2A0C46054601F10C010AD80EF021
:10243800C7FF60780021C0F11C022844BDE838407D
:102448000EF056BF283451F8043B45F8043BA1422E
:10245800F9D138BD38B54A78082A0D46044601F145
:102468000C010AD80EF0ACFF68780021C0F109020F
:102478002044BDE838400EF03BBFEB6803604B6872
:1024880043600B7A037238BD38B54A78072A0C4680
:10249800054601F10C010AD80EF092FF6078002180
:1024A800C0F108022844BDE838400EF021BFE368B7
:1024B80003604B68436038BD08B5242203480021F7
:1024C8000EF016FF024B00221A7008BDAC0C00205B
:1024D8007C0500202DE9F0411378037092F8018003
:1024E80080F80180FD2B04460F46154654D1937899
:1024F8008370D378C37013790371537943719379D7
:1025080083716B7A127A1B0403EB0223EA79134472
:1025180023F07F430A26A26863F31702A260A91971
:10252800424604F10C000EF04BFF7A7B904507D22F
:1025380008F10C00A2EB0802002120440EF0D8FE9E
:1025480063781E44AB195A78AB5D03EB0223A4F8F9
:102558000C31A378DB070ED5023615FA86F304F59D
:10256800887203F10C0153F8040B42F8040B8B42F8
:10257800F9D11B781370BB7A84F82131FB7A84F87F
:1025880022313B7B84F823317B7B84F824313B78F0
:1025980084F82031BDE8F0810023438093780371EB
:1025A800D37843711379837153790626B3E738B525
:1025B8004A78132A0C46054601F10C010AD80EF098
:1025C800FFFE60780021C0F114022844BDE83840BD
:1025D8000EF08EBE203451F8043B45F8043BA1426E
:1025E800F9D138BD2DE9F04F0C465188B1F58C7FF3
:1025F800054685B04FF0000010D31070D91CC9B241
:10260800012995BF01210023518053809CBF23706D
:1026180011700020287005B0BDE8F08F16780E2ED6
:1026280000F2908001A757F826F000BF05260008A1
:102638007126000899260008B72600084D270008CB
:102648004D2700084D2700084D2700084D27000892
:102658004D2700084D2700084D2700084D27000882
:102668004D270008C9260008481C5080635421786B
:10267800FD299BB206D10C330A21D3809180022315
:102688001370C6E708330621D38091800E23F7E73D
:10269800481C50806354D80742BFD1880D31D1807F
:1026A8000020012B8CBF034603231370B2E7481C9C
:1026B800508000208342635414BF03460E23F4E77E
:1026C800481C508063545388D1888B4232D30023EE
:1026D8005380137002232B7069802378FD2B37D128
:1026E80063792B72A3796B72637A227A1B0403EBEA
:1026F8000223E27913446B60637803F10C026A8069
:10270800A278D10701D519336B8000266968DFF8F4
:1027180000816E814FF4BC720C20B31801335B0842
:1027280000FB03F758F80770B9421AD25A1EB24292
:10273800F3D818E092889A423FF66BAF01232B70CA
:10274800002068E7107050809080D0802870F7E7EC
:10275800E3782B7223796B7263796B606378083343
:10276800D2E71E46E3D80C27774358F8073099423A
:1027780027D123782046FD2B10F801BF0CBF4FF05E
:102788000A094FF0060909EB0B03591E89B24744A1
:102798000193FFF7CBFC97F804A0ADF80E00514663
:1027A8000DF10E00FFF79EFC019BE218E35C5278E6
:1027B80003EB0223BDF80E209BB29A4209D00520F4
:1027C80000E003202870023801288CBF0020012077
:1027D80021E7BB79DA0706D5FA79934582BF04EB7E
:1027E80009018A5CAA729B0709D50C2303FB06839F
:1027F80062781B7A9A4282BF4C44E35CEB720C23EA
:1028080003FB068385F80CA05B796B730220DAE77B
:1028180084300108084B5B6A4FF0402202F5806360
:1028280053E8003F43F0200302F5806040E80031A0
:102838000029F3D1704700BF004400400A4A0B4BFF
:1028480012680B49A3FB02323220920C00FB02F201
:10285800084B486802F5FA72A3FB023292094B68EA
:102868001B1A9A42FBD870474802002083DE1B439C
:10287800001000E0D34D621008B5FFF7DFFF024BF0
:102888004FF480529A6108BD00040048024B4FF48F
:1028980080529A62FFF7D2BF0004004830B587B073
:1028A800034601AC00F1100518685968224603C2B6
:1028B8000833AB421446F7D10024094D8DF8144073
:1028C800A96801A8FDF754FC10B920B207B030BDC3
:1028D80001342E2C05F10C05F2D14FF0FF30F5E74D
:1028E8000C00002002780A4B90F801C08178D2438E
:1028F800D2B29A5C82EA0C0290F803C09A5C4A4011
:10290800995C027981EA0C01595C4A40985C7047ED
:10291800842F0108028810B58488531C23404488FA
:102928009C421EBF12189171038010BD411A88B2D3
:102938000B0444BF00F5007080B2704770B5104CAE
:102948000025234626782EB166788E4202D1A678D5
:1029580096420BD001350C2D04F10404F2D1002469
:1029680013F824501DB101340C2CF9D170BD012588
:1029780003F8245003EB8403D87059709A70F5E774
:10298800810500202DE9F8430B460D795A7A9E7A85
:10299800DF7A204B097A1B5CDB07044600D50DB9AA
:1029A800FFF7CCFF00231C491A4898464FF0010E48
:1029B8009C4201F8018B25D02DB90278920702D5E7
:1029C80001F801EC1EE0154A4FF0000C92F8009057
:1029D800B9F1000F0FD092F8039099450BD1002E52
:1029E800EED092F80190B14505D1002FE8D092F8C9
:1029F8000290B945E4D00CF1010CBCF10C0F02F1C6
:102A08000402E3D10133DBB2042B00F10100CFD182
:102A1800BDE8F883B10500207D0500208105002070
:102A280007B503688DF807101B6901220DF107012E
:102A3800984703B05DF804FBF0B50546FD2305F89B
:102A48000C3B85B004468DF8043090F8243103F12E
:102A58000C020244012B42D80026637066808DF870
:102A680005308B7A23718DF808308B7AADF80660C3
:102A780001338B7263798DF80930A3798DF80A30A8
:102A8800A368C3F317031A128DF80B3009211B141E
:102A98000DF105008DF80D308DF80C20FFF746FB81
:102AA8006778ADF802003A4629460DF10200FFF7B3
:102AB80025FB94F82311FFF715FB94F82421BDF8A2
:102AC8000230A4F80C31974210D207F10C00D21B47
:102AD8003146204405B0BDE8F0400EF009BC12F8BC
:102AE800010D0028B8D1013BDBB2B3E705B0F0BD5A
:102AF80070470000044AD2F8903023F40043C2F82B
:102B08009030FFF79BBE00BF0004005808B5FFF7E0
:102B180095FE044AD2F8903043F40043C2F890304E
:102B280008BD00BF00040058064B1B7843B1064A95
:102B380000231380054A1380054A1380054A138031
:102B4800704700BF08000020863D0020883D002017
:102B58008A3F00208C3F0020054B1B783BB9054A73
:102B68001380054A1380054A1380054A138070476D
:102B780008000020863D0020883D00208A3F002074
:102B88008C3F0020074B084A5B6A02F5006353E854
:102B9800003F43F0200302F5006040E800310029BF
:102BA800F3D170470038014000300140064B1878D7
:102BB80040B1064B1888064B1B8880B29BB2C01ADE
:102BC80018BF0120704700BF08000020883D002082
:102BD800863D002070B5044608460D46FDF7D2FA3A
:102BE800236882B2294620461B69BDE87040184711
:102BF80008B5FFF7EFFF08BDB0F1904F02D10120F3
:102C0800FFF727BA084B984205D003F5806398422E
:102C180003D10420F4E70220F2E7044B984201D1E3
:102C28008020EDE7704700BF00040048001C004802
:102C38000C4B984203D14FF40060FFF722BAB0F171
:102C4800804F05D0084B984205D14FF40030F4E787
:102C58000120FFF70ABA054B984202D14FF48020B1
:102C6800EBE77047002C0140004401400048014058
:102C78002DE9F04387B00E4605461446002114227C
:102C880001A89DF838809DF83C901F460EF030FB57
:102C980000960B2C07D8DFE804F007070A12141473
:102CA800141616161A1CFEE70323019301E00223EB
:102CB8000493032F11D8DFE807F011132111012322
:102CC800F6E70123F1E7012301930393F1E70223D8
:102CD800EBE7022301930123F7E7FEE702230293C0
:102CE800B8F1100F0CD8DFE808F02D2D0C111315D2
:102CF80017191B1D1F21232527292B000123EEE768
:102D0800FEE701230593022301931EE00223F9E75E
:102D18000323F7E70423F5E70523F3E70623F1E7A1
:102D28000723EFE70823EDE70923EBE70A23E9E7A1
:102D38000B23E7E70C23E5E70D23E3E70E23E1E7A1
:102D48000F23DFE7B8F1000FDDD1B9F1000F02D092
:102D58002846FFF751FF053C042C05D8DFE804F0AE
:102D6800030B04030B00AE62694628460CF098F882
:102D780007B0BDE8F083AE61F6E713B54FF0010C7C
:102D88000024CDE9004CFFF773FF02B010BD00002E
:102D980007B50E48FFF78AF9036823F001030360BB
:102DA800436823F400434360036843F0010303606E
:102DB80000220823CDE90032042103230A224FF020
:102DC8009040FFF755FF03B05DF804FB0044004056
:102DD80030B587B0002315460446ADF80630FFF736
:102DE80027FF042D04D8DFE805F02E3204363F0013
:102DF800FEE71E4B1E4A1B68B3FBF2F39BB2002290
:102E0800CDE90221013B01A92046ADF80430049226
:102E180005920CF071FA236823F080032360A368FD
:102E280023F4A03323F00703A360636823F070033F
:102E38006360636823F470036360A36823F080030E
:102E4800A36007B030BD094B0A4A1B68D4E7074B9B
:102E5800094A1B68D0E7054B064A1B68B3FBF2F327
:102E680003EB83035B00C9E70123C8E7480200209E
:102E780080A8120140420F0000127A0010B50446E3
:102E8800FFF7A6FF236843F00103236010BD00226B
:102E98004FF0FF31FFF7F2BF1A4B10B51A4C5B68C1
:102EA80023600BF063F94FF090400BF0BBFF17481D
:102EB8000BF0B8FF16480BF0B5FF16480CF056FAA1
:102EC80015480CF053FA0CF049F94FF0E0220023B2
:102ED80013615361936172B64FF0FF319A0002F1AA
:102EE800604202F561420133082BC2F88010C2F833
:102EF8008011F3D162B6034B1B6883F308882368FB
:102F08009847FEE70000FF1F7805002000040048EE
:102F18000008004800380140004400400749084ABA
:102F2800881AEFF30883521A1A44013A013B98426F
:102F380088BF0022AA210EF0DBB900BF00000120E3
:102F480000040000044B5A69586910F0020018BFC9
:102F5800C2F38000704700BF000400584FF0B04231
:102F6800D2F8943043F40043C2F894304FF47A73A3
:102F780000BF013B9BB2002BFAD14FF0B043D3F80E
:102F8800942022F40042C3F89420D3F894205204E9
:102F9800FBD40C4BD3F8902022F40042C3F89020C5
:102FA8004FF47A7200BF013A92B2002AFAD1D3F8EC
:102FB800902042F40042C3F890204FF400629A61D6
:102FC800704700BF0004005810B5032305224021B4
:102FD8004FF09040FFF7D1FEBDE8104003230522D3
:102FE80080214FF09040FFF7C8BE08B5FFF7AAFF51
:102FF800003818BF012008BD08B5FFF7F6FF00B973
:1030080008BD00BFF9E74FF0904380229A62402242
:103018009A6170474FF0904340229A6280229A61E9
:1030280070470000024B4FF480225A60704700BF7F
:1030380000E100E010B5134C0323204606220421CA
:10304800FFF79BFE1048032302224FF40051FFF7BD
:1030580094FE03231A464FF400414FF09040FFF7C7
:103068008CFE2046032305224FF48071FFF785FE6E
:10307800BDE810400323052201214FF09040FFF7DF
:103088007CBE00BF00040048000800484FF0904391
:103098001869C0F3C030704708B5FFF7F7FF00B9EB
:1030A80008BD00BFF9E74FF0904301229A624FF440
:1030B8008072C3F818247047044B4FF480729A62E8
:1030C8004FF0904301229A61704700BF0004004806
:1030D80016484169F02321F0F00193FAA3F3B3FAFB
:1030E80083F3022203F00F0302FA03F30B43436155
:1030F8000F4BD3F8842022F40052C3F88420D3F86D
:10310800802022F40052C3F880205A6822F400522A
:103118005A601A6842F400521A60064BD02283F8AB
:1031280029234FF400725A60704700BF0000014025
:103138000008005800E100E0054B4FF40052DA6047
:10314800D3F8802042F40052C3F88020704700BFB3
:10315800000800580023032202214FF09040FFF797
:103168000CBE4FF09043186980F00200C0F3400095
:103178007047000010B5074C002320460522102197
:10318800FFF7FBFD20460023BDE81040052208217B
:10319800FFF7F3BD0004004805494B691A04DB43F7
:1031A80002F4801203F0100313438B61704700BFD1
:1031B8000004004805494B691A04DB4302F4002265
:1031C80003F0080313438B61704700BF00040048F5
:1031D80008B50322002302214FF09040FFF7CDFDF0
:1031E800102200234FF090410869800758BF01332F
:1031F80002F1FF3258BFDBB212F0FF02F4D1082B04
:10320800024A8CBF00230123137008BD0800002068
:103218000C4BD3F8FC2022F08072C3F8FC20D3F8C2
:10322800FC2042F08072C3F8FC20A3F55D431A68C5
:1032380022F001021A601A6842F001021A600022A4
:103248005A60704700ED00E00649074B074A1B68C3
:10325800B3FBF2F310B54C6843434A68121B9A4219
:10326800FBD310BD001000E04802002040420F00D0
:103278001FB50223CDE9013101A801236946039353
:103288000BF0DEF800280CBF0420052005B05DF81F
:1032980004FB014608B501200BF08CF800280CBF90
:1032A8000420052008BD08B5FFF7E2FF031F5842B8
:1032B800584108BD08B5FFF7ECFF031F58425841B5
:1032C80008BD00002DE9F047294B2A4D01280E467C
:1032D80014462949294A0FBF79277827AA461D4647
:1032E80006BF88469A4690460BF018F83946284695
:1032F800FFF7D9FF28B900240BF022F82046BDE8D3
:10330800F087002E08BF4FF4FC64073424F007044C
:1033180005F11007B1463444AAEB050AA1450BD1C3
:103328004FF011324FF0FF332846FFF7C3FF041E5A
:1033380018BF0124A400DFE76EB90AEB0703D3E93D
:103348000023B3F1FF3F08BFB2F1FF3F06D10837B2
:1033580009F10809E2E7D9E90023F2E7B84505D9F8
:103368003846FFF7A7FF0028F1D1C4E70324C3E7D5
:1033780000C0030800C80308FFCF0308FFC70308FD
:1033880010B50AF0CBFF09487821FFF78CFF0446F7
:1033980038B107487921FFF786FF041E18BF0124BA
:1033A800A4000AF0CDFF204610BD00BF00C00308EE
:1033B80000C8030830B5084D002340F2EF749AB2F4
:1033C800914201D8042030BDA34203D05A5DC254B3
:1033D8000133F4E70320F6E710C0030838B50446C4
:1033E8000D4672B60A4601460020FFF76BFF62B62B
:1033F800042806D172B601202A462146FFF762FF4B
:1034080062B638BD38B5124B1C68D3F80058B4F111
:10341800113F09D1B5F1113F17D000221146012003
:10342800BDE83840FFF74EBFB5F1113F03D1002288
:1034380011461046F4E7FFF7A3FF042804D12C40F7
:1034480001340CBF0220012038BD0420FCE700BF76
:1034580000C00308044B9A689107FCD518739A6852
:10346800D207FCD5187B70470000015870B50C4690
:10347800451E8E18B44200D170BD15F8010FFFF734
:10348800E9FF04F8010BF5E7084611461A46FFF76D
:10349800EDBF000070B5064E04464518A54200D1A0
:1034A80070BD3078FFF7D6FF04F8010BF6E700BFD0
:1034B8003C02002008461146FFF7ECBF38B5044629
:1034C8004518AC4200D138BD14F8010BFFF7C2FF14
:1034D800F7E708461146FFF7F1BF000010B58CB0BA
:1034E8002822002102A80DF003FF4FF0B0431C4C26
:1034F8005A6E42F001025A665B6E03F001030193B3
:10350800019BFFF72BFD082208924FF482720023DB
:1035180003924FF40072CDE90533CDE909330293E4
:10352800079207234FF4E06202A920460B93049206
:103538000BF0A8FE636823F010036360636823F050
:1035480008036360236843F040032360A3689B0774
:10355800FCD5237B034BFF221A700CB010BD00BFB3
:10356800000001583C020020034B18739A68D207E8
:10357800FCD5187B704700BF0030014038B5441EA9
:103588008D18A94200D138BD14F8010FFFF7ECFFE0
:1035980001F8010BF5E7084611461A46FFF7EEBF9A
:1035A80038B5064D04460144A14200D138BD2878FB
:1035B800FFF7DAFF04F8010BF6E700BF3D02002031
:1035C80008461146FFF7ECBF10B5014404468C428B
:1035D80000D110BD14F8010BFFF7C6FFF7E7084646
:1035E8001146FFF7F1BF000070B58CB02E4C2822B1
:1035F800002102A80DF07CFE4FF48050FEF741FD3B
:1036080001460323204606224FF48056FFF7B5FBF8
:103618000125A6610624CDE9004503230A222021BD
:103628004FF09040FFF724FBCDE9004503230A2221
:1036380031464FF09040FFF71BFB03231A46CDE9B4
:1036480000454FF400614FF09040FFF711FB08224E
:10365800164C08924FF48272002303924FF40072C2
:10366800CDE90533CDE909330293079207234FF4D7
:10367800E06202A920460B9304920BF003FE6368F4
:1036880023F010036360636823F008036360236812
:1036980043F040032360A3689B07FCD5237B044BBE
:1036A800FF221A700CB070BD0004004800300140C1
:1036B8003D0200201B4B10B4DC69A00611D51A6826
:1036C80091060ED5184819495A6A038809880133A2
:1036D800C3F30A0389B299421FBF1549D2B2CA542B
:1036E800038010481F232206036215D503681B06B2
:1036F80012D5104B104A1988138889B29BB2994287
:103708000CD013880133C3F30803138013880B4AC2
:103718009BB2D35CDBB2836210BC704710BCFEF76F
:10372800D7BC00BF00380140883D0020863D0020FE
:10373800863500208C3F00208A3F00208A3D0020EB
:103748000A490B4A08B50B8812880133C3F30803EA
:1037580092B29A4207D0074AD05407480B80FEF726
:103768009CFC012008BD0020FCE700BF8C3F002026
:103778008A3F00208A3D00200038014038B50446C1
:103788004518AC4200D138BD14F8010BFFF7D8FF3B
:10379800F7E70000034B1B78084611460BB9FFF703
:1037A800EDBF704708000020034B1B780846114600
:1037B8000BB1FFF7E3BF704708000020054B064A2E
:1037C8001B8810880133C3F3080380B2181A18BF86
:1037D800012070478C3F00208A3F002008B5044B29
:1037E800187820B1FFF7EAFFB0FA80F0400908BD69
:1037F8000800002008B5054B1B782BB9FFF7DEFF42
:10380800B0FA80F0400908BD0020FCE7080000205D
:10381800054B064A1B8812889B1A98B21B0444BFA2
:1038280000F5006080B27047883D0020863D00208A
:10383800024B187808B1FFF7EBBF7047080000206B
:103848000848094A0188138889B29BB29942F9D07D
:1038580013880133C3F30A0313801388034A9BB206
:10386800D05C7047883D0020863D002086350020CA
:10387800024B187808B1FFF7E3BF70470800002033
:10388800034B1B780BB9FFF7DBBF0020704700BF65
:103898000800002070B588B00C4606461546002181
:1038A800202268460DF024FD231E18BF01231B03A8
:1038B800CDE9023569460C23034801960494059323
:1038C8000BF078FD08B070BD0038014010B5064C0B
:1038D800236823F001032360FFF7DCFF236843F02C
:1038E8000103236010BD00BF00380140044B1B7862
:1038F80008461BB100221146FFF7E8BF704700BF1A
:103908000800002000221146FFF7E0BF73B5304CD5
:10391800236823F001032360082501264FF4804023
:10392800FEF7AFFB4021CDE900562A4803230A22BF
:10393800FFF79EF903231A46CDE900562548802152
:10394800FFF796F9002211464FF4E130FFF7A2FF86
:10395800636823F490436360A36823F02A03A36099
:103968001D4BB02283F8242310225A602046FEF70C
:10397800AFFBFEF7A4FB40232362184B00211980FC
:10398800174B1980FEF792FB164B1980164B1980BE
:10399800636823F400636360A36823F00803A360EB
:1039A800636823F480436360A36823F02203A36061
:1039B800A36843F48053A360236833432360E36917
:1039C8009A02FCD5E3695B02F9D502B070BD00BF6D
:1039D800003801400004004800E100E08A3F002070
:1039E8008C3F0020863D0020883D002008B5FFF769
:1039F8008DFFBDE80840FFF7C5B8000008B5FFF720
:103A0800F5FFFFF7E5FB054B1B782BB9BDE8084030
:103A18004FF4E130FFF776BF08BD00BF0800002073
:103A2800024B1A68024B1A60704700BF9C3F002087
:103A3800980A0020054A064B1968136899421DBF69
:103A48000133012013600020704700BF980A00204E
:103A58009C3F0020034A044B11681B780B441360F9
:103A6800704700BF9C3F00204C020020014B1868A3
:103A7800704700BF9C3F00200148FFF708BA00BF0D
:103A880000440140014B586A80B27047004401402D
:103A980008B5FFF7F1FFBDE80840FFF7C1BF000018
:103AA800F8B51A4C1A4F90220021201D0DF020FC69
:103AB8001623062663800F23A38032462C2339461B
:103AC800A0192680FDF772FD124A134B0025C4E9A0
:103AD8000D2339462C23324604F13E00A587FDF715
:103AE80065FD1F23E3660D4984F87250012304F134
:103AF8007C00A4F87030C4E91D550DF059FC7F23F3
:103B080084F89130052384F89230F8BDE40400204D
:103B1800602801081F000F0003000500DC150108DC
:103B280070B5094E05460C46415C30460DF0F7FB72
:103B3800034628B1831B0133DBB2282B28BF00239F
:103B4800F35C2B5570BD00BF582F010870B50C46AB
:103B5800114606460DF02CFC44B1002505213046DF
:103B68000135FFF7DDFFEBB29C42F7D870BD0000CE
:103B7800F7B5054605F11106214C224A01463601E2
:103B88006846FFF7E3FFB01C694620440DF010FCBF
:103B9800264404EB0512002302277772A2F81A3193
:103BA800142202FB05400421012280F850104FF432
:103BB800807540F20111A0F84A70C264A0F8522042
:103BC80080F85520A0F85650A0F8581040F203206D
:103BD80084F83430E784A562A08584F82E2084F820
:103BE800302084F83330C4F83A30C4F83E30C4F892
:103BF8004230A4F84610A4F8481003B0F0BD00BF46
:103C0800280300209C150108F7B50546AF4CB04ABB
:103C180005F11106014637016846FFF797FFB81C02
:103C2800274469462044FDF7BDFB7B7AA94A052B4A
:103C380088BF022304EB061088BF7B721188437A81
:103C480041FA03F3DF070FD40223437261B1480737
:103C5800C1F3800308D441FA03F7FF07D8B240F153
:103C6800D18104EB0613587204EB05112B0191F86E
:103C78001A01052802D9002081F81A01E71850888E
:103C880097F81A1140FA01F1C90711D4012187F8F0
:103C98001A1168B18707C0F3400109D440FA01FC42
:103CA8001CF0010FCFB200F0B281E11881F81A714F
:103CB800E11891F81B01032802D9002081F81B01A3
:103CC80004EB0616717A012903D9042901D00021D1
:103CD8009180E618908896F81B1140FA01F111F0CE
:103CE80001010ED186F81B1158B110F0010108D15D
:103CF80040FA01F7FF07CEB240F18E81234483F8E2
:103D08001B61142303FB054191F84A00052802D9D9
:103D1800022081F84A0003FB054393F84B1004295D
:103D280002D9002183F84B10142303FB0543918E1D
:103D380093F84B0041FA00F0C00712D4012083F831
:103D48004B0071B18807C1F340030AD441FA03F666
:103D5800F707D8B240F16581142303FB054383F8C4
:103D68004B00142303FB054393F84C10032902D995
:103D7800012183F84C10142000FB0540D18E90F8E7
:103D88004C3041FA03F313F0010310D180F84C30A2
:103D980069B111F001030AD141FA03F6F607D8B266
:103DA80040F14481142303FB054383F84C0014239A
:103DB80003FB054393F84E10012902D9002183F82B
:103DC8004E10142000FB0540118F90F84E3041FA38
:103DD80003F313F0010310D180F84E3069B111F0EC
:103DE80001030AD141FA03F6F707D8B240F123815B
:103DF800142303FB054383F84E00142303FB0543F8
:103E080093F84F10022902D9002183F84F1014208B
:103E180000FB0540518F90F84F3041FA03F313F03F
:103E2800010310D180F84F3069B111F001030AD1B4
:103E380041FA03F6F607D8B240F10281142303FBD6
:103E4800054383F84F00142303FB054191F84D0007
:103E5800022802D9002081F84D0003FB054393F89E
:103E68005010052902D9042183F85010142303FBAC
:103E7800054191F85200012802D9012081F8520029
:103E880003FB054393F85510012902D9012183F852
:103E98005510142303FB054393F85310022902D944
:103EA800002183F85310142000FB0540918F90F8EF
:103EB800533041FA03F313F0010318D180F853305B
:103EC800A9B111F0010312D106E000BF28030020B8
:103ED8009C150108E404002041FA03F6F707D8B25C
:103EE80040F1B380142303FB054383F853001423E4
:103EF80003FB054191F856000C2802D9002081F8EF
:103F0800560003FB054393F84C10012906D193F89A
:103F18004F10022904BF002183F84F10142303FB1C
:103F28000543012183F8571040F20111A3F85810F6
:103F380094F82630052B02D9022384F8263094F809
:103F48002730042B02D9002384F82730B2F86C00FC
:103F580094F8273040FA03F313F0010F804B0ED189
:103F6800012184F8271050B18607C0F3400106D418
:103F780040FA01F7FF07CEB26CD583F8276094F8B2
:103F88002810022902D9002184F8281094F8291051
:103F9800022902D9012184F82910B2F86E1094F888
:103FA800292041FA02F212F001020CD184F82920EA
:103FB80049B111F0010206D141FA02F6F607D0B272
:103FC8004CD583F8290094F82A200C2A02D900221B
:103FD80084F82A2093F832200C2A02D9002283F888
:103FE800322093F82B20042A02D9002283F82B20B0
:103FF80000225C49104611F9014F14F1780F31DAAB
:10400800087031E00133102B7FF425AE2CE6013126
:1040180010297FF443AE4BE6013110297FF468AED6
:104028006FE60133102B7FF491AE9AE60133102B23
:104038007FF4B2AEBBE60133102B7FF4D3AEDCE6DF
:104048000133102B7FF4F4AEFDE60133102B7FF41F
:1040580043AF4CE7013110298AD190E70132102A89
:10406800AAD1B0E7782CCBDC0132D2B20C2AC2D16B
:104078003D490022012011F8014F0132022CD2B231
:1040880088BF0870042AF6D193F83420012A02D98F
:10409800002283F83420354AB2F8701093F834209F
:1040A80041FA02F212F001020CD183F8342049B12E
:1040B80011F0010206D141FA02F4E407D0B211D599
:1040C80083F8340093F82C20052A02D9032283F8B8
:1040D8002C2093F82D20032A08D80AD1002283F82F
:1040E800342006E00132102AE5D1EBE7022283F8FA
:1040F8002D2093F82E20022A02D9012283F82E209F
:1041080093F83020022A02D9012283F8302093F84C
:1041180033200C2A02D9002283F83320142101FB12
:104128000531FF2203EB05154FF6FF7081F851208A
:1041380081F8542083F82F2083F831204FF0FF3284
:10414800C5F81C21A5F820011A629A84A1F85A2002
:10415800A1F85C2083F83500DA861A8703B0F0BD31
:1041680028030020610300206D030020E4040020E0
:1041780030B5052804D8DFE800F01E0423191E23F3
:10418800FEE720251F2400220F21104B98700338CA
:10419800012894BF002001201A7119771A74A3F816
:1041A8004850A3F84A409873987630BD09256F2483
:1041B80000220721E9E71425322400220A21E4E736
:1041C8003525132401221921DFE700BFCC02002086
:1041D8002DE9F743A64FA74C00F1110907EB091881
:1041E80008F1020806464046FDF7F8F8042105469E
:1041F80001900DEB0100FDF799FF142303FB0673F3
:10420800E08393F84B00A5606561042804D8DFE8D3
:1042180000F03A3E04093500FEE7002301221D465E
:10422800114603E001231A461D46002107EB091930
:1042380084F8523099F80930637007EB061384F854
:10424800510093F81A0184F8532084F8545084F8E4
:104258005510FFF78DFF142303FB0673350193F800
:104268004A20854B13F92230237323766378052B74
:1042780012D8DFE803F00F5F6163656701231A4610
:1042880000251946D2E701231A461D46F9E70123FE
:104298000022C4E700236373784B617B1B88617637
:1042A80003F00102980748BF42F00202A2855A07AC
:1042B80048BFA28D84F8281044BF42F00402A285AA
:1042C800180742BFA28D42F01002A285DA0642BF4B
:1042D800A28D42F02002A285980642BFA38D43F02A
:1042E8000803A385002384F82A3021B94046FDF746
:1042F80095F884F82A003D4495F81B2184F8292074
:104308006AB1E18B02EB021303EB03230B44E38353
:10431800A3684FF0113101FB0233A360636194F885
:104328002850E38B6362052D0ED8DFE805F00E53A5
:104338005517494B0123AEE70223ACE70423AAE74C
:104348000523A8E70323A6E7FEE7A378032B03D8F2
:10435800DFE803F003464403FEE71825DFF820C131
:1043680084F820501CE90F008CE80F0040F2E2436B
:104378002846A4F84C30FCF7B5FB4FF07F51FCF70A
:1043880005FCFCF705FEB4F848204FF47A73B3FB3C
:10439800F2F3A4F84030142303FB06736D08052DCF
:1043A80093F85030C0B238BF0525A4F84E0084F801
:1043B8005050052B3DD8DFE803F0154236393C3F15
:1043C8000225CBE7A378022B08D0052B06D0012BBA
:1043D80006D0FEE71925C1E70625BFE70C25BDE78E
:1043E8001225BBE74FF416536364002384F8563054
:1043F80084F85830142303FB067696F84C20032AD9
:1044080003D096F84F30022B02D1012384F856309E
:10441800511E4B424B4194F8561084F8573089B1DD
:10442800012A0FD1FEE74FF41643DDE74FF461434D
:10443800DAE74FF4E133D7E74FF46133D4E74FF4C9
:104448009643D1E72378142000FB037393F84C308C
:10445800022B07D1012384F8583021B194F8583041
:104468001BB1FEE709B9012AF8D003B0BDE8F08313
:1044780028030020CC02002060280108E404002062
:10448800FC02002002484FF4DE72FF210CF030BF1E
:104498002803002002484FF4DE71FEF79FBF00BFDB
:1044A8002803002002484FF4DE71FEF783BF00BFE7
:1044B8002803002008B5FFF7F5FF034B1878BDE87F
:1044C8000840FFF7A1BB00BFCC02002038B5FFF7BA
:1044D800D9FFFEF797FF04280CD0FFF7D3FFFEF7AC
:1044E80091FF042803D1FFF7DDFF042806D0FFF76A
:1044F800C9FF03E0FFF7D6FF0428EED12F49304863
:104508002F4C10220CF018FF38B12E4910222046EB
:104518000CF012FF08B1FFF7B5FFA38AB3F5215FCE
:1045280028D008D30025E8B20135FFF721FB0A2D72
:10453800F9D10023E3774FF42153A382012522699F
:104548001E491F4842F642039A424FF010021CBF10
:10455800236101250CF0F0FE70B1184918481022AB
:10456800FDF7A2F8184919480822FDF79DF8FFF74A
:1045780091FF03E00025E2E7002DF8D1E37F104A20
:10458800092B84BF0023E377E17F1420002300FB7D
:104598000144013394F84C0082F84C000A2B02F1D4
:1045A8001402F6D10A4C2170FFF77AFA2078FFF747
:1045B8002BFB2078BDE83840FFF70ABEA315010899
:1045C80028030020B4150108C5150108DA040020E5
:1045D800CC02002030B5C01A1628A8BF16206FF0EC
:1045E8000805A8429DF80C40B8BF2846A042C8BF9D
:1045F80020B2C0B208701844107030BD07B5084624
:1046080011461A46162300930023FFF7E3FF03B071
:104618005DF804FB07B5084611461A4616230093B1
:104628000023FFF7D7FF03B05DF804FB0129F7B5B6
:10463800054600D9FEE70B4E06EB01131C460F0199
:104648006278F15D03619B780BF0C6F9E379019319
:10465800A379009322796379E17828460BF0E3F98E
:1046680003B0F0BD24450108836810B5044603B9BA
:10467800FEE700210BF072F94FF47A70FEF7E4FDC3
:10468800204601210BF081F9A36820461978FFF72D
:10469800CDFF10BD38B5836804466BB1024652F8A9
:1046A800183BDD6900F11903A847217E2046022244
:1046B800BDE838400BF019BA38BD000070B581600C
:1046C800897A86B0044601B101210BF05EF92046D3
:1046D8000BF0EDFA20460BF0C5FA217BFF2903D039
:1046E800FA2220460BF0CAFAA3685B7A013B042B36
:1046F80004D8DFE803F0043E3E414100FEE7E9222A
:10470800E12120460BF0F8FA012120460BF087FA48
:10471800962120460BF0C4FA382120460BF0D6FA31
:1047280020460BF0DBFAA368204693F90810FFF740
:10473800B1FFA3689D7A15B319782046FFF776FF75
:104748000022114620460BF03AF90023009340F26C
:10475800032220464FF6FF710BF094F920464FF6DE
:10476800FF710BF0B6F9204606B0BDE870400BF0BB
:1047780066BADB22D721C4E76F226B21C1E70F4B52
:104788000F49DE8B0F4B63614CF250330093204688
:1047980019230B220BF0C0FA0123CDE903335B2365
:1047A800CDE90153102319462046009504220BF049
:1047B800F1FA314620460BF011FBC1E7CC0200208C
:1047C800A08601000445010873B504460D46164647
:1047D8000DF107010DF106020BF0E0F99DF8061046
:1047E80033462A4620460BF08AF802B070BD38B529
:1047F80004461D4613460A4600210BF059F8204688
:104808004FF6FF710BF065F9A9012046BDE8384065
:104818000BF078B910B504460BF011FA20464FF6A4
:10482800FF71BDE810400BF054B9836873B50D46AD
:10483800144623B981220A70237002B070BD9E7A93
:104848000DF10601B6B10BF093F994F90030002B85
:1048580004DABDF806201344ADF80630BDF9063079
:10486800002B0BDB4FF6FF73ADF80630BDF80630B2
:104878002B70E2E70BF0C3FA2670EFE77F33F5DA27
:104888004FF68173F0E7000038B58168036891F945
:104898000810DD69044600F1190300F11802A84761
:1048A800A3689A7A42B11A78012A00D9FEE7044B24
:1048B80003EB0213236138BD024B6361FBE700BFC2
:1048C800244501080445010810B50A4CA06858B1F0
:1048D800236923B9636913B92046FFF7D5FFA36895
:1048E8009B7A23B123699868A0F57A7010BD636933
:1048F8009869F9E764300020836810B5044683B1ED
:1049080003691BB943690BB9FFF7BEFFA3689B7A1C
:104918001BB12369B3F90C0010BD6369B3F91C001E
:10492800FAE71846F8E7836810B5044643B1036907
:104938001BB943690BB9FFF7A7FF94F9190010BD1C
:104948001846FCE790F8D8305BB190F8D930074AA0
:10495800180102EB03139B681978135853F82100C8
:104968007047837D0E3350F82300704700280108F4
:104978002DE9F3419DF824701646402F88464FF0E4
:104988005B024FF0000104461D4628BF40270CF08B
:10499800AFFC904BDB8B23803278A37862F3020361
:1049A800A3707178C90001F00801DBB203F00703B6
:1049B80041EA08111943A1707279E37862F30003A0
:1049C800E370B279637962F38613637196F9020032
:1049D800FCF715FCE37860F34703E370F279237979
:1049E80062F300032371327A62F34603237132794A
:1049F800DBB202F0010203F07F0343EAC213237122
:104A080032796379C2F3450223F03F03134363719C
:104A1800A37967F34703A3712B78AA78E3716B78BE
:104A280002F01F0203F0070343EAC20323726A88F5
:104A3800637AC2F3451223F03F03134363722A7962
:104A4800DBB202F0030203F03F0343EA821363720E
:104A5800AB88C3F38703A3726A79E37AC2F380024F
:104A680023F001031343E372AA79DBB202F07F0259
:104A780003F0010343EA4203E372EA88237BC2F3AB
:104A8800C31223F00F03134323732B7AAA7AE37319
:104A98006B7A02F01F0203F0070343EAC203237490
:104AA8006A89637CC2F3451223F03F03134363749E
:104AB8002A7BDBB202F0030203F03F0343EA8213CE
:104AC8006374AB89C3F38703A3746A7BE37CC2F383
:104AD800800223F001031343E374AA7BDBB202F0E4
:104AE8007F0203F0010343EA4203E374EA89237D6A
:104AF800C2F3C31223F00F03134323752B8ADB0879
:104B080063756B8ADB08A375AB8ADB08E375EB8AF0
:104B1800DB0823762B8BB3F5C06F4ED2B3F5007F3D
:104B280094BF00230123227B63F3051222736B8B4E
:104B3800B3F5C06F43D2B3F5007F94BF00230123C0
:104B4800227B63F387122273AB8BB3F5C06F38D225
:104B5800B3F5007F94BF00230123227D63F3051280
:104B68002275EB8BB3F5C06F2DD2B3F5007F94BFE0
:104B780000230123227D63F38712089B22751F44BB
:104B880004F11802BB4220D14FF6FF7321460DF104
:104B980006000D22ADF80630FDF7B0FA2146BDF843
:104BA800063021F80D3F4C22FDF7A8FABDF8063073
:104BB800A4F8593002B0BDE8F0810223B3E702231C
:104BC800BEE70223C9E70223D4E713F8011B02F862
:104BD800011FD7E7CC02002013B59DF81040CDE99E
:104BE800003413460A460021FFF7C2FE02B010BD8A
:104BF80013B5144B0288DB8B9A4204461DD1837887
:104C080003F0F003102B01D0202B18D1A379A52B8A
:104C180015D84FF6FF730DF1060059222146ADF85D
:104C28000630FDF76BFAB4F85900BDF80630C01A23
:104C380018BF0120800002B010BD0120FBE7022050
:104C4800F9E700BFCC02002030B5374B027893F863
:104C5800261061F30302027093F8271061F307121C
:104C6800027093F82810427861F30302427093F8B7
:104C7800291061F30712427093F82A10827861F3C1
:104C88000302827093F83210827961F30302827111
:104C980093F82B10827861F30712827093F834101E
:104CA800C27961F30302C27193F82C10C27861F3E0
:104CB8000302C27093F82D1061F30712C27093F8C3
:104CC8002E10027961F303020271427993F83010D1
:104CD80061F30302427193F83310827961F307128A
:104CE800827103F1390100F10A0200F1160411F989
:104CF800015F02F8015FA242F9D193F84610C27D24
:104D080061F30102C27593F8471061F38302C2751B
:104D180093F8481061F30512C27593F8493063F3AC
:104D28008712C27530BD00BF280300200278314BBE
:104D3800C2F3030230B583F826200278C2F30312C7
:104D480083F827204278C2F3030283F828204278A8
:104D5800C2F3031283F829208278C2F3030283F88E
:104D68002A208279C2F3030283F832208278C2F3C0
:104D7800031283F82B20C279C2F3030283F834208C
:104D8800C278C2F3030283F82C20C278C2F303125C
:104D980083F82D200279C2F3030283F82E2042798A
:104DA800C2F3030283F830208279C2F3031283F836
:104DB800332003F1390100F10A0200F1160412F957
:104DC800015F01F8015FA242F9D1C27DC2F301027D
:104DD80083F84620C27DC2F3810283F84720C27D52
:104DE800C2F3011283F84820C27DC2F3811283F80E
:104DF800492030BD280300201FB58DF80C30012351
:104E0800019303AB009313460A460221FFF7B0FD56
:104E180005B05DF804FB0000F0B5224D012385F8CC
:104E28007230044685B0B0F80900FCF7E4FB686707
:104E3800B4F80B00FCF7DFFB1422A86704F10D019E
:104E480005F17C00FCF742FC94F9213085F891309B
:104E580094F8223085F8923004F12300FFF766FFBA
:104E68006E4604F1410304F1510718685968324647
:104E780003C20833BB421646F7D10B482C2308223D
:104E88006946FCF715FB94F85130A5F86C3094F896
:104E98005230A5F86E3094F85330A5F8703005B04C
:104EA800F0BD00BFE4040020220500202DE9F047F2
:104EB80092B0DFF890A0244C0DF108084FF040099B
:104EC80005460E46174600214A4640460CF010FAA1
:104ED8009AF8001004EB011122230DF10A000622B2
:104EE80001F589718DF80830FCF7DEFB9AF800109F
:104EF80004EB011205A892F81A3192F8194103F04F
:104F08000F0304F00F0444EA031492F81B3103F072
:104F18000F0344EA0324BDF8103023F47F6323F021
:104F28000F031C43ADF81040FFF78EFECDE9008952
:104F38003B46324602212846FFF71AFD12B0BDE86B
:104F4800F08700BFCC02002028030020034B04494F
:104F58001A68044801FB020018607047B805002071
:104F68000D6619005FF36E3C38B50A4A0A4D13788E
:104F78002C78A34203D101332B70287838BD1470E4
:104F8800FFF7E4FF6FF0004398423CBF01342C70F8
:104F9800F3E700BFB5050020B60500200A4A1268ED
:104FA80082600A4A002383808371838103841368A3
:104FB80003615368064A4361136883615368C36198
:104FC8004EF66023036070479C3F0020CB15010814
:104FD800D415010838B5114D114C0220FFF7C8F857
:104FE8002846FFF717FC2046FFF714FC28466FF009
:104FF8007F01FFF74FFB6FF07F012046FFF74AFB69
:105008002846FFF731FB2046FFF72EFB2846FFF71F
:1050180001FC2046FFF7FEFB38BD00BF64300020CE
:105028008030002008B590F8203002468BB9FEF792
:1050380098F810B982F8210008BD92F821300133A0
:105048005BB2312B82F82130F6DD012382F8203063
:10505800F2E7FEF786F818B1322382F82130EBE741
:1050680092F82130013B5BB2002B82F82130D8BF87
:1050780082F82000E0E70000134B90F820201B681E
:10508800CAB182689B1AB3F57A6F01D901234371BB
:105098000379ABB10D4B427B1B781AB1022B1CBFB5
:1050A800032202739A1E534253414373837953B1C7
:1050B8000323037370478360EAE701230371F8E76A
:1050C8004379002BF9D170479C3F00208D060020C2
:1050D8000346007B821E012A4FF0000202D893F893
:1050E800201009B91A7370471046704770B51B4CE9
:1050F8001B4E05465B22002120460CF0F9F82B696F
:1051080023606B696360174B174D1B7831789A1EC3
:1051180053425341627A05EB011163F30002627254
:1051280001F58971062204F10A00FCF7BDFA33780B
:1051380005EB0315237C95F81A2162F307132374F2
:1051480095F81B21637C592162F30303204663749D
:10515800FCF7ECFFA4F8590070BD00BFC530002073
:10516800CC0200208D060020280300200A4A38B50A
:10517800138801339BB2502B04460D4601D8138087
:1051880038BD002305491380FDF724FD2946204634
:10519800FDF720FDF4E700BF9C0A0020FC1601087B
:1051A8002DE9F84F154604460F466B496B4EFDF73F
:1051B80011FD29462046FDF70DFD694B0022012F00
:1051C8001A800FD11023B362082746F2A810B761DE
:1051D800FEF73AF8B762FEF737F829462046FFF798
:1051E800C5FFF2E7BB1E08220C2B00F2A880DFE8FF
:1051F80003F03141521C07A6A6A6626262626200F1
:10520800564E4FF008081027C6F8188046F2A81026
:10521800B762FEF719F8C6F82880B761FEF714F8E8
:1052280029462046FFF7A2FFEDE74C4E4FF008084D
:105238001027C6F8188046F2A810B761FEF704F8E0
:10524800C6F82880B762FDF7FFFF29462046FFF71A
:105258008DFFEDE7B262414E102746F2A810B76104
:10526800FDF7F2FFB762FDF7EFFF29462046FFF78B
:105278007DFFF2E71023B361384E082746F2A810E5
:10528800B761FDF7E1FFB762FDF7DEFF294620466B
:10529800FFF76CFFF2E7B261304E102746F2A81014
:1052A800B761FDF7D1FFB762FDF7CEFF294620466B
:1052B800FFF75CFFF2E7A7F1090BDFF8A0805FFAC0
:1052C8008BFB00264FF0080A5E453CBF1023C8F848
:1052D80018304FF0040946F2A810C8F818A0FDF7D6
:1052E800B3FFC8F828A0FDF7AFFF09F1FF39294639
:1052F8002046FFF73BFF19F0FF09ECD11023C8F84F
:1053080028304FF0040946F2A810C8F818A0FDF795
:105318009BFFC8F828A0FDF797FF09F1FF39294638
:105328002046FFF723FF19F0FF09ECD10136A7F15A
:105338000803F6B2DBB2B34238BF0026C4E7102335
:10534800B261B3614CF25030FDF77EFF294620462A
:10535800FFF70CFFF6E700BFFC1601080004004841
:105368009C0A002010B514461A4618B90348FFF7DE
:105378002BFA10BD02482146F9E700BF643000202F
:105388008030002038B514461D4668B9FDF73BFE4D
:105398000B482B462246FFF72AFA7D20FDF754FFDB
:1053A8000848FFF737FA38BDFDF77DFE05482B465C
:1053B8002246FFF71CFA7D20FDF746FF0048F0E77C
:1053C800643000208030002008B530B9054801F16C
:1053D8008E028C31FFF729FA08BD01F18F020248CD
:1053E8008D31F7E7643000208030002070B5114C13
:1053F8000D4606465B23224621462846FFF7B2FFA4
:10540800D6E90613206862689A4208BF88420ED11E
:1054180020465921FCF78AFEB4F85940231A5C4209
:105428005C4128460449FFF7CFFF601C70BD00248B
:10543800F7E700BFAB2E0020BC2F00200A4608B5B6
:1054480001460148FFF7ACFE04000020002303706A
:105458008370437003714371C370704703780022EF
:10546800022B427104D0032B09D0012B16D0FEE782
:1054780001230371437183784370C3707047837845
:105488004278991AA3EB020218BF012112F0060F05
:1054980014BF0122002201714271EDE702717047C9
:1054A80002788170002A0CBF022203220270FFF7E3
:1054B800D5BF000010B5437802789A421BD0052B5F
:1054C8008ABF052303700370027888BF43700A4BB4
:1054D8000A4813F922100A4C83682173217613B104
:1054E8001972FFF7D7F80748836823B194F91810A1
:1054F8001972FFF7CFF810BD60280108643000204A
:10550800CC0200208030002010B50AB9437010BDCD
:10551800541E0B2CFBD80332D2B231F8122040F2C1
:105528007E618A4203D95AB222EAE2721AE0B2F5DF
:10553800C17F02D29A1E52B2F6E740F2A9518A42BE
:1055480004D95AB2052A1CDCDA1EF4E740F25621C7
:105558008A4218D940F2D4418A4208D95AB2042A58
:10556800F2DD02229A42C8BF5AB24270CFE7B2F5C2
:105578004B7F04D25AB2032AE6DD0122F2E75A1E13
:10558800D9E70322EEE70022ECE70000074B2822C8
:1055980002FB00339B681A78542A05D15878A0F189
:1055A800780358425841704700207047782801080E
:1055B800074B282202FB00339B681A78522A05D130
:1055C8005878A0F178035842584170470020704736
:1055D80078280108074B282202FB00339B681A78B9
:1055E800542A04D15878783818BF01207047012010
:1055F800704700BF7828010828230B4A434310B599
:10560800D1580446FFF7D4FF48B92046FFF7BEFF3C
:10561800064B1B7828B103EB830301EB8301084693
:1056280010BD01EB0311FAE778280108CC0200202D
:105638002B2838B505461AD80E4B282202FB003312
:105648004CB21B79022B0DD0FE2B10D1FFF7D4FFE3
:105658000378E4B2A3420AD004702846BDE8384073
:10566800FFF7B8BFFFF7C8FF90F90030F2E7002056
:1056780038BD00BF782801082B2838B504460D46E8
:1056880019D80E4B282202FB00331B79FF2B12D1AD
:10569800FFF7B2FF06222946FCF72BF858B9204637
:1056A800FFF7AAFF29460622FCF710F82046BDE8B6
:1056B8003840FFF78FBF002038BD00BF78280108A9
:1056C8002DE9F043074615462820394A414350182A
:1056D800012B046A87B025D15258364B9A4235D0EF
:1056E800A3F1CE018A4233D03349F23B9A4208BF34
:1056F8000C46FF238DF800304FF0000801262046A5
:10570800FAF740FD5FFA88F9484529D806F11803E9
:105718006B44AE4203F8188C30D80020387007B0BC
:10572800BDE8F083022BE4D15258224B9A4211D0A3
:10573800591C8A4210D0A3F1CE018A420ED0A3F19F
:10574800F2018A420AD01D49EC3BCFE71C4CD0E756
:10575800194CCEE71B4CCCE71B4CCAE71B4CC8E7DF
:1057680014F809302C2B06D106F118036B440136C6
:1057780003F8188CF6B208F10108C0E705F1180320
:105788000DEB0305002315F8182C15F9175C0132E9
:10579800D2B29918C9B2A94207EB030003DB002370
:1057A80003700120BBE7615C01700133DBB2F0E7F5
:1057B8007828010841040020DD15010811160108A8
:1057C8002E160108B316010891160108671601087C
:1057D800054B282202FB00335B6A0BB1188870471F
:1057E8004FF6FF70704700BF782801080B4B28223E
:1057F80002FB003370B51E6A3046FAF7C3FC00227C
:1058080001461446D5B2631CA942D8B200D870BD6F
:10581800735D01322C2B08BF0446F3E77828010892
:105828000F4B282202FB003310B51B79FE2B0146D3
:1058380014D1FFF7CDFF04460846FFF7D7FF002233
:1058480001461046D3B2994200D810BD44FA02F37B
:10585800DB0744BF431CD8B20132F3E7FF20F4E76B
:10586800782801082DE9F04F4FF0000A1D4E93B03B
:1058780004460F46D146D6F808805FFA8AF54FF0FD
:10588800000B0DE018F8030001920BF00DFDC3B2F8
:10589800019A202B08BF5F2302F8403C0BF1010B53
:1058A8005FFA8BF340460193FAF76CFC019B03F116
:1058B800480298426A44E5D802F8409C394602A852
:1058C800FAF756FC48B10AF1010ABAF12C0F06F1B1
:1058D8002806D0D10025284600E00120257013B005
:1058E800BDE8F08F782801082DE9F0411D4E2823E6
:1058F80003FB016604463379FE2B0D46174618D084
:10590800FF2B21D0022B28D10846FFF775FE214630
:1059180090F9000009F0CDFE35692B783BB11249AA
:1059280020460BF0EDFC294620460BF0E9FC01204F
:1059380015E00846FFF760FE3B46027829462046F8
:10594800BDE8F041FFF7BCBE0846FFF755FE06224A
:1059580001462046FBF7BAFEE9E700202070BDE8C3
:10596800F08100BF78280108F3170108F8B5194B32
:105978001646282202FB063300241A790470022AEC
:1059880007460D4603D0FE2A13D02046F8BD93F9EA
:1059980018209142F9DB93F91C309942F5DC4FF05D
:1059A800000165F307013046FFF742FE0124387015
:1059B800EBE70029E9DB3046FFF718FFA842E4DDF2
:1059C8003046FFF705FF40FA05F313F00100E6D172
:1059D8000446DAE7782801082DE9F8430023037024
:1059E800124B1746282202FB073306461B79FF2B6A
:1059F8000C4603D000252846BDE8F8830846FAF788
:105A0800C1FB0628F6D104F1FF3804F1050918F89E
:105A1800010FFBF7ADFC05460028EBD0C845F6D1D1
:105A280021463846FFF728FE3070E4E77828010859
:105A3800F8B5104E4FF0280C0CFB0266002736799B
:105A48000770FE2E04460B46154603D0FF2E0BD0DA
:105A5800022E0DD118460BF093FB2A46014620462C
:105A6800BDE8F840FFF782BFBDE8F840FFF7B4BFD4
:105A78003846F8BD7828010810B504460846B2B97A
:105A8800FBF7CCFC042812D8DFE800F003090B0D63
:105A98000F00084920460BF08BFC012010BD064979
:105AA800F8E70649F6E70649F4E70649F2E7002071
:105AB800F4E700BFE0160108E5160108EA16010838
:105AC800EF160108F516010810B504460068FDF741
:105AD80081F802492068FDF77DF810BDFB16010822
:105AE8000B1E18BF0123122A14D91D2A14D9312AD2
:105AF8008CBF0822052203710023016080F88530DD
:105B08004371C0F8883080F88C3080F88D20A0F878
:105B18008E3070470122EEE70322ECE790F88530DB
:105B2800642B08D8C2180133DBB2517180F8853074
:105B3800184400234371704708B50530FAF718FB7D
:105B4800B0FA80F0400908BD2DE9F043064691B04F
:105B5800084688461546FAF715FB06F10509044676
:105B68004846FAF70FFBE4B2631CC7B2BB4203DB3B
:105B7800002011B0BDE8F0832246414648460BF0AC
:105B8800DBFB0028F4D1231D22461E44BA420346FB
:105B98001BD300F140036B44002403F8404C002859
:105BA800E6D09DF800303D2BE2D1302368468DF8D1
:105BB8000030FAF7E7FA2346DAB2904212D868467C
:105BC8000BF0DEFA28600120D3E716F8011F202920
:105BD80005D040336B440130C0B203F8401C013299
:105BE800D2B2D3E740326A44013312F8402C303A3B
:105BF800092AE1D9BCE7000010B50D4B1B78022B30
:105C080004460ED10B4B93F8722052B19B6FB3F53B
:105C1800215F07D20849FFF757FF08492046FFF7D9
:105C280053FF10BDFDD00649FFF74EFF0549F5E7C4
:105C38008D060020E4040020FE1601083417010830
:105C48006A170108A017010810B50446FFF7D4FF2A
:105C580020680749FCF7CCFF064B206819783031DB
:105C6800C9B2FCF7DDFE04492046FFF72DFF10BD41
:105C7800D6170108CC020020DC1501082DE9F047F1
:105C88004379702B90B080460F46164671D18379C0
:105C9800202B6ED1C0790BF0FFFA00285CD00025CC
:105CA8004FF0020A2C4608F105094846FAF76AFA45
:105CB800824522D305F140030DEB0305002305F8C7
:105CC800403CC4B3E8461D4618F8010B0BF0ECFA4B
:105CD80078550135EBB2A342F6D300253D55013482
:105CE800E4B26846FAF74EFA6719FFB2874206EB44
:105CF800050334D300221A702DE008EB0A035B7900
:105D08003D2B0ED0202B07D005F140016A1C0DEB6E
:105D1800010505F8403CD5B20AF101035FFA83FAA0
:105D2800C3E72C46F0E705F140036B4413F8400C39
:105D38000BF0BAFA78556846FAF724FAE5B2A842A1
:105D480007EB050304F10104EDD800220A491A7093
:105D580030460BF02DFB012010B0BDE8F08707F1AD
:105D680040020DEB0207013517F8402C1A70EDB20E
:105D7800B7E70020F0E700BFE01701082DE9FF476B
:105D88002C4E282303FB016604463379FE2B0D466F
:105D980020D0FF2B4BD0022B2DD196F91850264935
:105DA8000068FCF725FF2846694609F082FC694629
:105DB8002046FFF789FE96F91C5020492068FCF719
:105DC80017FF6946284609F074FC69462046FFF724
:105DD8007BFE10E00846FFF7FBFCDFF86490DFF875
:105DE80064A080460027FEB2012332462946684651
:105DF800FFF766FC10B904B0BDE8F087BBB248FAFB
:105E080003F3DB0711D520684946FCF7F1FE06F1DC
:105E180030012068C9B2FCF703FE20685146FCF740
:105E2800E7FE69462046FFF74FFE0137DBE70649E4
:105E3800CDE700BF78280108E2170108EA17010832
:105E4800F2170108F5170108F9170108F0B504461B
:105E58008BB008460D46FFF7E3FC254F254906465B
:105E68002068FCF7C5FE282303FB05772068B9687E
:105E7800FCF7BEFE20492068FCF7BAFE2EB91F4980
:105E88002046FFF721FE0BB0F0BD0122294602A8EB
:105E9800FFF72AFD206802A9FCF7AAFE3B79FE2B32
:105EA80003D0FF2B1AD01649EAE72846FFF7A4FBD0
:105EB800057814492068FCF79BFE05F1300120683D
:105EC800C9B2FCF7ADFD10492068FCF791FE012E20
:105ED800E9D10E492068FCF78BFEE4E70C4B02A9D8
:105EE8005A786846FFF7C8FD0028DCD06946F1E714
:105EF80078280108F2170108F517010808180108A1
:105F0800DC15010818180108061801081B180108F3
:105F1800CC02002070B590F88E3004466BB990F82A
:105F28008F30012B01D9032B07D1214B1B78022B72
:105F380003D020492046FFF7C7FD1D4E002594F8E1
:105F48008E102B2903D9002384F88C3020E04B1CB9
:105F580084F88E3094F88F30012B09D10846FFF76A
:105F680015FB0028EBD10846FFF722FB38B1E6E71E
:105F7800022B0ED10846FFF709FB0028DFD0204688
:105F8800FFF764FF013594F88D30EDB2AB42D6D2FD
:105F980070BD032B08D10846FFF70AFB0028CED0B6
:105FA8003378022BDFD1EAE7002BF9D0E7E700BF0F
:105FB8008D0600202A18010838B53D4B1A6890F85C
:105FC8008C30012B044671D1D0F88830D31AB3F540
:105FD800FA7F6BD3374DC0F888202846FBF7DDF8E9
:105FE80009F076FB01462068FCF702FE324920687A
:105FF800FCF7FEFD05F11400FBF749FD09F068FB0D
:1060080001462068FCF7F4FD2C492068FCF7F0FDF8
:1060180095F8940009F05CFB01462068FCF7E8FD60
:1060280027492068FCF7E4FD95F98C0009F05AFB34
:1060380001462068FCF7DCFD22492068FCF7D8FD02
:1060480095F9920009F04EFB01462068FCF7D0FD57
:106058001B492068FCF7CCFD95F98E0009F042FB3E
:1060680001462068FCF7C4FD17492068FCF7C0FD0D
:1060780005F15000FBF711FD80B209F03DFB014628
:106088002068FCF7B5FD0E492068FCF7B1FD05F165
:106098006400FBF702FD80B209F02EFB0146206880
:1060A800FCF7A6FD09492046FFF70EFD38BD00BFE5
:1060B8009C3F0020BC2F0020471801084918010800
:1060C8004C1801084A1801084F180108521801080D
:1060D80030B5044689B0FFF78FFD13492046FFF716
:1060E800F3FC12492068FCF783FD114B1B78022B47
:1060F80018D1104D95F8723093B1206805F17C01E4
:10610800FCF776FD0C492068FCF772FD696F68465C
:10611800FBF77EFA69462046FFF7D6FC09B030BD8A
:106128000649F8E70649F6E7541801086F18010808
:106138008D060020E40400204C1801087618010898
:10614800301801082DE9F043304EDFF8C480DFF83D
:10615800C49091B00446002794F88D20FBB29A426F
:1061680009D994F88E50F37DAB4207F1010705D8A1
:10617800002384F88C3011B0BDE8F083284609F07C
:10618800A7FA01462068FCF733FD41462068FCF772
:106198002FFD73190E35187E09F09AFA014620680A
:1061A800FCF726FD1C492068FCF722FD56F825005F
:1061B80009F0ACFA01462068FCF71AFD1749206877
:1061C800FCF716FD164908A80BF0F2F856F825005A
:1061D800FAF784FC4946FAF7D9FC09F045FFFAF7C3
:1061E800D7FE694609F02FFA6846FBF749F9206897
:1061F8006946FCF7FDFC08A92046FFF765FC94F802
:106208008E30013384F88E30A6E700BFA00A002044
:106218008B18010800007A3A921801089C180108A6
:10622800A21801082DE9F041254E264FDFF8988085
:106238000446002594F88D20EBB29A423ED994F892
:106248008E30102B37D8DFE803F00913181A1C1EFC
:1062580020222426282A2C2E303234002046FFF70C
:10626800CBFC94F88E30013384F88E300135E1E7A9
:1062780016492046FFF728FCF3E71549F9E71549C1
:10628800F7E71549F5E71549F3E71549F1E7154922
:10629800EFE71549EDE71549EBE71549E9E7154932
:1062A800E7E71549E5E71549E3E74146E1E73946F8
:1062B800DFE73146DDE7002384F88C30BDE8F08164
:1062C800121B0108DB1A0108AE1A0108A7180108F9
:1062D800C7180108F1180108161901083E19010824
:1062E8006219010886190108AF190108D8190108AF
:1062F8001C1A01083E1A0108601A01087F1A0108D1
:106308002DE9F043037993B00446C3B190F88C307B
:10631800013B032B19D8DFE803F00252575C0068F1
:1063280003685B69984768B1206803689B69984768
:106338000023AB4984F88C302046FFF7C5FB13B027
:10634800BDE8F0832046FFF737FEA64B1E6894F899
:1063580085308BB1D4F88830F31AB3F5FA6F0BD9BE
:10636800A1492046FFF7B0FBA0492046FFF7ACFB48
:10637800002384F8853063719B4FDFF87482DFF85F
:106388007492206803685B6998470028D7D0206812
:1063980003689B6998470A280546C4F888601DD099
:1063A8000D281BD02C2819D03B2817D0014620686F
:1063B800FCF736FB29462046FFF7B0FBE1E713B0B0
:1063C800BDE8F043FFF72EBF13B0BDE8F043FFF779
:1063D800A1BD13B0BDE8F043FFF7B4BE394620466F
:1063E800FFF772FB41462046FFF7A6FB50B1022398
:1063F80084F88C30002384F88E30002384F88530AC
:106408006371BEE749462046FFF796FB0028EED1A8
:1064180079492046FFF790FB0028E8D177492046C4
:10642800FFF78AFB054618B12046FFF751FEE4E75F
:1064380073492046FFF780FB40B12046FFF704FC74
:10644800032384F88C30A4F88E50D6E76D49204693
:10645800FFF772FB50B12046FFF7F6FB032384F8E1
:106468008C304FF48073A4F88E30C6E76649204616
:10647800FFF762FB40B12046FFF7E6FB032384F8F1
:106488008C304FF40073EEE760492046FFF754FB69
:1064980040B12046FFF7D8FB032384F88C304FF433
:1064A8004073E0E70AAA02A92046FFF7E7FB0028A5
:1064B80046D002A90DF10200FFF7D4F920B95449DA
:1064C8002046FFF701FB98E7524B1B78022B06D0BA
:1064D8009DF80200FFF76CF808B14F49F0E79DF806
:1064E80028303F2B0DD12046FFF7AEFB9DF8025018
:1064F80020462946FFF7AAFC29462046FFF73EFC1E
:106508007BE70BB94549DBE79DF802500AA92A4603
:106518000DF10300FFF78CFA08B94149D0E720468E
:10652800FFF792FB29462046FFF790FC9DF80330C1
:10653800002B3FF462AF05213A48FBF7D8FA5CE735
:1065480039492046FFF7F8FA90B136480621FBF79B
:10655800CEFA2046FFF778FB2E4B1B78022B05D08E
:106568002D492046FFF7B0FA3049A9E73049A7E797
:1065780030492046FFF7E0FA28B101212948FBF706
:10658800B6FA2D499CE72D492046FFF7D5FA90B178
:1065980024480721FBF7ABFA2046FFF755FB1D4BB4
:1065A8001B78022B05D01C492046FFF78DFA244999
:1065B80086E7244984E7244901AA2046FFF7C4FA5C
:1065C80000285AD0019D092D01D9204978E7204695
:1065D800FFF73AFB1E4B1B789D423DD11D496FE7E3
:1065E800541B01089C3F00206E1B0108701B01080A
:1065F800012701087A1B0108E01701080126010894
:106608007F1B0108821B0108871B01088D1B0108DD
:10661800931B01088D0600202A180108AF1B0108EA
:10662800C71B0108A4300020DA1B0108E11B010880
:10663800F81B01080C1C0108111C0108281C010882
:106648002F1C0108481C01085E1C01086A1C01086F
:10665800CC0200208E1C01082A461D480A21FBF79F
:1066680048FA1C492068FCF7C3FA05F13001C9B2A1
:106678002068FCF7D5F9184922E718492046FFF7A2
:106688005BFA054640B10123154984F88C30204651
:10669800FFF71AFA134913E713492046FFF74CFA94
:1066A80028B1042384F88C3084F88E50A5E60F496D
:1066B8002046FFF741FA08B103213DE794F8851019
:1066C8000B4A0C4B00290CBF11461946F8E600BFCF
:1066D800A4300020A31C0108DC150108CC1C01080B
:1066E800B91C0108D21C0108EF1C0108F91C01089B
:1066F8003A1B0108461B01080148FFF701BE00BF0D
:10670800F405002070B5254CE569AB0607D523686C
:106718009E0604D5606A224BC0B21B6898471F23A7
:106728002806236215D52368190612D51D4B1E4A63
:106738001988138889B29BB2994219D013880133FA
:10674800C3F3080313801388184A9BB2D35CDBB2E7
:10675800A3626A0620D5114803685B061CD5FBF7BF
:10676800AEFC40230362124BBDE870401B6818471B
:106778000A48FBF7ADFC402323624FF0402202F5A4
:10678800806353E8003F43F0400302F5806040E82F
:1067980000310029F3D1DCE770BD00BF00440040A0
:1067A80040020020843500208235002082330020FA
:1067B800440200200848094A0188138889B29BB21C
:1067C8009942F9D013880133C3F30803138013885F
:1067D800034A9BB2D05C7047803300207E33002090
:1067E8007E310020FFF7E6BF70B588B00C4606463C
:1067F80015460021202268460AF07AFD231E18BF9C
:1068080001231B03CDE9023569460C230348019691
:106818000494059308F0CEFD08B070BD0044004014
:1068280010B5064C236823F001032360FFF7DCFF53
:10683800236843F00103236010BD00BF00440040FB
:1068480013B5164C2046FBF731FC19B314484FF426
:1068580000524FF48061FFF7E3FF236823F0010340
:106868002360636843F400436360636823F4803300
:106878006360236843F00103236001220823CDE904
:10688800003203231A4604214FF09040FCF7F0F938
:10689800FBF7C0FF012002B010BD00BF004400405C
:1068A800A086010013B5164C2046FBF7FFFB19B371
:1068B80014484FF400524FF48061FFF7B1FF23688A
:1068C80023F001032360636843F400436360636853
:1068D80043F480336360236843F00103236001229B
:1068E8000823CDE900320421032302224FF090400F
:1068F800FCF7BEF9FBF78EFF012002B010BD00BF08
:1069080000440040A086010073B5304C236823F092
:1069180001030825236001264FF40030FBF7A5FB8F
:106928000421CDE9005603230A224FF09040FCF7DA
:106938009FF903231A462946CDE900564FF09040A7
:10694800FCF796F9002211462148FFF74DFF6368CE
:1069580023F490436360A36823F02A03A3601D4BCC
:10696800A02283F8252320225A602046FBF7B0FB9B
:10697800FBF7A5FB40232362174B00211980174B17
:106988001980FBF793FB164B1980164B1980636827
:1069980023F400636360A36823F00803A3606368BB
:1069A80023F480436360A36823F02203A360A368F1
:1069B80043F48053A360236833432360E3699A0256
:1069C800FCD5E3695B02F9D502B070BD0044004014
:1069D800801A060000E100E082350020843500209E
:1069E8007E330020803300200649074A0B8812882E
:1069F8000133C3F3080392B29A421EBF034AD0542C
:106A08000B807047843500208235002082330020B7
:106A1800F8B5012380F86C3090F8BD30044603F0D7
:106A2800FF005BB194F8BD5004F16C070026B3B2C7
:106A38009D4204D8002384F8BD300120F8BD17F822
:106A4800010FFFF7D1FF0136F1E700000148FBF71E
:106A580024BB00BF0044004007B521B103B05DF876
:106A680004EBFCF795B90E4B1A6822F001021A6084
:106A78005A6842F400425A601A6842F001021A60E9
:106A88000823019100930222032304214FF0904030
:106A9800FCF7EEF803B05DF804EBFBF7BBBE00BFF4
:106AA8000044004037B50446FFF72EFF164B1A681E
:106AB80022F001021A605A6842F400325A605A6899
:106AC80042F480325A605A6842F400425A601A68A6
:106AD80042F001021A6008250123CDE90053022281
:106AE800032304214FF09040FCF7C2F82946032302
:106AF80002224FF09040FCF740F90021204603B0F5
:106B0800BDE83040FFF7A8BF004400400022828162
:106B18000271C280028182720261FFF7C3BF0368FB
:106B280010B504461B689847237A082B03D9092B0C
:106B380002D00023237210BD236820465B68984763
:106B48000028F6D0FCF724F90A232372BDE8104088
:106B5800FFF77CBF01460148FFF7E1BFD0150020D1
:106B680001460148FFF7DBBF9406002010B500215D
:106B78000446FFF771FF0023237210BD0148FFF799
:106B8800F5BF00BFD01500200148FFF7EFBF00BFD9
:106B98009406002008B5017A094A0929126801D823
:106BA800026108BD0169521A142AFAD9002101723A
:106BB800FFF752FF0348FBF782FA40230362F0E72E
:106BC8009C3F0020004400400238C0B210289ABF01
:106BD800014B185C00207047CA2701083B4B02464E
:106BE800586A137A10B580B233B19389C31A9BB22D
:106BF800FA2B84BF00231372137A9081052B19D8BE
:106C0800DFE803F003080E334A564F2912D1012357
:106C180013720FE0572901D10223F9E70023F7E7A0
:106C28000023FF29937206D141F204731381537E26
:106C3800002BF3D110BD9F290FD901F01F000124AB
:106C4800947282F83200FFF7BFFF507218B982F8C9
:106C58004B400923DCE70523DAE71829DED80029A9
:106C6800F7D0032351721372E1E7B2F86E02B2F85B
:106C78007242431C2340B2F870429C421EBF8018E7
:106C880080F87412A2F86E32937A517A0133DBB22B
:106C980099429372DDD9CDE7907A431C1044DBB258
:106CA8009372C176517A9942C4D801239376D0E77A
:106CB800907A431C1044DBB2937280F83210517AF8
:106CC8009942B7D2012382F84B30C2E70044014011
:106CD8002DE9F04389B0002301AFB0F868908DF832
:106CE80004300446B8460125B4F86A2048461146DF
:106CF800EEB2FBF71BFEA0B1192D11D091451FBFB5
:106D0800A318B4F86C1093F86E30013214BF0A401F
:106D1800002308F8013F18BFA4F86A200135E3E70B
:106D28002E46B6B20024013417F8010BA4B2FFF7BF
:106D38005BFEA642F7D8012009B0BDE8F08370B524
:106D480090F8665000F14C040026B3B29D4200D87A
:106D580070BD14F8010FFFF747FE0136F5E770B56F
:106D6800457E044605B1FEE7012680F84C6090F8A0
:106D7800663033B1FFF7E3FF84F86650354628469E
:106D880070BDB0F86A10B0F86800FBF7CFFD0028B6
:106D9800F5D02046FFF79CFFF0E7027FC37E02F0A4
:106DA800070243EA02230B80838BC3F3CA034B8099
:106DB800C369C3F38A338B8090F82030C27F03F015
:106DC8000F03DB0143EA5203CB80038CC3F30A139E
:106DD8000B81036AC3F3CA334B8190F8243090F8CF
:106DE800232003F01F039B0143EA92038B81838CCA
:106DF800C3F34A13CB81C38CC3F30A030B8290F805
:106E0800283090F8272003F03F035B0143EAD203C0
:106E18004B82836AC3F38A138B82438DC3F34A037D
:106E2800CB8290F82C3090F82B2003F07F031B01C5
:106E380043EA12130B83C36AC3F3CA134B83C38D8C
:106E4800C3F38A038B8390F8303090F82F20DB004F
:106E580043EA5213CB8390F8312040F2547312F076
:106E6800010F14BF1A46AC220A8490F8312012F0A0
:106E7800020F08BFAC234B847047437E70B50446AD
:106E88000D463BB1002303728E18B54203D100238F
:106E98002372A37670BD236815F8011B1B68204672
:106EA8009847F2E70346407E30B568B193F86640EC
:106EB80004F0FF054CB103F14D040C6093F8661023
:106EC8001170002283F8662030BD2846FCE70000D8
:106ED80042765AB30123037640F2FF11A0F86C10F2
:106EE80040F2FF710023A0F872127F2180F84C3025
:106EF800A0F86A308376A0F8683080F84B30A0F8A4
:106F0800703280F86630A0F86E32A0F8763AA0F8B1
:106F1800743AA0F8781A80F8FA3A52B9054B064A3A
:106F28001A60064B064A1A60FFF7F0BD0176002981
:106F3800D2D17047400200205D6B00084402002057
:106F4800856B0008F8B5477E04460D4617B1002644
:106F58003046F8BD037E002BF9D0FFF71BFEA37E59
:106F680003F0FF06002BF2D0A77629462046FFF74C
:106F780014FFEDE7427E10B50346E2B9007EB8B1D2
:106F880093F84C4004F0FF0094B11C7983F84C202E
:106F98000CB11A71DA80DC889A790134052ADC8010
:106FA80007D0092A05D0012A4FF0000305D10B703C
:106FB80010BD0123FBE70020FAE71846F8E703466F
:106FC800007E60B193F84B2002F0FF003AB1002236
:106FD80083F84B2093F8323003F01F030B7070478F
:106FE800F8B506460D461746002119224D300AF01D
:106FF8007FF92846FFF7E8FD05F01F050446603DC8
:107008000134024686F84D50394606F14E00E4B286
:107018000AF0D6F986F86640F8BD70B590F8FA4AD5
:10702800C4B9B0F8745AB0F8762AAE1AB3B23604B6
:1070380044BF80339BB27BB1954208D0831801329C
:1070480093F87A4AB0F8783A1A40A0F8762A0C7081
:10705800012070BD0020FCE71846FAE710B5404C47
:1070680086B01822002168460AF042F923788DF884
:10707800063094F85430002B5ED13A48FDF73CFCBA
:10708800ADF800003748FDF74EFC9DF8073094F83E
:1070980051208DF8030062F303038DF80730324B5B
:1070A80093F87220002A4ED09DF8052042F0010284
:1070B8008DF8052093F8912093F892308DF80420EC
:1070C80003F00F039DF80720284863F30712284BA5
:1070D8008DF807201A78931E5A425A41254B1B797E
:1070E8005B0043F0010343EA820390F89320402AAF
:1070F8008CBF0022012243EAC2039DF8022003F05C
:107108000F0322F00F0213438DF80230FAF745F807
:107118009DF8023040288CBF0020012060F3041342
:107128008DF8023014482C236A460B218DF808305C
:10713800FFF756FF06B010BD1048FDF7DDFBADF8B0
:1071480000000E489FE7BDF8043023F4FF7323F0D6
:10715800010343F07F03ADF804300523B2E700BF15
:10716800CC02002080300020E4040020BC2F002046
:107178008D060020C0050020D015002064300020B6
:107188007FB51822002168460AF0B2F842F642009C
:10719800FAF720FAADF800004FF42150FAF71AFA7E
:1071A8000749ADF80200142201A8FAF77DFA05484C
:1071B8006A460421FFF714FF07B05DF804FB00BF1F
:1071C800041D0108D015002010B5124C86B01822F5
:1071D800002168460AF08CF894F87230B3B1606FF9
:1071E800FAF7F8F9ADF80000A06FFAF7F3F91422EE
:1071F800ADF8020004F17C0101A8FAF755FA064837
:107208006A460521FFF7ECFE06B010BD03491422BB
:10721800F2E700BFE4040020D0150020DC150108C7
:107228002DE9F04F0C463549282303FB041189B09A
:1072380007462046FEF7CCFA0B79D1F82080FE2BC2
:10724800814603D14FF6FF73984206D1414638462E
:1072580009B0BDE8F04F0AF0ABB82046FEF7CCF90C
:10726800002590F800B02E46AA462C46EAB24046C1
:107278000192F8F787FF019A013090424FF02D01F3
:1072880002D809B0BDE8F08F18F802000AF1200C06
:10729800EC440AF101032C28DBB20CF8180C00D0DE
:1072A80040BB5E4503D049FA06F0C00718D50DF17A
:1072B800080E0022D0B254FA82FC83425FFA8CFC9A
:1072C80008D85444013404F0FF040136502CF6B2B7
:1072D8000FD9FEE71EF8010B07F80C000132E9E7A9
:1072E8003955631CDBB218F80220FA540234E4B2B0
:1072F800EBE7002301359A46B8E700BF7828010874
:10730800054B1870054B064800221A70054B0122E0
:1073180007211A70FBF7FEBA152E0020162E002042
:1073280044200020142E0020054A0648002313702C
:10733800054A1370054A07211370FBF7EBBA00BF23
:10734800152E002044200020162E0020142E002088
:1073580010B50B78033B0C46082B0BD8DFE803F07D
:1073680010050C1A1D0A0A0A0E00042100F67420E2
:10737800FBF7D0FA207810BD0521F7E70B21F5E7D8
:10738800042100F67420FBF7C5FA0521FBF7C2FAC1
:107398000B21EDE7FFF7C8FFECE74878FFF7B0FFF0
:1073A800E8E707B58DF807100DF10701FFF7D0FFE3
:1073B80003B05DF804FB0000F0B5704D2C782B2C61
:1073C80087B00ED918220021684609F091FFFF23E3
:1073D8006B488DF800306A460721FFF701FE07B0B9
:1073E800F0BD684E3178182200294AD1664F6846A8
:1073F80009F07EFF282303FB04738DF800401B79F6
:10740800FE2B29D0FF2B2FD0022B09D10123204698
:107418008DF80130FEF7F0F890F900308DF8123051
:107428002B78282202FB03770DF10200B96810229D
:10743800FAF73AF9524807216A46FFF7D1FD0123C6
:10744800297852483370FFF7EBFE5148072107B0FF
:10745800BDE8F040FBF75EBA042320468DF8013002
:10746800FEF7CAF80378D9E7052320468DF80130DE
:10747800FEF7C2F8062201460DF11200FAF714F9D8
:10748800CEE7012947D10021684609F031FF3E4B7C
:107498008DF80040282202FB04331A79022A0BD007
:1074A800FE2A19D0002436486A460821FFF798FDBD
:1074B80044B302233370C8E71A7D8DF805201A7E7D
:1074C8008DF801201A7F8DF80320196906220DF125
:1074D8000700FAF7E9F8E5E75B6A83B11B882B49EF
:1074E800ADF8013015220DF10300FAF7DDF8274851
:1074F800F8F748FE142894BF00240124D3E74FF678
:10750800FF73ECE734702B7801332B70214B1B7819
:10751800002B9AD063E7022968464FF0000116D184
:1075280009F0E6FE1C498DF8004017220DF1010014
:10753800FAF7BAF81548F8F725FE6A46044609210D
:107548000F48FFF74DFD2B2C15D90323B2E709F09F
:10755800CFFE12498DF8004017220DF10100FAF70D
:10756800A3F89DF800300648803B6A4609218DF84B
:107578000030FFF735FD00233370C4E7152E0020D7
:10758800D0150020162E002078280108172E00207C
:1075980044200020142E00202C2E0020432E0020F2
:1075A80010B500230B70024600782B280C4611D822
:1075B800094B282101FB00331B79FF2B06D0B2F9B8
:1075C8000110FEF735F82070012010BD511CFEF7A0
:1075D80053F8F8E71846F8E7782801080438072828
:1075E8000DD8DFE800F004060C080C0C0C0AFFF7B5
:1075F800C7BDFFF7E9BDFFF7DFBEFFF72FBD704737
:10760800D20638B505460C4604D5BDE838402049B1
:1076180009F0CEBECB044CBF1E491F4909F0C8FE75
:10762800A1070BD51D49284609F0C2FEE3072ED451
:1076380028461B49BDE8384009F062BEA20501D5BD
:107648001849F0E7230601D51749ECE7E00501D50D
:107658001649E8E7164BA34301D11649E3E7E103CE
:1076680001D51549DFE7220501D51449DBE7E30613
:1076780001D51349D7E7600701D51249D3E7210798
:1076880001D51149CFE7E202D0D51049CBE738BD83
:10769800101D0108151D0108191D01081E1D0108EE
:1076A800431D0108231D0108DA210108CD23010823
:1076B80010000100281D01082D1D01083A220108AB
:1076C800321D0108351D01083A1D01083E1D01083B
:1076D80010B51422044600212A3009F009FE0023BF
:1076E800C4F8D032A4F8D432012384F8D63210BDBD
:1076F8000B68C0F890304B68C0F894300B7A80F86B
:107708009830012380F82D3080F8333090F8963087
:10771800DB0980F8D5327047993001F1280351F818
:10772800042B40F8042B9942F9D10B8803808B78FD
:107738008370704710B500F1C40301F1340251F8A9
:10774800044B43F8044B9142F9D1012380F82E30C1
:1077580010BDF83001F11C0351F8042B40F8042B3C
:107768009942F9D10B780370704710B500F21513E0
:1077780001F11C0251F8044B43F8044B9142F9D132
:10778800012380F8323010BD10B500F2311301F139
:107798001C0251F8044B43F8044B9142F9D140F2D2
:1077A80001134385012380F8303080F8D23290F8F5
:1077B800D53253B990F8D4323BB9D0F83931C0F842
:1077C8002C32D0F83531C0F8283210BD00F26710DD
:1077D80001F1100351F8042B40F8042B9942F9D118
:1077E8000B880380704700F24D1001F1180351F81F
:1077F800042B40F8042B9942F9D10B880380704779
:1078080010B500F2791301F1140251F8044B43F852
:10781800044B9142F9D1012380F83130D0F89930E6
:1078280013F0100308D0D0F89D3013F010031CBFDC
:10783800D0F8A130C3F3001380F83D3010BD00F23A
:107848008D1001F1140351F8042B40F8042B9942D0
:10785800F9D10B880380704791F8203030B57BB997
:107868000B4600F2A31201F1340453F8045B42F80A
:10787800045BA342F9D11B881380012380F82F30C1
:1078880091F82030012B0ED100F2D91301F1340206
:1078980051F8044B43F8044B9142F9D10A881A80F5
:1078A800012380F8343030BD0B68C0F80F324B68C4
:1078B800C0F813320B7A80F81732012380F8D332DC
:1078C80070470B68C0F818324B68C0F81C320123A7
:1078D80080F8323070470B68C0F820324B68C0F827
:1078E8002432012380F83630704710B500F50A734A
:1078F80001F13C0251F8044B43F8044B9142F9D191
:10790800012380F8303080F8D43210BD10B500F56E
:10791800197301F1340251F8044B43F8044B9142B6
:10792800F9D10A881A80012380F82C3010BDF0B5EF
:1079380000252C460126AB4206D803680C4004FA01
:1079480002F213430360F0BD06FA05F73C43013524
:10795800F1E770B50446084694F82A6016B900267F
:10796800304670BD94F8E0300022022B84F82A20BB
:10797800F5D90A60D4F83551002DC8BF6D423223BD
:10798800B5FBF3F11E2301EB4101FFF7D0FFD4F85B
:10799800351102231E22C90FFFF7C9FFE0E770B5B2
:1079A8000446084694F82B6016B90026304670BD88
:1079B80094F8E0300022022B84F82B20F5D9D4F873
:1079C80039510260002DC8BF6D423223B5FBF3F177
:1079D8001E2301EB4101FFF7AAFFD4F83931002B30
:1079E8004FF002034FF01E02B4BF03211946FFF700
:1079F8009EFFDBE738B50446084694F8D022AAB9BA
:107A080094F82C30DBB384F82C2004F5197304F2B5
:107A18009A2204F5267153F8045B42F8045B8B4202
:107A2800F9D11B8813800123A4F8D0320023036006
:107A3800182594F8D132312B06D85A1C234484F8DF
:107A4800D12293F89B12E1B994F89A1201231940B4
:107A58000722FFF76CFF94F89A1201230F22C1F353
:107A68004001FFF764FF94F89A1201231722C1F32B
:107A78008001FFF75CFF002384F8D0320123184609
:107A880038BD2A46083D0723EDB2FFF750FFF82D11
:107A9800CFD194F8D132312BD6D8EFE703462DE970
:107AA800F04793F82D600846002E62D093F81552DF
:107AB800D3F89010B3F88B4193F8D58293F8D3722A
:107AC8000022AD1A83F82D2001F1010118BF01250C
:107AD8004CB1632CD7BFC4EB84143F2431346422E7
:107AE800D8BFB4FBF2F4B3F91331002B44D06422AD
:107AF80093FBF2F3522BA8BF5223132BB8BF1323C7
:107B0800A3F113094FF0000A05235246C0F800A05C
:107B1800FFF70DFF022305225146FFF708FF4146F4
:107B280001230722FFF703FF01230822FFF7FFFEC7
:107B3800514601230922FFF7FAFE02230A22FFF722
:107B4800F6FE01230C22FFF7F2FE01230D2239462F
:107B5800FFF7EDFE01230E222946FFF7E8FE072373
:107B680013222146FFF7E3FE06231A224946FFF7B0
:107B7800DEFE3046BDE8F0879946C3E72DE9F843B5
:107B880090F82E800D46B8F1000F3AD090F8E13009
:107B98000021FF2B80F82E1003D00F2B28BF0F23B6
:107BA800194690F8E090B9F1030F2DD84FF0000670
:107BB8002FD07F273446002228462A600423FFF767
:107BC800B6FE022304224946FFF7B1FE0122022134
:107BD8003846F9F7E3FF0823014606222846FFF74F
:107BE800A6FE02230E223146FFF7A1FE022211460D
:107BF8002046F9F7D3FF0A23014616222846FFF745
:107C080096FE4046BDE8F883A9F10306062E28BF74
:107C180006260A23B0F8D870D0F8D440B7FBF3F79B
:107C28000B4B7F2FA8BF7F279C4208DC094B9C4247
:107C380009DB64234FF0030994FBF3F4BBE7064C1C
:107C48004FF00309B7E7054C4FF00309B3E700BF4E
:107C5800C3C9C1003D363EFF18F00100E80FFEFF22
:107C68002DE9F04F90F8303085B005460E462BB917
:107C780000230093009805B0BDE8F08F002380F83A
:107C8800303090F8D2320093002BF1D0D0F828028F
:107C9800F8F728FF6A49F8F779FF6A49F8F776FF95
:107CA8008146D5F83501F8F71DFF6549F8F76EFFED
:107CB8006449F8F76BFF8046484608F0EBF88346BE
:107CC800404608F0E7F80746D5F83901F8F70AFF03
:107CD8005B49F8F75BFF5B49F8F758FF0446D5F8AE
:107CE8002C02F8F7FFFE5649F8F750FF5549F8F708
:107CF8004DFF01462046F8F73FFE824608F006F998
:107D08000190404608F002F90446484608F0FEF89B
:107D18000390504608F0BEF8214602905846F8F7FE
:107D280035FF039B044619463846F8F72FFF029A99
:107D38001146F8F72BFF01462046F8F71DFE01997A
:107D480004463846F8F722FF214608F087F83E49EE
:107D5800F8F71CFF00210446F9F7B6F820B12046D1
:107D68003A49F8F70BFE04462046F9F7EBF880B2DB
:107D7800A0F1B40424B2002CBCBFB43004B2B4F5F2
:107D8800B47FA8BFA4F5B47449464046A8BF24B23E
:107D9800F8F7F2FD4FF07C51F8F7F8FE08F0B6F866
:107DA8004FF07C5180465046F8F7F0FE08F0AEF8E8
:107DB8000146F8F7EBFE5946F8F7E8FE3946F8F7BA
:107DC800E5FE414607464046F8F7E0FE01463846DC
:107DD800F8F7D4FD08F044F8002708F01FF81C490C
:107DE800D5F841513760642395FBF3F5F8F7CEFEDB
:107DF800F9F7A8F8F8F776FEF9F7A4F802220321B4
:107E0800F9F7CCFE0C2301463A463046FFF78FFDC2
:107E18002846F8F767FEF9F795F802220321F9F7E3
:107E2800BDFE0D2301460C223046FFF780FD0723D7
:107E38001922032194FBF1F1FFF779FD1AE700BF3E
:107E480095BFD63335FA8E3CE12E65420000B44327
:107E5800706D424B2DE9F84390F8319004460D4679
:107E6800B9F1000F3BD000261E4980F83160D0F8E8
:107E78008501F8F78BFE08F0F7F81A498046D4F820
:107E88007D01F8F783FE08F0EFF8B4F989112E6048
:107E98000746404601EB8104F9F754F80122022114
:107EA800F9F77CFE0923014632462846FFF73FFDD5
:107EB8003846F9F747F801220221F9F76FFE08233F
:107EC800014609222846FFF732FD0B2311222146DD
:107ED800FFF72DFD01231C223146FFF728FD4846F8
:107EE800BDE8F883000020412DE9F84390F83D9063
:107EF80004460D46B9F1000F3BD000271E4980F813
:107F08003D70D0F88501F8F741FE08F0ADF81A4940
:107F18008046D4F87901F8F739FE08F0A5F8B4F9E5
:107F280089112F600646404601EB8104F9F70AF8EB
:107F380001220221F9F732FE092301463A46284672
:107F4800FFF7F5FC3046F8F7FDFF01220221F9F7AB
:107F580025FE0823014609222846FFF7E8FC0B23E3
:107F680011222146FFF7E3FC01231C221946FFF7E3
:107F7800DEFC4846BDE8F883000020412DE9F843BF
:107F880090F8329004460D46B9F1000F46D000270C
:107F9800244980F83270D0F81901F8F7F7FD224922
:107FA800F8F7F4FD2149F8F7E9FC08F05DF81D49F8
:107FB8008046D4F81D01F8F7E9FD1B49F8F7E6FDFE
:107FC8001B49F8F7DBFC08F04FF81A490646D4F8C5
:107FD8001802F8F7DBFD08F047F82F600446404622
:107FE800F8F7B0FF0B2301463A462846FFF79FFCF7
:107FF8003046F8F7A7FF0A2301460B222846FFF769
:1080080096FC2046F8F79EFF01220321F9F7C6FDEA
:108018000B23014615222846FFF789FC4846BDE890
:10802800F88300BFE12E65420000A04000006144D3
:108038000000E1430000C84238B50346084693F8FB
:10804800334014B90024204638BD93F8D652691C31
:10805800C9B20022042983F8332083F8D61203D941
:10806800012183F8D612EDE7012DEBD193F8941096
:1080780002601823FFF75BFC042318222946FFF748
:1080880056FCE0E71C2945D8DFE801F00F1214166A
:10809800181A1C1E44204422442426282A2C2E3038
:1080A800323436383A3C3E4042001B4909F080B928
:1080B8001A49FBE71A49F9E71A49F7E71A49F5E7B0
:1080C8001A49F3E71A49F1E71A49EFE71A49EDE7C0
:1080D8001A49EBE71A49E9E71A49E7E71A49E5E7D0
:1080E8001A49E3E71A49E1E71A49DFE71A49DDE7E0
:1080F8001A49DBE71A49D9E71A49D7E71A49D5E7F0
:108108001A49D3E71A49D1E71A49CFE71A49CDE7FF
:108118001A49CBE71A49C9E7D1210108191D0108F5
:10812800451D01084A1D01084F1D0108541D01087D
:10813800591D01085E1D0108631D0108681D01081D
:108148006D1D0108721D0108771D01087C1D0108BD
:10815800811D0108861D01088B1D0108901D01085D
:10816800951D01089A1D01089F1D0108A41D0108FD
:10817800A91D0108AE1D0108B31D0108B81D01089D
:10818800DC150108192941D8DFE801F00D10121497
:1081980016181A1C1E4020222426282A2C2E30327B
:1081A8003436383A3C3E1A4909F002B91949FBE716
:1081B8001949F9E71949F7E71949F5E71949F3E7BB
:1081C8001949F1E71949EFE71949EDE71949EBE7CB
:1081D8001949E9E71949E7E71949E5E71949E3E7DB
:1081E8001949E1E71949DFE71949DDE71949DBE7EB
:1081F8001949D9E71949D7E71949D5E71949D3E7FB
:108208001949D1E71949CFE71949CDE71949CBE70A
:10821800231D01085E1D0108D1210108BD1D0108AB
:10822800191D0108C21D0108C71D0108CC1D010840
:10823800771D01084A1D0108591D0108541D010830
:10824800D11D01088B1D01084F1D0108D61D01080D
:10825800DB1D0108E01D0108E51D0108EA1D0108F4
:10826800EF1D0108F41D0108F91D0108FE1D010894
:10827800031E0108DC150108102925D8DFE801F0E4
:10828800090C240E1012141618241A1C1E2424205B
:1082980022000E4909F08CB80D49FBE70D49F9E7B2
:1082A8000D49F7E70D49F5E70D49F3E70D49F1E702
:1082B8000D49EFE70D49EDE70D49EBE70D49E9E712
:1082C8000D49E7E70D49E5E70D49E3E7231D0108F7
:1082D800191D0108081E0108CD230108541D0108B5
:1082E8009F1D01080D1E0108121E01084A1D0108E4
:1082F800591D0108951D01084F1D0108D61D0108CB
:10830800DC150108142921D8DFE801F00B0E101242
:108318001420201620182020202020201A20201C7D
:108328001E000B4909F044B80A49FBE70A49F9E776
:108338000A49F7E70A49F5E70A49F3E70A49F1E77D
:108348000A49EFE70A49EDE70A49EBE70A49E9E78D
:10835800D1210108191D0108171E01084A1D01082D
:108368004F1D01085E1D01081C1E01087C1D010827
:10837800231D0108211E0108DC15010823289ABFC6
:10838800014B185C02207047DB2701080B46013BB4
:108398001146032B0BD8DFE803F002040608FFF7A9
:1083A80071BEFFF7EFBEFFF767BFFFF7ABBF01492D
:1083B80008F0FEBFDC15010838B5384B0446821CAE
:1083C80003F1280153F8040B42F8040B8B42F9D14E
:1083D80000252946C4E9245584F898502B2204F135
:1083E800990008F085FF2946342204F1C40008F0FA
:1083F8007FFF29461D2204F1F80008F079FF29467D
:108408001C2204F2151008F073FF29461C2204F2FE
:10841800311008F06DFF29461A2204F24D1008F0B9
:1084280067FF2946122204F2671008F061FF294607
:10843800142204F2791008F05BFF2946162204F290
:108448008D1008F055FF2946362204F2A31008F0D3
:108458004FFF2946362204F2D91008F049FF294671
:10846800C4E98655C4E98855C4F80F52C4F81352B4
:1084780084F817523C2204F50A7008F039FF29469F
:10848800362204F5197008F033FF3622294604F223
:108498009A2008F02DFF204638BD00BFFC130108C4
:1084A8002DE9F04FC77E837E457F867F90F820E0D8
:1084B80090F82B8090F819C0BF000C4647EA931734
:1084C80003F03F01037F03F0010247EA822705F02A
:1084D8000F02D20142EA530206F07F031B0143EA6E
:1084E8001513C57F89B06D0045EAD6150EF0030651
:1084F800059345EA462390F82160009306F01F058E
:10850800AD0145EA9E0390F8225090F824E00193CB
:10851800ED0045EA561390F8235002930EF0070633
:1085280045EA062390F82550039305F03F067601A7
:1085380046EADE0390F8266090F827E00493B60038
:1085480046EA95160EF0010546EA852690F8285069
:10855800069205F00F0B4FEACB1B4BEA5E0B90F827
:1085680029E00EF07F0A4FEA0A1A4AEA151A90F82B
:108578002A506D0045EADE1508F0030E45EA4E253F
:1085880090F82CE00EF01F094FEA891949EA98097A
:10859800490190F82D80007E41EADC010CF0070CBF
:1085A80040EA0C204FEAC80848EA5E180791F8F735
:1085B8006DFE079920800846F8F768FE6080384607
:1085C800F8F764FE069AA0801046F8F75FFE059B50
:1085D800E0801846F8F75AFE20810098F8F756FE12
:1085E80060810198F8F752FEA0810298F8F74EFED4
:1085F800E0810398F8F74AFE20820498F8F746FECF
:1086080060823046F8F742FEA0825846F8F73EFEF0
:10861800E0825046F8F73AFE20832846F8F736FEFF
:1086280060834846F8F732FEA0834046F8F72EFEEE
:10863800E08309B0BDE8F08F4A78013A92B202317E
:108648000020F8F785BE000038B5044601750029FA
:1086580044D04FF6FF730025A0F8F030204B80F887
:10866800BD5080F8CE5080F86C50C0F8D05080F8DB
:10867800655080F8DC5080F86650C0F8E05080F80B
:10868800675080F8EA5080F86850C0F8EC5080F8DD
:108698006A50C0F8F43080F86B5080F80751C0F881
:1086A800085180F80E51C0F8105180F81651C0F8E2
:1086B800185100F58E70FFF70BF80A4B0A4A1A603A
:1086C8000A4B0B4AC4F8F453A4F8F853C4F8FC5303
:1086D8001A602046BDE83840FEF718BA38BD00BF1A
:1086E8000000C07F40020020696B0008440200209F
:1086F800916B0008037D70B504460D4613B900263A
:10870800304670BDFEF746FA94F8653003F0FF0670
:10871800002BF4D0002384F8653004F115012046BD
:10872800FFF78AFFA37D23449B7D8342E7D1294637
:108738002046FFF7B5FEE3E70346007D30B500B3FA
:1087480093F86C4004F0FF00DCB11D79002483F835
:108758006C4065B1132A1C7114D8134C227802B9E5
:10876800DA800132D2B2022A88BF00222270DC8865
:108778009A790134012ADC8002D0022A00D01AB981
:108788000A7030BDDC80F2E793F8672002F0FF043E
:1087980032B1002283F8672004230B702046F0E7EB
:1087A80003230B70EDE700BFBD050020027D0346E3
:1087B8000AB90020704790F8682002F0FF0022B143
:1087C800002283F868200A70704793F86A2002F044
:1087D800FF002AB1002283F86A2001230B7070473A
:1087E80093F86B2002F0FF0022B1002283F86B207F
:1087F8000223F3E793F8662002F0FF00002AD8D09E
:10880800002283F866205A7DEE2AD2D1DB7D812BA7
:10881800CFD10323E2E738B504461D46EA230846CC
:1088280084F86D30AB1C114684F86E302A4684F803
:108838006F0004F1700008F0C3FD04F16D012046DB
:10884800FFF7FAFE6319043583F87000EDB284F877
:10885800BD5038BD13460A468221FFF7DCBF000031
:1088680070B50C4600F1BE060546102200213046C0
:1088780008F03EFD6379032B10D12079FFF77EFDC8
:1088880022680146D2B23046FFF780FD94F90630DF
:10889800002B03DB0349304608F032FD012385F83D
:1088A800CE3070BD431D0108002310B51A464FF69F
:1088B800FF74191D00EB410101334988A14218BF1B
:1088C80052180A2BF5D1B0F829301344B0F82B20F0
:1088D8001A44B0F82D30B0F82F001344184410BDD6
:1088E8002DE9F04190F82F7004460D4697B3002605
:1088F80080F82F6000F2A310FFF7D6FFB4F9C1315A
:10890800D4F8A3812E60B342B8BF34464FF0640256
:1089180090FBF2F1A8BF0A222846A8BF93FBF2F405
:1089280009230022FFF703F8012202212046F9F764
:1089380035F90823014609222846FEF7F8FF47F6CD
:10894800FF7141454FF00F034FF01102A8BF414698
:10895800FEF7EDFF3846BDE8F0812DE9F04190F8CB
:10896800347004460D4697B3002680F8346000F250
:10897800D910FFF799FFB4F9F731D4F8D9812E60EF
:10898800B342B8BF34464FF0640290FBF2F1A8BF7F
:108998000A222846A8BF93FBF2F409230022FEF717
:1089A800C6FF012202212046F9F7F8F808230146FC
:1089B80009222846FEF7BBFF47F6FF7141454FF0F5
:1089C8000F034FF01102A8BF4146FEF7B0FF38462B
:1089D800BDE8F081F0B591B00D46F22301A9044637
:1089E8001646ADF80830FFF759F838B12389ADF8C5
:1089F8000A30019B039301238DF8093001A9204611
:108A0800FFF728FA70B19DF8093010A9062202FB79
:108A18000312218A22F8361C0133019942F8341CCA
:108A28008DF8093001A92046FFF75EFA70B19DF86C
:108A3800093010A9062202FB0312218D22F8361CE8
:108A48000133019942F8341C8DF8093001A92046F8
:108A5800FFF794FA70B19DF8093010A9062202FBBD
:108A68000312618A22F8361C0133019942F8341C3A
:108A78008DF8093001A92046FFF780F870B19DF8FC
:108A8800093010A9062202FB0312618922F8361C5C
:108A98000133019942F8341C8DF8093001A92046A8
:108AA800FEF757FF70B19DF8093010A9062202FBA6
:108AB8000312618822F8361C0133019942F8341CEC
:108AC8008DF8093001A92046FEF769FF70B19DF8BD
:108AD800093010A9062202FB0312A18822F8361CCD
:108AE8000133019942F8341C8DF809309DF809705A
:108AF800082F11D801A92046FFF7F2FE60B110AA8D
:108B0800062303FB0723A28923F8362C0137019A91
:108B180043F8342C8DF809709DF80970082F11D886
:108B280001A92046FFF719FF60B110AA062303FB2D
:108B38000723E28A23F8362C0137019A43F8342CAC
:108B48008DF809709DF80970082F11D801A92046E1
:108B5800FFF786F860B110AA062303FB0723E28912
:108B680023F8362C0137019A43F8342C8DF8097014
:108B78009DF80970082F11D801A92046FFF75CFA63
:108B880060B110AA062303FB0723A28A23F8362C18
:108B98000137019A43F8342C8DF809709DF8097053
:108BA800082F11D801A92046FEF724FF60B110AAAA
:108BB800062303FB0723E28823F8362C0137019AA2
:108BC80043F8342C8DF809709DF8090050B100EB7A
:108BD800400043000233DAB2327002A9284608F096
:108BE800EFFB012011B0F0BD10B5524BD0F8D020EA
:108BF8001B6894B004463AB19A1A40F6C4118A42E6
:108C080084BF012280F8CE20D4F8E0203AB19A1A25
:108C180040F6C4118A4284BF012284F8DC20D4F8CB
:108C280008213AB19A1A40F6C4118A4284BF012237
:108C380084F80721D4F810213AB19A1A40F6C411E1
:108C48008A4284BF012284F80E21D4F8EC203AB17C
:108C58009A1A40F6C4118A4284BF012284F8EA2095
:108C6800D4F818213AB19A1A40F6C4118A4284BF3E
:108C7800012284F8162194F8CE2072B1002284F8DB
:108C8800CE20C4F8D03004F1BE02102321212046A2
:108C980014B0BDE81040FFF7BEBD94F8DC1041B138
:108CA800C4F8E030082384F8DC20194604F1D40223
:108CB800EDE794F8072142B184F80711C4F80831A8
:108CC80004F1F8020F230221E1E794F80E1141B1F3
:108CD80084F80E21C4F8103104F5867202230721A6
:108CE800D5E794F8EA2042B184F8EA10C4F8EC30E9
:108CF80004F1E40206231E21C9E794F8161141B1D4
:108D080084F81621C4F8183104F58A72022309215F
:108D1800BDE70DF1030201A904F58E70FFF75AFEB5
:108D280030B19DF8033001AA80212046FFF773FD7A
:108D380014B010BD9C3F002070B591F82050044637
:108D48000E465DBB0846FFF7AFFD642390FBF3F0CA
:108D580040BAA4F8D400B6F91E30581C1CBF0A2526
:108D680093FBF5F56DBAA4F8D6503368591C16D0A4
:108D78000C4A934228BF13461A0C84F8D8201A0AC2
:108D880084F8D92084F8DA3096F923305A1C08BFC1
:108D9800002384F8DB30012384F8DC3070BD002325
:108DA800EAE700BFFFFF7F0038B50D4604460F49CC
:108DB800A868F7F7EBFEF8F7C5F840BAA4F8E4009E
:108DC80068680A49F7F7E2FEF8F7BCF840BAA4F871
:108DD800E600E8680549F7F7D9FEF8F7B3F8012384
:108DE80040BAA4F8E80084F8EA3038BD00401C46D0
:108DF80010B54B681BBAC0F8F8308B681BBA4FF433
:108E08007A72C0F8FC30CB6893FBF2F31344044643
:108E180083F310035BBAA0F804314B8B5BBA11499A
:108E2800A0F80231D0F8F400F7F7B0FE0E49F7F7D2
:108E380061FFF8F7ADF840BA94F8F030A4F80001F3
:108E4800FF2B0CD094F8F120FF2A02D0934238BFB0
:108E5800134684F80631012384F8073110BD002336
:108E6800F7E700BF0000C8426666664010B50B46CB
:108E78004A68C0F8F42004460649D868F7F786FE21
:108E8800F8F760F8012340BAA4F80C0184F80E3111
:108E980010BD00BF0000C84270B58A68C2F317024F
:108EA8004A2A90B004460B4600F0F48040D8212AA4
:108EB80022D8172A06D8002A79D0012A00F005817D
:108EC80010B070BD183A092AFAD801A151F822F059
:108ED80007900008C98E0008C98E00081F91000875
:108EE800C98E0008C98E0008EB8F0008C98E0008DB
:108EF800C98E0008B79000082A2A00F032813E2A5D
:108F0800DED14D78192D01F10C0100F24E812A466F
:108F180001A808F055FA01ABC5F11A020021581949
:108F280008F0E6F901A904F58E70FEF75CFCC7E7C6
:108F3800AD2A00F0588129D8932A45D01BD87C2A1D
:108F480000F08580882ABBD14D78152D01F10C01E0
:108F580000F239812A4601A808F032FA01ABC5F1BE
:108F680016020021581908F0C3F901A904F58E70FA
:108F7800FEF765FCA4E7A22AA2D101A8F9F76AFACC
:108F880001A904F58E70FEF78FFC99E7F22A00F02C
:108F98003381FD2A00F05481E22A91D101A8F9F722
:108FA80073FA01A904F58E70FEF795FC88E701A80D
:108FB800F9F750FA01A92046FFF752FC01A904F578
:108FC8008E70FEF795FB7BE701A8F9F70BFA01A96C
:108FD8002046FFF7B1FE01A904F58E70FEF73CFCB0
:108FE8006EE7194601A8F9F71AFA01A92046FFF712
:108FF800DBFE01A904F58E70FEF7B7FB60E75D782C
:10900800332D03F10C0114D82A4601A808F0D8F929
:1090180001ABC5F134020021581908F069F99DF82F
:10902800213084F8F03001A904F58E70FEF782FB38
:1090380046E70A4601AD3C33106851682E4603C620
:1090480008329A423546F7D110683060E7E74D7824
:10905800382D01F10C010FD82A4601A808F0B0F903
:1090680001ABC5F139020021581908F041F99DF802
:10907800253084F8F13023E70A4601AD44331068FF
:1090880051682E4603C608329A423546F7D11378FE
:109098003370ECE701A8F9F78AFA01A92046FFF72F
:1090A800E5FE01A904F58E70FEF7AAFB08E719464C
:1090B80001A8F9F7B4F901A92046FFF799FE01A91B
:1090C80004F58E70FEF760FBFAE64D782A2D01F163
:1090D8000C0110D82A4601A808F072F901ABC5F1B5
:1090E8002B020021581908F003F901A904F58E7024
:1090F800FEF712FBE4E60A4601AD34331068516806
:109108002E4603C608329A423546F7D1118893781D
:10911800B3703180E9E75D781C2D03F10C0110D89C
:109128002A4601A808F04CF901ABC5F11D0200213F
:10913800581908F0DDF801A904F58E70FEF709FB4F
:10914800BEE60A4601AD2433106851682E4603C6B0
:1091580008329A423546F7D1106830601379337176
:10916800E9E74D78112D01F10C0110D82A4601A824
:1091780008F026F901ABC5F112020021581908F0D0
:10918800B7F801A904F58E70FEF720FB98E60A46A9
:1091980001AD1C33106851682E4603C608329A4246
:1091A8003546F7D113883380EBE70A4601AD2433FF
:1091B800106851682E4603C608329A423546F7D1E0
:1091C80013883380AEE60A4601AD1C331068516837
:1091D8002E4603C608329A423546F7D110683060E9
:1091E8009388B380C1E601A8F9F74EF901A904F5FF
:1091F8008E70FEF766FB63E64D783B2D01F10C019E
:1092080010D82A4601A808F0DBF801ABC5F13C02EA
:109218000021581908F06CF801A904F58E70FEF7C2
:1092280064FB4DE60A4601AD4433106851682E468A
:1092380003C608329A423546F7D110683060EBE72A
:1092480001A8F9F7CFF801A904F58E70FEF75EFBC7
:1092580036E600BF4A7922B18B79012B01D1FFF79D
:109268001BBE7047B0F5E16F03DC10F5E16F04DB5E
:109278007047A0F5616000B2F4E700F5616000B2E4
:10928800F3E7000038B5B0F8F8330D4613F00801DD
:10929800AA8808BFC0F8081113F0020308BFC0F875
:1092A8001831B2F5005F044600F0B28007D86C2A86
:1092B80017D06D2A00F08F806A2A60D038BD42F23C
:1092C80002039A423BD042F6FF739A42F6D1D0F895
:1092D800FC23A968BE30FEF793F9012384F8CE3049
:1092E800ECE7B5F90A00FFF7BDFFF7F7FBFB4C49C0
:1092F800F7F74CFCF7F726FE40BAA4F8E400B5F9F6
:109308000800FFF7AFFFF7F7EDFB4549F7F73EFC1D
:10931800F7F718FE40BAA4F8E600B5F90C00FFF715
:10932800A1FFF7F7DFFB3F49F7F730FCF7F70AFE35
:10933800012340BAA4F8E80084F8EA30BEE7B5F89B
:1093480009300A22B3FBF2F35BBAA0F8D430B5F8BF
:109358000B30B3FBF2F35BBAA0F8D630D5F8113076
:1093680080F8DA301A0C80F8D8201A0A80F8D92048
:109378006B7F80F8DB30012380F8DC309EE7002922
:109388009CD0D5F80A301BBAC0F8F830D5F80E30A2
:109398001BBAC0F8FC30AB8A242253433233642210
:1093A800B3FBF2F35BBAA0F80031EB8A0A214B4316
:1093B8005BBAA0F80231D0F8F43393FBF2F303F56B
:1093C8007A735BBAA0F804316B7A80F8063101230E
:1093D80080F8073172E7B5F90C2052BAA0F80C21D1
:1093E800012280F80E21002B3FF468AFD5F80E104B
:1093F8000A2391FBF3F303F51C53103383F30F0394
:109408005BBAA0F81431C0F8F41380F8072155E7C7
:10941800AB89A0F8F833D5F81130C0F8FC334DE724
:1094280058A08B416E882E4330B5204C85B0054638
:1094380094F99200F7F762FF00238DF805308DF854
:10944800073094F895308DF80830194B94F893202C
:109458008DF8040098788DF80620F7F73FFF8DF80F
:1094680009001448FBF75FFAF7F712FF8DF80A00B6
:109478002046F7F780FEF7F741FF8DF80B002046EE
:10948800F7F78BFE8DF80C002046F7F77DFE8DF878
:109498000D002046F7F792FE0A238DF8050001AA71
:1094A80014212846FFF7B7F905B030BDBC2F0020BE
:1094B800CC0200206430002073B5184C05462046C5
:1094C800F7F759FEF7F71AFF8DF800002046F7F76F
:1094D80052FE06461248FBF70FFA01463046F7F7E8
:1094E80017FF8DF801002046F7F757FE8DF80200A8
:1094F8002046F7F749FEFF238DF80430094B8DF815
:1095080003009878F7F7F2FE06238DF805006A46FF
:109518001D212846FFF77FF902B070BDBC2F00203F
:1095280064300020CC020020F7B5144D144E0446D8
:1095380095F99200F7F7E2FE8DF80000304695F9AC
:109548009270FBF7D9F901463846F7F7E1FE95F82E
:1095580093308DF801008DF80230304600238DF8E5
:109568000330FBF7E0F905238DF804006A461C2157
:109578002046FFF750F903B0F0BD00BFBC2F002014
:109588006430002030B591B04EF6EA631A49ADF860
:109598000030044614220DF10200F8F797F80DF197
:1095A8000200F6F7EFFDC3B2DA1CD0B2694651FAF1
:1095B80082F26D250DF800504C20507052209070AA
:1095C8005320D070312010716FF02B0050710120A2
:1095D8005072032000219072113306209171D171CD
:1095E8001172D07211735173DBB26A462921204679
:1095F800FFF711F911B030BD041D01080038024B06
:1096080018BF0120187070477C0500202DE9F04133
:10961800002A4AD1042B00F2A1809EB2002B42D02E
:109628004D4C4FF0800EFF250F8894F81EC0C35D87
:1096380023EA0C03C355A37F01325B081FFA82FC9F
:10964800A3773BB90B8801330B8084F81EE00B88A5
:10965800C554A37FB1F8008010F8087027EA030307
:1096680000F80830A37F5B08A3773BB90B88013368
:109678000B8084F81EE00B88C554A37FB1F80080E6
:1096880010F8087027EA030300F80830A37F5B0886
:10969800A37733B90B8801330B8084F81EE00B885D
:1096A800C5546645C0D8BDE8F081FF2AFBD1032B1D
:1096B80000F249819FB2002BF5D0274C0025802667
:1096C800B1F800C094F81EE010F80C3023EA0E033D
:1096D80000F80C30A37F01355B081FFA85FCA377DF
:1096E80033B90B8801330B80A6770B88C254A37F4C
:1096F800B1F8008010F808E02EEA030300F80830FB
:10970800A37F5B08A37733B90B8801330B80A67757
:109718000B88C254A37F5B08A37733B90B88013346
:109728000B80A6770B88C254A37FB1F8008010F88D
:1097380008E02EEA030300F80830A37F5B08A3774C
:109748002BB90B8801330B80A6770B88C254674569
:10975800B6D8BDE8F08100BFAC0C00200D889A4C4B
:10976800425DA67F22EA06024255A27F520803F50F
:10977800C063A2773AB90A8801320A808022A277A8
:109788000A88FF2585540D88A67F425D22EA0602D5
:109798004255A27F5208A2773AB90A8801320A8054
:1097A8008022A2770A88FF258554A27F5208A277D3
:1097B8003AB90A8801320A808022A2770A88FF25EE
:1097C8008554A27F5208A2773AB90A8801320A80E2
:1097D8008022A2770A88FF2585540D88A67F425DDE
:1097E80022EA06024255A27F5208A2773AB90A88AD
:1097F80001320A808022A2770A88FF2585541E0636
:1098080005D40D88A67F425D22EA06024255A27F52
:109818005208A2773AB90A8801320A808022A277D0
:109828000A88FF2585545D0605D40D88A67F425D0C
:1098380022EA06024255A27F5208A2773AB90A885C
:1098480001320A808022A2770A88FF2585549A0669
:1098580005D40D88A67F425D22EA06024255A27F02
:109868005208A2773AB90A8801320A808022A27780
:109878000A88FF258554DF0605D40D88A67F425D3A
:1098880022EA06024255A27F5208A2773AB90A880C
:1098980001320A808022A2770A88FF2585541E0794
:1098A80005D40D88A67F425D22EA06024255A27FB2
:1098B8005208A2773AB90A8801320A808022A27730
:1098C8000A88FF2585545D0705D40D88A67F425D6B
:1098D80022EA06024255A27F5208A2773AB90A88BC
:1098E80001320A808022A2770A88FF2585549A07C8
:1098F80005D40D88A67F425D22EA06024255A27F62
:109908005208A2773AB90A8801320A808022A277DF
:109918000A88FF258554DB0705D40A88A57F835C60
:1099280023EA05038354A37F5B08A377002B7FF406
:10993800BAAE0B88802201330B80A2770B88FF22F6
:10994800C254BDE8F0810E881F4C855DA77F25EACB
:1099580007058555A57F6D0803F5E063A57735B93B
:109968000D8801350D808025A5770D8842550D8815
:10997800A67F425D22EA06024255A27F5208A277DC
:109988003AB90A8801320A808022A2770A88FF251C
:109998008554A27F5208A2773AB90A8801320A8010
:1099A8008022A2770A88FF258554A27F5208A277D1
:1099B800002A7FF418AF0A8801320A808022A27731
:1099C8000A88FF2585540EE7AC0C00202DE9F047E6
:1099D8009C4C802500270F80A577FF2505709846A9
:1099E800002B00F02C8103F1FF3912FA89F9561E79
:1099F800BA463B460BE0554540F0C0800137BFB240
:109A08000A88424580F0B3804E4500F0078116F879
:109A1800015F002BEFD16B1EDBB2FD2B00F2AA8099
:109A28003F2B40F2E18005F14103DBB23F2B00F20E
:109A3800AC80A37F01355B08EDB2A377002B00F063
:109A4800E4805B08A37743B90B8801330B8080233C
:109A5800A3770B88FF22C254A37FAA0608D4B1F8C3
:109A680000C010F80C2022EA030300F80C30A37F92
:109A78005B08A37743B90B8801330B808023A37756
:109A88000B88FF22C254A37FEA0608D4B1F800C0AD
:109A980010F80C2022EA030300F80C30A37F5B08BF
:109AA800A37743B90B8801330B808023A3770B88F6
:109AB800FF22C254A37F2A0708D4B1F800C010F8C7
:109AC8000C2022EA030300F80C30A37F5B08A3777D
:109AD80043B90B8801330B808023A3770B88FF22BF
:109AE800C254A37F6A0708D4B1F800C010F80C204C
:109AF80022EA030300F80C30A37F5B08A37743B97D
:109B08000B8801330B808023A3770B88FF22C25474
:109B1800A37FAA0708D4B1F800C010F80C2022EAE5
:109B2800030300F80C30A37F5B08A37743B90B88C5
:109B380001330B808023A3770B88FF22C254A37FB5
:109B4800EA0705D40D88425D22EA03034355A37F43
:109B58005B08A377BBB90A8801320A808022A27702
:109B68000A88FF2585540A884245FFF44DAF002036
:109B7800BDE8F0870127AA463B4641E7FBB25246BB
:109B8800FFF744FD47E700233AE70A8894F81EC028
:109B9800835C23EA0C038354A37F3F355B08EDB253
:109BA800A37743B90B8801330B808023A3770B88F5
:109BB800FF22C254A37F5B08A37743B90B88013304
:109BC8000B808023A3770B88FF22C254A37F6A06E9
:109BD8003FF537AFB1F800C010F80C2022EA0303B4
:109BE80000F80C30A37F2CE7A37F7F355B08EDB22C
:109BF800A377002BEED10B8801330B808023A3774A
:109C08000B88FF22C254A37FE4E70B8801330B8043
:109C18008023A3770B88FF22C254E3E75BB9A37FB5
:109C2800802B1EBF013292B20A80904594BF00205B
:109C38000120BDE8F087FBB25246FFF7E7FC0A882F
:109C4800EDE700BFAC0C00202DE9F04F47F26F7331
:109C58000022827003800B78A3F1FE03B3FA83F32A
:109C68005B0983708A780D4612F001011CBF43F02E
:109C780080038370D5F8202122F07F4222F0FF0272
:109C880085B0044612B143F008038370AA68C2F392
:109C98001702FF2A1ED9B2F5803F18D363F07F035D
:109CA800A37041F002014FF0020B09234FF00A0C98
:109CB8000822E1700B20CDF804C01E4617464FF06D
:109CC800070E4FF006094FF0050A042117E043F08C
:109CD8000203A370180600F1D68008234FF0090C80
:109CE80007220A204FF0000BCDF804C01E46174685
:109CF8004FF0060E4FF005094FF0040A032195F8BE
:109D0800018004F8018004EB0108297904F80A109D
:109D1800697904F80910A97904F80E10A1780907DF
:109D280009D595F82111A15495F82211A15503469A
:109D3800674662460646A968A154A278900707D5E7
:109D4800BA1C1F46AB68C3F30F23A35596B233461C
:109D5800BBF1000F05D05A1C1F46AB7AA35596B22B
:109D68003346A278D10606D55A1C1F4695F82331EA
:109D7800A35596B23346454A127803F1010914FAFD
:109D880089FA05F10C0B42B16B785A460DF10E01B8
:109D98005046FFF71BFE00285AD16A7850465946AC
:109DA8001FFA82FA07F00CFB2278394B6178D2430C
:109DB800D2B2072F9A5C82EA0102995CA27882EA01
:109DC8000102995CE27882EA0102995C227982EACE
:109DD8000102995C627982EA0102995CA27982EABD
:109DE8000102995CE27982EA0102995C1BD0227A2D
:109DF8005140082F595C16D0627A5140092F595C9E
:109E080011D0A27A51400A2F595C0CD0E27A514005
:109E18000B2F595C07D0227B51400C2F595C1EBF79
:109E2800627B5140595CA1551AFA89F39BB2B5F887
:109E38000C21E2545A1CB5F80C1192B2090AA1542B
:109E4800AA78981CD20780B20BD405B0BDE8F08F71
:109E5800A378BDF80EA043F04003A37088F800A0D3
:109E6800A2E7D5F81071D5F81811D5F81461275064
:109E780022180F335660916095F81C11117398B22F
:109E880005B0BDE8F08F4FF0000B0EE77C05002011
:109E9800842F01082DE9F04F944D0C4683B00146FC
:109EA80007462846164607F08BFA914A0023802079
:109EB8002380138482F82200002E00F0CD8095F8CC
:109EC80000C04FF0400B4FEADC1C82F822B09E46DF
:109ED8004FF0FF0892F8229015F803A04FEA4C0CB7
:109EE8001AEA090F4FEA590118BF4CF0010C82F821
:109EF8002210002900F0B380BCF1020F00F0448466
:109F0800BCF1030F00F0DF83BCF1010F40F0BA8011
:109F18009E4240F2A18015F8039019EA010F14BF80
:109F28004FF0010C4FF0000C5FEA510A40F0B68385
:109F380001339BB29E42138482F8220040F28C8047
:109F4800E95600294FEA4C0C01DA4CF0010C82F872
:109F580022B0402100919E427ED9009915F80390C5
:109F68004FEA4C0C19EA010F00995FFA8CFC18BFF4
:109F78004CF0010C5FEA510A40F0268401339BB291
:109F88009E42138482F8220066D94FEA4C0115F9E3
:109F980003C015F80390BCF1000FC9B201DA41F013
:109FA80001014FEA410C19F0400F5FFA8CFC18BF11
:109FB800202100F09F854CF0010C002940F09B8582
:109FC80001339BB29E42138482F8220044D915F9CA
:109FD80003904FEA4C0CB9F1000F5FFA8CF115F8B9
:109FE80003C001DA41F0010149001CF0400FC9B279
:109FF80018BF4FF0200A00F0B98541F0010182F83E
:10A0080022A0BAF1000F03D10133138482F8220091
:10A018007D2921D84131238803F1010CA4F800C01F
:10A02800F954138C9E4217D992F8221015F803C0E0
:10A0380011EA0C0F4FEA510114BF4FF0010C4FF019
:10A04800000C82F8221021B901339BB2138482F8E4
:10A0580022009E423FF63EAF03B0BDE8F08F0133C9
:10A068009BB2BCF1020F138482F8220000F0AD818C
:10A07800BCF1030F00F03482BCF1010F4FF08001F6
:10A088003FF446AF9E42E7D915F803C011EA0C0F1A
:10A098001ED05FEA51092DD101339BB29E42138431
:10A0A80082F82200D8D9E9560029C0F2E8804FF09A
:10A0B80080094FEA590182F8221019B90133138433
:10A0C80082F822002388591C218007F80380A8E71A
:10A0D800490882F8221019B90133138482F8220042
:10A0E8002388591C218007F803E09AE7800B002099
:10A0F800AC0C002019EA0C0FDBD0890840F0C080B6
:10A1080001339BB29E42138482F82200A4D9E956F7
:10A118000029C0F2668280215FEA510C40F041823A
:10A1280001339BB29E42138482F8220094D9E95CE1
:10A138004FEAD11C49064FEA4C0C40F1BD8420215E
:10A148004CF0010C82F8221029B901339BB2138418
:10A1580082F8220080219E427FF67EAF15F8039098
:10A168004FEA4C0C11EA090F5FFA8CFC18BF4CF04F
:10A17800010C490840F06E8301339BB29E42138460
:10A1880082F822007FF668AFE9564FEA4C0C0029A6
:10A198005FFA8CFC80F2318480215FEA51094CF02F
:10A1A800010C40F0658301339BB29E42138482F810
:10A1B80022007FF651AF4FEA4C0115F903C0BCF1FC
:10A1C800000FC9B280F225844FF080095FEA59096F
:10A1D80041F0010140F0598301339BB29E42138440
:10A1E80082F822007FF638AF15F903C04900BCF1A8
:10A1F800000FC9B280F226844FF080095FEA59093E
:10A2080041F0010140F04D8301339BB29E4213841B
:10A2180082F822007FF620AF15F903C04900BCF18F
:10A22800000FC9B2C0F211844FF0400915F803C0FD
:10A23800490019EA0C0FC9B200F052834FEA5909D4
:10A2480041F0010182F82290B9F1000F40F0048436
:10A2580001339BB2138482F822001FFA81FC002983
:10A268003FF4E0AE00232188013301F10109A4F88D
:10A27800009007F801E099B26145F4D3D1E6402196
:10A2880015F803C011EA0C0F3FF446AF490840F037
:10A29800A98101339BB29E42138482F822007FF683
:10A2A800DBAE15F803904FEAD91C19F0400F4FEABE
:10A2B8004C0C00F0F58320214CF0010C002940F0F3
:10A2C800F08301339BB29E42138482F822007FF60A
:10A2D800C3AE4FEA4C0C5FFA8CF115F903C015F8C0
:10A2E8000390BCF1000F01DA41F00101490019F0B7
:10A2F800400FC9B218BF4FF0200C00F02C8441F079
:10A308000101BCF1000F40F0288401339BB29E424A
:10A31800138482F822007FF69FAE15F903C0490026
:10A32800BCF1000FC9B201DA41F0010182F822B094
:10A338004FF0400A9E427FF68FAE15F803C04900E1
:10A348001AEA0C0FC9B218BF41F001015FEA5A0CB2
:10A3580040F0D58201339BB29E42138482F82200DA
:10A368007FF67AAE15F903C04900BCF1000FC9B2F7
:10A37800C0F275834FF0400C15F8039049001CEAB1
:10A38800090FC9B200F0DA824FEA5C0C41F0010112
:10A3980082F822C0BCF1000F40F0688301339BB201
:10A3A800138482F822001FFA81FC00293FF43AAE98
:10A3B80000232188013301F10109A4F8009007F86E
:10A3C800018099B28C45F4D82BE69E427FF644AEC4
:10A3D800E95C4FF04009C909B2F820C04B0015F8F4
:10A3E8000C1019EA010F4FEA590A01D043F0010392
:10A3F800BAF1000F40F0B1820CF1010C1FFA8CFC8D
:10A408006645A2F820C082F822007FF625AE15F92D
:10A418000C905900B9F1000FC9B280F2DC824023D8
:10A4280041F00101002B40F0A5820CF1010C1FFA4C
:10A438008CFC6645A2F820C082F822007FF60CAE9C
:10A4480015F90C304FEA4109002B5FFA89F980F2BF
:10A45800CB82402149F00109002940F09A820CF191
:10A46800010C1FFA8CFC6645A2F820C082F8220075
:10A478007FF6F2AD15F90C104FEA49030029DBB25B
:10A4880080F2BE824FF0400943F00103B9F1000F9A
:10A4980040F08E820CF1010C1FFA8CFC6645A2F884
:10A4A80020C082F822007FF6D7AD15F90C105B00AA
:10A4B8000029DBB280F2C382402143F0010382F815
:10A4C800221029B90CF1010CA2F820C082F8220050
:10A4D8002188013301F1010CA4F800C07B54A0E5E8
:10A4E8009E427FF6B9AD15F803C04FF040094FEA18
:10A4F800DC111CEA090F4FEA41014FEA590A01D061
:10A5080041F00101BAF1000F40F0368301339BB2EC
:10A518009E42138482F822007FF69EAD15F90390BF
:10A5280015F803C04900B9F1000FC9B201DA41F0CA
:10A53800010149001CF0400FC9B218BF4FF0200AB2
:10A5480000F0F18241F00101BAF1000F40F0ED8214
:10A5580001339BB29E42138482F822007FF67CADC1
:10A5680015F9039015F803C04900B9F1000FC9B2F5
:10A5780001DA41F0010149001CF0400FC9B218BFCF
:10A588004FF0200A00F0DA8241F0010182F822A09F
:10A59800BAF1000F03D10133138482F82200413944
:10A5A80039E515F8039019EA0C0F14BF4FF0010CA8
:10A5B8004FF0000C5FEA910A40F0378201339BB2FA
:10A5C8009E42138482F822007FF646ADE9560029A0
:10A5D8004FEA4C0C01DA4CF0010C82F822B0402111
:10A5E800B9E5402115F8039019EA010F14BF4FF09F
:10A5F800010C4FF0000C5FEA510A40F00D82013364
:10A608009BB29E42138482F822007FF625ADE9565C
:10A6180015F8039000294FEA4C0C01DA4CF0010CB4
:10A628004FEA4C0C19F0400F5FFA8CFC18BF4FF042
:10A63800200A00F048824CF0010CBAF1000F40F0FB
:10A64800448201339BB29E42138482F822007FF633
:10A6580003AD15F903904FEA4C01B9F1000F15F855
:10A6680003C0C9B201DA41F0010149001CF0400FF2
:10A67800C9B218BF4FF0200A00F0658241F001010D
:10A6880082F822A0BAF1000F7FF454AE01339BB2D6
:10A69800138482F822004FF0800A4BE6890819EAF1
:10A6A8000A0F00914FEA4C0C01D04CF0010C82F8D3
:10A6B800221000297FF44FAC01339BB2138482F837
:10A6C8002200802146E415F803C01CEA010F14BFDC
:10A6D800012100215FEA99097FF40BAF01339BB296
:10A6E8009E42138482F822007FF6B6AC15F90390D7
:10A6F80015F803C0B9F1000F4FEA410101DA41F042
:10A7080001011CF0400F4FEA410118BF4FF020092A
:10A7180000F0BB8141F00101B9F1000F40F0B781B1
:10A7280001339BB29E42138482F822007FF694ACD8
:10A7380015F9039015F803C04900B9F1000FC9B223
:10A7480001DA41F0010149001CF0400FC9B218BFFD
:10A758004FF0200900F0C38141F00101B9F1000F69
:10A7680040F0BF8101339BB29E42138482F82200DD
:10A778007FF672ACEB564900002BC9B201DA41F002
:10A78800010182F822B00AE792F8229019EA0A0F2A
:10A7980014BF012100215FEA59097FF41DAE01337E
:10A7A8001FFA83FC6645A2F820C082F822007FF6D3
:10A7B80053AC15F90C90B9F1000F4FEA410380F240
:10A7C80002814FF0400A11E64FEA4C0C890819EA59
:10A7D8000A0F5FFA8CFC019101D04CF0010C0029A2
:10A7E80040F0D38101339BB29E42138482F8220049
:10A7F8007FF632AC4FEA4C0115F903C015F8039007
:10A80800BCF1000FC9B201DA41F00101490019F0A9
:10A81800400F5FFA81FA18BF4FF0200C00F07681E4
:10A828004AF0010ABCF1000F40F0728101339BB27B
:10A838009E42138482F822007FF60EACEB564FEA54
:10A848004A01002BC9B201DA41F0010182F822B0B5
:10A85800FFF7DEBB15F803904FEA4C0C11EA090F1D
:10A868005FFA8CFC7FF499AC5FEA51093FF49BAC2A
:10A878004FEA4C0115F803C019EA0C0FC9B27FF46E
:10A88800A5AC5FEA59093FF4A7AC15F803C0490025
:10A8980019EA0C0FC9B27FF4B1AC5FEA59093FF469
:10A8A800B3AC15F803C0490019EA0C0FC9B201D0BE
:10A8B80041F001015FEA59097FF4B8AC01339BB25A
:10A8C8009E42138482F822007FF6C6AB15F903C0B6
:10A8D8004900BCF1000FC9B2C0F2BA804FF080093C
:10A8E8004FEA590982F82290B9F1000F3FF4B0AC51
:10A8F8001FFA81FC00297FF4B5ACFFF795BB15F86A
:10A90800039049001CEA090FC9B201D041F00101C6
:10A918005FEA5C0C7FF430AD01339BB29E42138436
:10A9280082F822007FF698AB15F903C04900BCF104
:10A93800000FC9B2C0F296804FF0800C4FEA5C0C51
:10A9480082F822C0BCF1000F3FF428AD1FFA81FC49
:10A9580000297FF42DADFFF767BB15F80C9059005F
:10A968001AEA090FC9B24FEA5A037FF459AD002B0E
:10A978003FF45BAD15F80CA04FEA410913EA0A0F42
:10A988005FFA89F94FEA53017FF464AD00293FF477
:10A9980066AD15F80CA04FEA490311EA0A0FDBB2BD
:10A9A8004FEA51097FF470ADB9F1000F3FF472AD71
:10A9B80015F80CA05B0019EA0A0FDBB24FEA59013F
:10A9C8003FF47DAD79E515F80C305B064FEA81015F
:10A9D8004FD5202324E59B005FFA83F915F80C3046
:10A9E800590648D5202135E58900CBB215F80C1059
:10A9F800490642D54FF0200946E54FF0400937E7B0
:10AA080015F80C104FEA89034906DBB238D5202126
:10AA180053E54FF0400938E719EA0A0F4FEA910168
:10AA28004FEA4C0C3FF44AAC46E419EA0A0F4FEAE5
:10AA3800D1014FEA4C0C3FF485ABFFF781BB82F89C
:10AA480022B045E54FF040092BE74FF080092FE78A
:10AA580041F0010182F822B01FFA81FC02E44FF0B4
:10AA6800800C53E741F0010182F822B01FFA81FC03
:10AA78009EE420237EE720218BE74FF0200997E70B
:10AA88004FF0200182F8221022E54FF020094900FA
:10AA980019EA0C0FC9B24FEA590A3FF455AD51E50E
:10AAA80020214FEA4C0C19EA010F5FFA8CFC4FEA9F
:10AAB800510A3FF4C2ADBEE54FF0200182F82210E2
:10AAC8002021FFF748BB4FF0200A4FEA4C0119EA52
:10AAD8000A0FC9B24FEA5A0C3FF413AC0FE44FF017
:10AAE8002009490019EA0C0FC9B24FEA590A3FF484
:10AAF8004DAD49E520214FEA4C0C11EA090F5FFAE8
:10AB08008CFA4FEA510C3FF48DAE89E64FF0200CD9
:10AB18004FEA4A0119EA0C0FC9B24FEA5C0A3FF43E
:10AB28006EAAFFF76ABA4FF0200A49001AEA0C0F1A
:10AB3800C9B24FEA5A093FF411AE0DE64FF02003AF
:10AB480082F822302BE54FF0200C82F822C04FF01B
:10AB5800200AFFF7EFBB4FF0200C490019EA0C0F51
:10AB6800C9B24FEA5C0A3FF48BAD87E54FF020038A
:10AB780082F82230FFF74CBA49001AEA0C0F4FEA64
:10AB88009909C9B23FF4C8ADC4E58A4600994FEAAD
:10AB98004C0C19EA0A0F4FEAD1015FFA8CFC3FF41A
:10ABA8000CAAFFF708BA00BF2DE9F04F5788B7F590
:10ABB8008F7F8BB0144606460BD9002222700022E4
:10ABC8006F2B628000F06581002333700BB0BDE805
:10ABD800F08F12780E2A0D4624D80E2A00F2118121
:10ABE80001A151F822F000BFC7AB000817AE00085A
:10ABF8000BAE00080BAE000817AE000817AE000831
:10AC080017AE000817AE000817AE000817AE000808
:10AC180065AE00080BAE00080BAE00080BAE0008CE
:10AC280089AE0008692A40F2EA806A2A40F0E98081
:10AC38009C4FFA8A02F1FF3C1FFA8CFC002A00F0B4
:10AC480078820CF1030CDFF860E2BC44FF22B91CE7
:10AC580011F8010B424061451EF80220F8D19342D9
:10AC680000F0D08100222270C4F80220E280FA8A23
:10AC7800022AA9D939796F2900F02E83032AA3D093
:10AC880079796F2900F03883042A9DD0B9796F2922
:10AC980000F03583052A97D0F9796F2900F03E83B3
:10ACA800062A91D0397A6F2900F04582072A8BD07D
:10ACB800797A6F2900F03583082A85D0B97A6F2907
:10ACC80000F03283092A3FF47FAFF97A6F2900F048
:10ACD8002E830A2A3FF478AF397B6F2900F02A8344
:10ACE8000B2A3FF471AF797B6F2900F026830C2A79
:10ACF8003FF46AAFB97B6F2900F022830D2A3FF435
:10AD080063AFF97B6F2900F01E830E2A3FF45CAF16
:10AD1800397C6F2900F01D830F2A3FF455AF797CE9
:10AD28006F2900F01383102A3FF44EAFB97C6F29C6
:10AD380000F01283112A3FF447AFF97C6F2900F025
:10AD48000E83122A3FF440AF397D6F2908BF4FF0B8
:10AD580012087FF439AF02F101091FFA89F93A4460
:10AD6800A7F816905FFA89F9937050494A4602A8E5
:10AD780006F026FB6F234FF0010CBB704FF0000E5E
:10AD88006423A7F800E0A7F816C0237008EB0C03AB
:10AD980099451FFA89F27FF617AF901E02A9A0EB1A
:10ADA80008005A1E0B440A4413FA80F04FF06A0850
:10ADB8004FF007094FF0660A05E0002B40F0BE810E
:10ADC80090423FF401AFFB8A12F8011F07EB030B17
:10ADD80001338BF80210FB822378092BEDD9A3F1FC
:10ADE800640BBBF1050FEBD8653B042B00F2BA826C
:10ADF800DFE813F01F01170112010E011B01632A7E
:10AE080005D800232370C4F80230E380DDE6254F1F
:10AE1800FA8AB91801328B70FA822278092A00F26C
:10AE2800A480002A3FF4D0AE013A082A3FF6CCAEFF
:10AE380001A151F822F000BF01B10008D1AB000810
:10AE4800D1AB000863B0000863B00008EBB000089D
:10AE5800B7B0000825B10008D5B000087A1C628098
:10AE6800104EEB55A088727F618883189942FFF6CF
:10AE7800ADAE33785F0600F1E4810E232370A5E6BA
:10AE88007A1C6280EB55E2886388934210D20123D2
:10AE98009BE604490A800122CA8264228B702270D0
:10AEA800002392E6AC0C0020842F0108AE0C002091
:10AEB8000023638023700223037042802B78FD2BCC
:10AEC80000F08780EB7803722B7943726B794360CB
:10AED8006A780832728000224FF4BC70DFF8CCC266
:10AEE8007281F6210446013499424FEA54042ED85F
:10AEF80049D38B4240F08A802B78FD2B7FD04FF0CE
:10AF0800060B2846DFF8A48210F801AF0BEB0A09FC
:10AF180009F1FF3189B2F7F709F904EB440708EBA7
:10AF28008707ADF808003979019102A8F7F7DAF830
:10AF380005EB090215F809305278019903EB022351
:10AF4800BDF808209BB29A421FD005233DE6601E3B
:10AF58001418824204F1010780F06C8127F0010186
:10AF680001EB57015CF82110BDE7A2F16401052946
:10AF78003FF62AAE653A042A00F2FD81DFE802F0C6
:10AF8800817D797593002246E2E7BB79DA0706D519
:10AF9800FA79924582BF521912F80B20B2729B07B8
:10AFA8000BD56300234408EB83036A781B7A9A4223
:10AFB80082BF5B1913F80B30F3724FEA4409A144BE
:10AFC80008EB8908317398F8053073730BB0BDE846
:10AFD800F08F6B790372AB7943726B7A297AEA79CD
:10AFE8001B0403EB0123134443606A7802F10C014C
:10AFF8004180A978C9077FF56EAF19326AE74FF02B
:10B008000A0B7EE70A2201232270DEE50323DCE532
:10B01800F97684F80090D3E64FF06803B976237088
:10B02800CEE6797084F800C0CAE6397784F80080E3
:10B03800C6E6397001F00103618887F801E0033B37
:10B0480001F1010BA4F802B06B5497F90030002B02
:10B05800ACBF634653462370B2E66288511C6180D8
:10B06800AB54237801332370AEE50722FB762270B8
:10B0780016E76822BB76227012E701227B702270E5
:10B088000EE762883B70002103F00103033B7970EF
:10B09800511C6180AB5497F90030002BC0F232810B
:10B0A8000123237090E56A223B772270F8E66288D4
:10B0B800511C6180AB543B787A78134313F0020338
:10B0C80040F0D7806288511C6180AB546288511C63
:10B0D8006180AB543B78D8064CBF69236A23237040
:10B0E80072E56288511C6180AB543B781D074CBFE8
:10B0F80067230723237067E562883A83511C6180C0
:10B10800AB543A787B7712F0010200F0D080062227
:10B118000833A280E3800423237055E56288511C1C
:10B128006180AB547B7813F00203CFD009232370DE
:10B138004AE5FF2293E54FF006080CE6013B082B91
:10B148003FF63EAE0FF2040B5BF823F08DB100081A
:10B15800C9AD0008C9AD000879B1000879B1000887
:10B1680007B20008D5B1000821B20008B9B100083B
:10B17800638803F1010BA4F802B0E9542378013382
:10B1880023701DE663883B8303F1010BA4F802B02A
:10B19800E9543B78797713F001036DD00831062321
:10B1A800E180A380042323700AE600BF84300108ED
:10B1B800638803F1010BA4F802B0E9543B78DB067D
:10B1C8007FF534AF4FF069032370F9E5638803F125
:10B1D800010BA4F802B0E9543B7879780B4313F0DB
:10B1E800020343D1618801F1010BA4F802B06B544A
:10B1F800618801F1010BA4F802B06B54DEE76388A3
:10B2080003F1010BA4F802B0E9543B7819077FF564
:10B2180000AF67232370D3E5638803F1010BA4F81B
:10B2280002B0E9547B7813F00203E1D04FF0090330
:10B238002370C5E5574902EB4200144651F8201027
:10B2480057E602A92844FEF725FE737FBDF80810CB
:10B258006288CB1A9BB21A446280727F1A44727752
:10B26800E2881344E380338BE95406E6082323700D
:10B27800A6E508232370A7E40C31E18079784FF024
:10B288000A0B11F00101A4F804B028D0618801F17B
:10B29800010BA4F802B005F801C0618801F1010BA7
:10B2A800A4F802B06B54E3880D33E3807AE7797829
:10B2B8000C33E38011F001014FF00A03A38024D07E
:10B2C8006388012158186080E9546388591861809F
:10B2D800EA54E3880D331DE74FF002083BE5638825
:10B2E80003F1010BA4F802B0E954638803F1010BE0
:10B2F800A4F802B0E95455E74FF003082BE54FF0E6
:10B30800040828E5662323705EE463885A1C62807B
:10B31800E95463885A1C6280E954FCE64FF005083A
:10B3280019E54FF0070816E54FF0080813E54FF048
:10B33800090810E54FF00A080DE54FF00B080AE57B
:10B348004FF00C0807E54FF00D0804E54FF00F0823
:10B3580001E54FF00E08FEE44FF01008FBE44FF053
:10B368001108F8E477290ED084F800E0C4F802E068
:10B37800A4F806E024E5772B09D000232370C4F84D
:10B388000230E38020E44FF06503237018E565235D
:10B39800237019E48430010870B500F5EF6604469F
:10B3A80000F5CA613046F6F7CEFF0546A068036887
:10B3B8002A461B6931469847E06830B103682A4637
:10B3C80031461B69BDE87040184770BD08B5034693
:10B3D800806840B1B3F84C14B3F84A04F7F7A6FAFA
:10B3E800003818BF012008BD0346806880B1B3F853
:10B3F8004C24B3F84A14914209D09918013291F8B3
:10B408005004B3F84E140A40A3F84C2470470020A7
:10B418007047836810B504467BB10023A0F84C340C
:10B42800A0F84A34C06810B10368DB699847A0687F
:10B438000368BDE81040DB69184710BDF8B5224F16
:10B4480004463846F5F797FEF5F7EFFE064697F9F6
:10B458009200F5F7EAFE05463846F5F795FE6423AF
:10B4680084F86236FF2384F86436332384F855362B
:10B47800442384F85636D4F8583684F860666D222A
:10B4880062F31703C4F85836C0F10A000023C4F861
:10B498005C3684F8713700B24FF43943A4F8723738
:10B4A80080F30700092384F8630684F8615604F5DD
:10B4B800CA6084F8743704F5A471F7F7BDFA20461A
:10B4C800BDE8F840FFF768BFBC2F002010B5332354
:10B4D80080F85536442380F85636D0F85836144A42
:10B4E800C0F860266FF31703C0F85836002380F8B9
:10B4F8005C3680F85D3680F85E3680F85F3680F816
:10B5080071374FF44853A0F87237032209230446D1
:10B5180080F8642680F8743700F5A47100F5CA60D5
:10B52800F7F78AFA2046BDE81040FFF735BF00BF9D
:10B538000008800470B586B004460021102202A8D5
:10B54800019105F0D5FE01AB03CB01ABC4F8800631
:10B55800C4F8841603CB01ABC4F88806C4F88C166B
:10B5680003CB04F5D362C4F89006C4F8941601AB73
:10B5780005AE1D4603CDB542106051602B4602F161
:10B588000802F6D12B881380332384F855364423D8
:10B5980084F85636D4F85836942262F317031021EB
:10B5A8004222C4F8583684F85C16002384F86C26C6
:10B5B8002021282284F85D1684F85E3684F85F36E8
:10B5C80084F8603684F8613684F8623684F8633625
:10B5D80084F8643684F8653684F8663684F8673605
:10B5E80084F8683684F8693684F86A3684F86B36E5
:10B5F80084F86D2684F86E3684F86F3684F87036D1
:10B6080084F8713684F8723684F8733684F87436A0
:10B6180084F8753684F8763684F8773684F8783680
:10B6280084F8793684F87A3684F87B3684F871376A
:10B638004FF43243094AA4F872374E2304F5CA601E
:10B64800C4F87C2684F8743704F5A471F7F7F4F984
:10B65800204606B0BDE87040FFF79EBED016CB0F5F
:10B6680010B504469DF8080084F85E26002284F888
:10B678005F2684F8602684F8612684F8622684F8B8
:10B688006326332284F85526442284F85626D4F8B3
:10B698005826A4F85C1684F8643684F871374D216E
:10B6A8008F2361F3170284F873370A2384F8650639
:10B6B80084F87207C4F8582604F5CA6084F8743709
:10B6C80004F5A471F7F7B8F92046BDE81040FFF774
:10B6D80063BE0000F0B502298BB004460D461CD1AC
:10B6E8003F4B40481B7800EB031000F58970F5F7D5
:10B6F80075FE3D4B18603D4A0C236B43D718D35851
:10B708003A7900210191511E082908D8DFE801F093
:10B7180009095E5E6262070765002D29EBD90BB047
:10B72800F0BD1B788DF8043000218DF8242005A881
:10B738001022019E05F0DCFDBF683846F4F722FDB3
:10B74800C2B2102A28BF1022394605A805F038FED3
:10B758002E229DF8243084F860260022C4F85C6606
:10B76800A4F8625684F8743684F8612605AB04F2AE
:10B77800646509AE1A4603CAB24228606960134676
:10B7880005F10805F6D1332384F85536442384F8A7
:10B798005636D4F85836162262F31703C4F85836CA
:10B7A800002384F871374FF45C43A4F872371923E7
:10B7B80004F5CA6084F8743704F5A471F7F73CF906
:10B7C80020460BB0BDE8F040FFF7E6BD1B88ADF89A
:10B7D8000430A9E71B680193A6E71B680193A3E758
:10B7E800CC02002028030020E80500200C000020DF
:10B7F8002DE9F041884D894F2B78142202FB037301
:10B8080088B093F85530012B04460E4613D191F8B1
:10B81800213133B1332B0ED191F822310BB1442BA6
:10B8280009D1B368C3F31703172B54D006D8142BC8
:10B838002DD0152B43D008B0BDE8F08103F18073FB
:10B848004B3B23F07F43012BF5D8D6F82031744ABF
:10B8580023F07F4323F0FF039342ECD1358DF0684A
:10B8680040F207239D4200F0D180B5F5027F00F039
:10B87800BE80B5F5007F08D1F5F78AFB942800F063
:10B88800B680B0F5967F00F0C1800222B6E002A82B
:10B898003146F6F78CFEBDF90800002804DA03A843
:10B8A800F6F7FCFF0028C6DB2D28C4DCA4F8BA088C
:10B8B800B4F8B03843F01003A4F8B038BBE701235C
:10B8C80084F8B8380023A4F8BA38564B1B68643B90
:10B8D800C4F8BC38AFE7D6F82031514A23F07F438B
:10B8E80023F0FF039342A6D196F80180B8F1160F12
:10B8F80006F10C012ED8424602A805F061FD02AB04
:10B90800C8F11702002103EB080005F0F1FC0DF166
:10B918000E00F6F7C3FFB0F100088CDB424A9DF831
:10B928001E1008EB4803980002EB83031B79994229
:10B9380081D1B8F12D0F1FFA88F622DC0139029B5C
:10B94800125808291DD8DFE801F01B1B39393B3B89
:10B958001C1C3D000B4602AA1C3618685968944600
:10B96800ACE803000833B3426246F6D11868CCF855
:10B97800000099889B798CF80630ACF80410C6E76B
:10B9880013702878F8F740F92A78142303FB027318
:10B99800012183F8551097F82D300BB987F82D1031
:10B9A800B8F1020F10D1214B07EB0210196800F50E
:10B9B8008970F5F74DFDA4F8BA6879E71380E0E7D8
:10B9C8001360DEE71360DCE7B8F1000FF3D1184B22
:10B9D8001A78002AEFD083F8008060232380114B67
:10B9E8001B680BB16360E6E74FF0FF33FAE7B4F882
:10B9F800B03843F00203A4F8B0380022B3790093BA
:10BA0800737929462046FFF72BFE14E7B4F8B038BF
:10BA180043F00403EFE700BFCC0200202803002016
:10BA2800003344009C3F00200C000020E805002063
:10BA38007A2E002010B52F4B1A782F4B142101FBBA
:10BA48000233044693F85530012B37D12B4BD0F8ED
:10BA5800B4281B689A1AB2F57A7F21BFB0F8B028CB
:10BA6800C0F8B43842F00102A0F8B02890F8B8281D
:10BA780062B1D0F8BC289A1A312A81BFB0F8B02830
:10BA8800C0F8BC3842F01003A0F8B038B4F8B038A9
:10BA9800DA0614D523F01003A4F8B038B4F8BA18AD
:10BAA8002046FFF717FEB4F8BA3801339BB22D2BA6
:10BAB800A4F8BA3802D9002384F8B83810BD98071A
:10BAC80008D523F00203A4F8B0382046BDE810409A
:10BAD800FFF730BD590702D523F00403F3E7DA076F
:10BAE800ECD523F00103A4F8B0382046BDE8104097
:10BAF800FFF7ECBCCC020020280300209C3F00206C
:10BB080038B5134B134A1B68C0F8B438002380F8C3
:10BB1800B838A0F8BA38C0F8BC38A0F8B0381370F4
:10BB28000D4B0E481B780E4D00EB031000F5897085
:10BB3800F5F754FC0B4B02241860E0B2F9F75CFDF2
:10BB480001342C2C286305F10C05F6D138BD00BF53
:10BB58009C3F00207A2E0020CC02002028030020E1
:10BB68000C000020E805002000230370FF23437029
:10BB78008370C37003717047F8B53A4D04462E7848
:10BB88003948142707FB060090F84F60012E0CD0A7
:10BB9800022E0CD076B9A16090F84C30032B18BF58
:10BBA8000022A368E26033B9FEE7A360F4E7A2606D
:10BBB8000022F6E7FEE70023C4E90433C4E9523360
:10BBC800C4E95433A3617F23A4F85831F6F774FC11
:10BBD800A878022844D0431F58425841234940F2CC
:10BBE800FF12FDF70BFD0220A4F84E24204A08702E
:10BBF800002348708870C8701E4913705370937082
:10BC0800D370C4F8DA31C4F8DE31C4F8E231C4F8CC
:10BC18001233C4F81633C4F81A33A4F84C34A4F811
:10BC28004A341A4601330C2B0A70CA704A708A705B
:10BC380001F10401F6D1104B1B6803F57A7304F681
:10BC4800A800C4F8A438FFF78FFF84F8AD2884F85B
:10BC5800AE28228062602046BDE8F840FFF750BF5A
:10BC68000120BBE7CC02002028030020B1050020FA
:10BC78007D050020810500209C3F00200346407878
:10BC8800FF2805D0012803D19B78012B08BF02208B
:10BC98007047007840B14B79834204D18879431EBC
:10BCA8005842584170470020704710B54B790370CF
:10BCB8009379DB0943705379032B044607D1107934
:10BCC800FCF75CFBE0701368DBB2237110BDFF2347
:10BCD800C370FAE77FB58B6833F07F4305460C469F
:10BCE80000F6A8060ED18B79012B0BD101A8F6F727
:10BCF800B1FB9DF80930082B04D001AA2146304633
:10BD0800FFF7D3FF21463046FFF7C3FF78B3A36898
:10BD1800C3F31703F52B16D16678012E29D83246BE
:10BD280004F10C0101A805F04BFB01ABC6F10202BE
:10BD38000021981905F0DCFA9DF805309A1E534247
:10BD4800534185F8AA3895F8AD3853B195F8AE380F
:10BD580021790A480133DBB2CB1A59425941F5F728
:10BD68002AFA012385F8AD38237985F8AE3804B06E
:10BD780070BDA389ADF80430DEE700BFBC2F0020FA
:10BD88007FB52E4E044600F11C05B4F85411B4F8E2
:10BD98005621881A83B2000444BF80339BB20BB982
:10BDA80004B070BD91421FBFB4F85811A3180132F6
:10BDB8000A4096F82D101ABF93F85A31A4F8562164
:10BDC8000023022904F110022946684620D1FEF713
:10BDD800EBFE9DF80030022BD7D1E368DBB9A068F1
:10BDE8000368BDF802201B692946984704F5CA660E
:10BDF8002A4669463046F6F76DFB31461048FDF78E
:10BE080029FA3146204604B0BDE87040FFF762BF0A
:10BE1800F6F7E8FBDDE70B4E69460020F6F7B2FDC2
:10BE2800737833B1A068BDF80220036829461B69FE
:10BE38009847B378002BD9D0E068D1E728030020D1
:10BE4800940600207D0500200148FFF717BF00BFBA
:10BE5800B815002070B5594C594E86B000211622ED
:10BE6800684605F045FA2046F5F797F994F88C30BE
:10BE78008DF800008DF80130204694F88D308DF84B
:10BE88000230F5F781F994F8913094F890208DF804
:10BE980003005B0002F0010203F00203134394F86D
:10BEA800A52043EA821394F8A62043EAC2139DF81A
:10BEB8000B2002F03C02134320468DF80B30F5F7B7
:10BEC8005AF905463046F8F717FD01462846F5F7B2
:10BED8001FFA94F893308DF8073094F8943094F85A
:10BEE80095208DF8083094F8963094F992508DF892
:10BEF8000400DB00920002F0040203F0080313437D
:10BF08009DF80B208DF8095022F00C02134330469F
:10BF18008DF80B30F8F7F0FC01462846F5F7F8F9EC
:10BF28008DF80A0004F12800F5F7B1FD8DF80C0032
:10BF38002046F5F7FEF88DF80D0004F11400F5F72A
:10BF4800A6FD8DF80E0004F13C00F5F7A0FD8DF874
:10BF58000F002046F5F7FEF88DF810002046F5F79B
:10BF68002DF994F8A7308DF81230164B8DF8110082
:10BF7800DB7D8DF81330FFF767FF134B1A78931E9C
:10BF88005A425A4100F0030343EA02230F4A104879
:10BF9800127943EA4223BDF8142023F0FC039B05E1
:10BFA80022F4407222F003029B0D134302216A46D9
:10BFB800ADF81430FBF714F806B070BDBC2F0020A4
:10BFC80064300020A00A00208D060020C005002053
:10BFD800D015002070B54C88B4F5427F03464FF069
:10BFE80000000AD80D780B2D77D8DFE805F0060F8A
:10BFF8001C2C2F32383B54575B6DA2F1240462424B
:10C00800488062410A7083F809033EE04D2A01D056
:10C01800582A06D11A7002220A70002083F80903F0
:10C0280070BD0022F8E702F0FD003C2801D0212A6B
:10C03800F7D15A701A784D2A0CBF082203220A70C9
:10C0480000229A70E9E79A700422DBE79A800522B9
:10C05800D8E7988800EB02229A800622DCE7DA808B
:10C068000722CFE7D88800EB022292B2002ADA80B2
:10C078000CBF0B220A220A7000224A80012283F890
:10C088000923DB88B3F5407F01D80020C8E70020EA
:10C0980008704880C4E7DA800922B3E79A800A2248
:10C0A8000A70EBE7B4F5407F3CBFE41822724A8877
:10C0B800013292B24A80D88890429CBF0B220A7003
:10C0C800012283F80923E0E783F808230222087095
:10C0D800488083F809230120A2E708704880D4E744
:10C0E800CB88B3F5407F70B531D8242303700B7823
:10C0F80043704B7883700B784D2B14D1CB88C37069
:10C108008B88037105230022CD88D4189542A6B2E6
:10C1180010FA84F415D891F808232270CA880132DD
:10C12800981880B270BD8B78C3708B8803718B8828
:10C138001B0A4371CB888371CB881B0AC371082300
:10C14800E1E78C180132247A845592B2DCE70020AA
:10C15800E8E700002DE9F74F16464A88B2F5427F16
:10C1680004460D462ED80B780A2B0FD9A3F164028A
:10C17800032A03D90020287068802DE0653B8F4F83
:10C18800022B33D8DFE803F063A4A70000210A2BB1
:10C19800F0D801A050F823F0CDC10008E7C100088D
:10C1A8007DC100087DC100082BC2000839C2000803
:10C1B80045C200084BC200087DC100087DC10008C7
:10C1C800B9C20008A6F124077E424FF000007E4164
:10C1D80068802E7084F8090303B0BDE8F08F6F2ED5
:10C1E8000CBF642300232B700020F3E716F0040F24
:10C1F80014BF4D2358233E7023703A78D1070ED4CC
:10C2080012F0020F14BF21233E236370C2F3C00350
:10C21800D20648BF43F00203A3700423E3E73C239C
:10C22800F3E7A68005232B7084F809130020D3E7D1
:10C23800A38803EB0623A3800623D4E7E68007231D
:10C24800F1E7E38803EB0623E3806523CBE70DF1F1
:10C2580006007E70F6F74AF83978F6F73FF8A788AF
:10C268002179F6F73BF8390AF6F738F8E788A17923
:10C27800F6F734F8390AF6F731F89DF80630B34284
:10C2880006D000232B706B80032384F80933CDE795
:10C29800002F0CBF66230A232B70012384F809336F
:10C2A80000236B80E288B2F5407FBFD92B70BDE7D1
:10C2B800B2F5407F3CBF121916726B8801339BB2EE
:10C2C8006B80E2889A4201D866232B700123DCE751
:10C2D8007E806723F9E7B7F8028097F8009008EBAB
:10C2E80006284FF6FF730DF106001FFA88F8494635
:10C2F800ADF80630A7F80280F5F7F4FE2679B4F811
:10C3080004A03146F5F7EEFE4FEA1A21F5F7EAFEEA
:10C3180094F806B0B4F806A05946F5F7E3FE4FEADC
:10C328001A21F5F7DFFE797804F10807F5F7DAFE48
:10C3380052463946F5F7E2FEBDF8063043453AD194
:10C3480019F0040015D086EA0B01E21D002398B20B
:10C35800824584F8081307D80223012000222A7096
:10C368006A8084F8093337E712F8010F0133414036
:10C37800EDE7A178F4F7E6FF217984F80803F4F7EC
:10C38800E1FFA18884F80803090AF4F7DBFFA17923
:10C3980084F80803F4F7D6FFE18884F80803090A4B
:10C3A800F4F7D0FFE28884F808033946F4F7D0FFA1
:10C3B80084F80803D0E703230020CFE7102E0020DD
:10C3C800CB88B3F5407F2DE9F04104460D464AD8A5
:10C3D8004B783C2B40D0A3F12100434243415B0002
:10C3E8002A784D2AAA7808BF43F00403D10748BF2A
:10C3F80043F0080392074FF02402227048BF43F02D
:10C4080010036F226270A370AB88E370AB881B0ABD
:10C418002371EB886371EB88A71C1B0AA37138464C
:10C42800F6F760FA0822E071E988A2F108039BB2E6
:10C43800561C8B42B6B204EB02080FD3063189B200
:10C448003846F5F773FE88F80000000AA055E8881A
:10C458000A3080B2BDE8F0810123C1E72B441B7A82
:10C46800A3543246E0E70020F4E710B5044681788B
:10C478000020F4F767FF217984F80803F4F762FFD6
:10C48800A18884F80803090AF4F75CFFA17984F805
:10C498000803F4F757FFE18884F80803090AF4F75A
:10C4A80051FFE28884F8080304F10801F4F750FF0B
:10C4B80084F8080310BD00002DE9F74FC788DFF89E
:10C4C80090800D4604463A4600F1080100262846A9
:10C4D80004F076FF55FA87F7E6804FF03B09BD4236
:10C4E80005D1204603B0BDE8F04FFFF7BEBF15F8F1
:10C4F800013BFF2B2AD0FE2B28D0FF2E1ED1362B36
:10C50800EDD858F833204FF0000A10460192F3F79F
:10C5180039FE5FFA8AFB5845E388019A0AF1010A55
:10C5280005D85A1C2344E28083F80890D7E7591CA1
:10C53800E180234412F80B101972E6E7FE2ECED1E3
:10C54800E288511C2244E1801372C8E71E46C6E700
:10C558004845010830B50F4B1C780F4B142505FBD7
:10C56800043393F84F30012B03D0022B10D00BB1BA
:10C57800FEE7114600234360C0F81233A0F82236C4
:10C58800A0F8203640F2FF330160A0F8243630BD11
:10C598000021EFE7CC02002028030020F8B5B0F80E
:10C5A8002026B0F82236D21A93B2120444BF03F5FB
:10C5B80080639BB2E62B044608D800F2163500F2D9
:10C5C8001236206803685B69984700B9F8BD20688F
:10C5D80003689B699847314602462846FFF7FAFCEC
:10C5E8000028EED004F6262729463846FFF7E8FE4D
:10C5F80000239AB29042E4D9B4F82016B4F824C6BD
:10C608004A1C02EA0C02B4F822C694451EBF091956
:10C6180017F803C081F826C603F1010318BFA4F870
:10C628002026E6E7F8B500F1080504460A46011D8C
:10C638002846FFF78FFD70B3637A3E2B14D004F6BB
:10C64800262629463046FFF74BFD0246206801683A
:10C658000F693146B847637A3E2B1CD129460E48EC
:10C66800BDE8F840FCF70EBEA389742B0AD042F649
:10C67800FF729B1A18BF0123A27A9207EBD4002BF2
:10C68800DDD1E8E70023A37204F626212846FFF748
:10C6980013FF0123F0E7F8BD9406002003680BB1EF
:10C6A800FFF7C0BF70470346006868B1B3F820269B
:10C6B800B3F82236D31A98B21B0444BF00F5806041
:10C6C80080B2003818BF012070470346006880B167
:10C6D800B3F82226B3F82016914209D099180132EE
:10C6E80091F82606B3F824160A40A3F822267047C4
:10C6F800002070470346006838B10022A3F82226BC
:10C70800A3F820260368DB691847704710B504466C
:10C718000548FEF77EFE0548FFF7ECFF60680368F2
:10C72800BDE81040DB691847100D0020D02000201C
:10C7380070B50A4C25780A4C142606FB054494F873
:10C748004F40012C03D0022C05D00CB1FEE719464E
:10C75800416011B9FEE71146FAE770BDCC0200202E
:10C7680028030020024B1A790AB901225A7170472E
:10C77800C0050020024B1A790AB101229A7170474C
:10C78800C0050020F8B572B6384D0024F6F740FD14
:10C798000226F7F77DF9F6F7EDFCF6F7DBFC3448EF
:10C7A800F7F72CF9F7F792FEC5E90444AC602E734D
:10C7B800F6F794FE2F4B1C70F6F706FC2E4B2F480D
:10C7C800D02283F83223F6F73FFD214628462C4D28
:10C7D80003F0C4F84FF47A70F6F736FDC5E904445F
:10C7E800AC602E73F6F700FF264B274E1C70F6F749
:10C7F80021FCF6F76DFC254B20484FF40052DA6017
:10C808000427F6F721FD41F28830B762F6F71CFDE0
:10C818004CF25030B761F6F717FD2846F6F73CFCA6
:10C82800214628461A4C03F099F84FF47A70F6F727
:10C838000BFD94F8572094F856101648FAF748FB61
:10C8480094F857101448FBF7FFFE94F85840134823
:10C858002146F5F7B7FA3CB1114B124A1A60124B50
:10C86800124A1A60FAF750F862B6F8BD6430002030
:10C87800340200203C02002000E100E0E0930400C4
:10C88800803000203D0200200004004800080058C5
:10C89800CC020020D015002094060020D00C0020E7
:10C8A800400200209121000844020020F92A0008D3
:10C8B80073B51648164C4FF6FF7103F09FF92080A8
:10C8C80023889B0712D5134E35798DB10F4808235D
:10C8D8006A46002103F013F8D6E90602DDE90013E1
:10C8E8009A4208BF884201D00023238002B070BD5D
:10C8F80002236A460548294603F001F8064BDA8BFD
:10C90800BDF800309A4218BF2580EFE76430002058
:10C91800FE0C0020C0050020CC020020184B4FF46C
:10C92800005273B5DA601748174C4FF6FF7103F0E1
:10C9380065F9208023889B0712D5144E35798DB16F
:10C94800104808236A46002102F0D9FFD6E90602FA
:10C95800DDE900139A4208BF884201D000232380F2
:10C9680002B070BD02236A460648294602F0C7FF96
:10C97800074BDA8BBDF800309A4218BF2580EFE7E5
:10C988000008005880300020FC0C0020C005002062
:10C99800CC020020044A00231370044A1380044A7E
:10C9A8001370044A137070470A0D00200C0D002004
:10C9B800C4300020940A0020024B1878B0FA80F0A6
:10C9C800400970470A0D00200D4A11780346A9B99D
:10C9D80010700C4A012010700B4A032B118009D0EB
:10C9E800042B01D083420AD1084B002283F872201D
:10C9F800012070474FF4FA73138070470020704786
:10CA08000A0D0020C43000200C0D0020E404002092
:10CA1800034A00231370034A1380034A13707047B4
:10CA28000A0D00200C0D0020C43000200A4A08B569
:10CA3800138883B1013B9BB2138063B9074B1B7802
:10CA4800032B02BF064B01221A70FFF7E1FF054BCB
:10CA5800002283F8FA2A08BD0C0D00200A0D0020D8
:10CA6800940A0020D015002010B5C379212B0ED1CF
:10CA7800074CF8F7D1F9FFF7CBFF94F8FA1A032916
:10CA880002D12046FAF78DFC002384F8FA3A10BD4B
:10CA9800D015002010B50D4B1B78013B032B14D883
:10CAA800DFE803F002090D072023BDE81040F8F77E
:10CAB800A3B92423F9E7BDE81040F8F7F7B9232311
:10CAC800F8F79AF9024B00221A7010BD0A0D0020DF
:10CAD800C4300020034B01221A7000225A711A71C7
:10CAE800704700BF7B2E0020054A064B12791B7F3A
:10CAF8001AB105495B22F8F745BC04495B22FAE7FD
:10CB0800C0050020CC020020C530002020310020C4
:10CB180038B5114B1A79054632B10146002218463C
:10CB2800BDE83840F8F762BC0C4A0D495B23F8F7BA
:10CB380019FC7DB90A48F8F75BF80128044607D0C4
:10CB480000280849284614BF01240224F8F73CFCB1
:10CB5800204638BD0148EEE7C0050020612F0020BF
:10CB6800062F0020BC2F0020024B1878831E584245
:10CB7800584170478D060020044B1B78022B06BFD6
:10CB8800034B93F872000020704700BF8D06002009
:10CB9800E404002010B5184B1A78184B04461420EA
:10CBA80000FB023393F85500012822D1228893060E
:10CBB80005D522F02002228005230B7010BD12F04B
:10CBC800400317D0FFF7D8FF28B1FFF7F5FE10B9DB
:10CBD80000230120F1E7606830B1094B1B681B1A7C
:10CBE800312BF5D90023636022F04002228006230E
:10CBF800EFE700231846E0E7CC02002028030020D6
:10CC08009C3F002013B50DF107010446FFF7C2FF52
:10CC180018B19DF8070002B010BD2080FBE70000A6
:10CC28002DE9F04106460C461546FFF7A5FF70B101
:10CC3800184B93F82D30581E012819D8164BB3F805
:10CC48005861B3F85671002291B28D4201D8BDE8FF
:10CC5800F081B3F85401411C3140B9421FBFC018DC
:10CC680014F802C080F85AC1A3F854110132EBE756
:10CC7800032B09D1094E0D44AC42E8D014F8011B2E
:10CC88003046FFF70BFDF7E770680368BDE8F04131
:10CC98001B69184728030020100D0020D020002011
:10CCA800F8B5214B214D1F79CB78C3F3000385F8E4
:10CCB80095304B79C3F3801385F896300646C878CB
:10CCC80040080C46F4F7ABFA85F892002379C3F3D1
:10CCD800060385F893306379227903F03F035B00FC
:10CCE80043EAD21385F89430E6B1DFB1A37803F0B4
:10CCF800F003202B04D12046BDE8F840FFF7B4BE6E
:10CD0800A2790B48E11D5208FFF78AFFA17905F1C6
:10CD180064004908F4F7BDFE05F13C00BDE8F840A1
:10CD2800F4F7B1BEF8BD00BF7B2E0020BC2F002059
:10CD38009C30002070B50546B8B9184B184E1B78C2
:10CD4800184A14794CBB022B174812D1B17801F05C
:10CD58000701F8F7A5FB4379C3B931460120FFF76E
:10CD68009FFF1248F4F7E2F909E0114B114E1B78C6
:10CD7800E6E701229342027044710471EDD80B4832
:10CD880080F89050BDE87040F4F7CEB90A4B1C7497
:10CD98005C825C61094B1C71DFE770BD060D0020E9
:10CDA800062F0020C00500207B2E0020BC2F00206D
:10CDB800070D0020612F0020100D0020D02000203A
:10CDC80010B50246FFF7D8FEB8B10C4B93F82D30DA
:10CDD800591E012904D8BDE810400948FEF7F6BAE3
:10CDE800032B04D1BDE810400648FFF75CBC50682F
:10CDF8000368BDE810405B69184710BD2803002090
:10CE0800100D0020D020002010B50246FFF7B4FE18
:10CE1800B8B10C4B93F82D30591E012904D8BDE840
:10CE280010400948FEF7E0BA032B04D1BDE81040D2
:10CE38000648FFF74ABC50680368BDE810409B6984
:10CE4800184710BD28030020100D0020D020002016
:10CE58002DE9F04FDFF8C88098F8004097B0814678
:10CE68000E461746002C53D12E4B1B78022B4BD164
:10CE7800DFF8B4B00DF1180A25465846ECB2FFF7B2
:10CE88009FFF40B15846FFF7BFFF0135402D0AF814
:10CE9800010BF2D12C4625482146F4F7FAFD244827
:10CEA800F4F7F1FD234D8DF8129095F8A4308DF824
:10CEB8000C30214B85F89190DB788DF80D302846A1
:10CEC80095F890308DF81130F4F755F98DF80E007B
:10CED800F8F74AF810F0010F8DF8130018BF3E4616
:10CEE80028468DF81460F4F758F998F800308DF852
:10CEF80010007BB9114A1248009406AB03A9F7F752
:10CF08006BFE17B0BDE8F08F0748FFF7FFFBC9E7D6
:10CF18000024C7E7094A0A4803A9FFF7BBFDF0E761
:10CF2800C43000208D0600209C3000200C300020EA
:10CF3800E42F0020BC2F00207B2E0020822E002012
:10CF48002031002030B4084C257925B1014620460F
:10CF580030BCF8F7CBB8054C94F8A430013384F80A
:10CF6800A43030BCFFF774BFC0050020BC2F0020E0
:10CF780008B50246FFF700FE18B9A2F82206A2F883
:10CF88002006054B93F82D30032B04D1BDE808404B
:10CF98001046FFF703BB08BD2803002070B5002327
:10CFA8009CB2A24200D870BD058886886C1C3440AB
:10CFB8004688A6421EBF2D18CE5CAE7103F1010350
:10CFC80018BF0480ECE708B56830FFF7E7FF08BD35
:10CFD800A0F11400F7E7000038B50A4B93F82D309C
:10CFE80000F5EF65022B0446284608D1FCF72CFE15
:10CFF8000246294604F24A40FFF7D0FF38BDF5F74C
:10D00800A2F9F5E7280300202DE9FF410446B0F80E
:10D018004C14B0F84A04F5F789FCE3684BBBDD28EB
:10D0280008D804F5F37604F5ED75A06803685B6924
:10D03800984710B904B0BDE8F081A06803689B69FF
:10D0480098472A46034631466846F5F7CBFA002842
:10D05800EBD09DF80030022BECD104F5CA653246BE
:10D0680069462846F5F736FA29462046FFF7B4FF01
:10D0780094E0DD28DED84D4D2B780133DBB2012B4F
:10D088002B700FD900232B70A06803685B69984741
:10D0980050B901232B70E06803685B69984730B981
:10D0A800287004E0002BEFD02B78012BF3D004F587
:10D0B800F37604F5ED772B78002B36D1A06803685A
:10D0C8005B69984788B3A06803689B6998473A46A4
:10D0D800034631466846F5F785FA0028EBD0DFF8B5
:10D0E800D08069460120F5F74DFC98F8023033B13D
:10D0F800E068BDF80220036831461B6998479DF82F
:10D108000030022B11D104F5CA6732466946384609
:10D11800F5F7E0F998F800301BB139462046FFF7DB
:10D128005BFF39462046FEF763FB04F21E3604F225
:10D1380012372B78012B7FF47DAFE06803685B69B9
:10D14800984700283FF476AFE06803689B699847E2
:10D158003A46034631466846F5F744FA0028E8D0CF
:10D16800134F69460220F5F70DFC7B7833B1A068B0
:10D17800BDF80220036831461B6998479DF80030C6
:10D18800022B7FF457AF04F5CA6532466946284634
:10D19800F5F7A0F93B78002B7FF466AF29462046C7
:10D1A80004B0BDE8F041FEF723BB00BFBC0500207A
:10D1B8007D0500201D4B70B51D680446FFF7DCFC9B
:10D1C80058B9C4F8A458A4F85601A4F85401A4F80E
:10D1D8004C04A4F84A0484F8AD08154E96F82D308E
:10D1E800013B012B21D82046FEF7CAFD2046FFF758
:10D1F8000BFF104B1B78142202FB036696F8523083
:10D2080063B1D4F8A438EB1AB3F57A7F08D3C4F81D
:10D21800A4582046BDE87040FEF710B9C4F8A458D9
:10D228002046BDE87040FEF705BC70BD9C3F00205D
:10D2380028030020CC0200202DE9F04FDFF8A08160
:10D24800684C98F80030012B87B000F269810BB95F
:10D25800F5F764FEFFF796FA616C6348F6F746FB4C
:10D26800624B00221A809A70614B08229A62072545
:10D278004CF25030013DF5F79DFFF5F7E5FF15F04D
:10D28800FF05F5D15B4802F0E8FC013880B24FF6A3
:10D29800FD76B04203D958490120F8F7CFF857482E
:10D2A80002F0DBFC013880B2B04202D954490220B6
:10D2B800F3E7544B1D80544B1D8094F8523013B93A
:10D2C80094F8543043B14B485049F7F7F7F97D20AB
:10D2D800F5F7BAFFF5F7A6FE94F8533013B994F8AA
:10D2E800553043B145484A49F7F7E8F97D20F5F745
:10D2F800ABFFF5F721FF4748F7F750FE94F820B049
:10D30800BBF1200F00D9FEE794F82870424EA38D98
:10D318000393052F616A94F829C094F82A30B771ED
:10D3280000D9FEE73D4A380102EB071E125802B940
:10D33800FEE7DEF808009EF80C90B26030619EF8B7
:10D34800042002920020F27186F80C9086F8D970B9
:10D35800B08282468646039A0241D20707D5012247
:10D3680002FA00FA4EEA0A0A1FFA8AFE92460130C9
:10D378000628F0D12848BAF1000F01D0A0F814E02F
:10D38800B0F814E0BEF1000F00D1FEE7029AA2EB5C
:10D398000902D2B25A4528BF5A46052FC27500F075
:10D3A800F980012F00F2FE800CF1FF37FFB200F088
:10D3B800E880022F34D85D1EEDB2032D09D80C2A5F
:10D3C80001D90C25C575C57D954200D9C27565463C
:10D3D80029E0122A84BF1223C3750023F3E700BF94
:10D3E800A82E0020CC02002034020020020D0020CC
:10D3F8000004004864300020261E01088030002008
:10D40800301E0108FC0C0020FE0C0020D002002079
:10D41800DC020020C0050020A00A00200028010826
:10D42800052B28BF002369482A46F4F789FA002506
:10D43800674B86F8D850B5756448FF261E705E7035
:10D44800F7F780FA0146634802F0ADFA5F48F7F74C
:10D4580079FA0146604802F0A6FA604B1D80604BDD
:10D468001D70604B1D70604B1D80604B1D80604BB4
:10D478001D70604B1D80604B1D70604B1D70604BB4
:10D488001D70604B01201D70FFF784FAFFF79CFAAE
:10D49800B4F84830B4F84A2094F840105A48F3F7E2
:10D4A80009FEB4F848105948F4F751F95848F7F705
:10D4B800CDFF2278574B5848142101FB023393F8CB
:10D4C8004E10F4F787FC554B554A56495648FEF717
:10D4D80053FB524A53495548FFF73CF81346514904
:10D4E8004F4A5348FFF724F9B4F8482051495248A5
:10D4F800F8F7F6FA3748F7F716FA5048F4F7FEFA4D
:10D508004F48F4F7D6FA4F48F4F726FC4E4B1D70F7
:10D518004E4B1D804E4B1D80F6F782FA88F800604E
:10D52800F6F788FA2F4D002800F0B580314A1388A5
:10D538000BB1013B1380294A13880BB9B4F8483062
:10D54800013B9BB2012B138030D1254A1370FFF7A2
:10D558006DFA2B78002B40F09E80254B3D4A1978B8
:10D56800138802292BD173B3013B9BB213809278A5
:10D57800002A73D0002B7AD1F5F70EFEF5F71AFEC4
:10D5880075E0022F04D80C2A01D90C23C37565460F
:10D59800002348E70CF1FF33022BF9D8082AF6D903
:10D5A8000823F3E70948F4F765F940E7002BCED1E3
:10D5B80001232B70284B5A6A0B4B1A80C7E7002BA4
:10D5C800D2D1C723D2E740F2F313CFE7A00A002055
:10D5D800A92E002064300020803000207C310020FB
:10D5E800000D0020950A0020782E0020080D00204C
:10D5F8008D060020900600208E0600208C06002054
:10D60800070D0020060D0020BC2F0020B0300020A0
:10D618007B2E002028030020D00C00203802002098
:10D62800E415002034020020100D0020D020002036
:10D638009C30002000000020F4050020903F0020CE
:10D64800A430002084060020A62E0020C030002030
:10D65800C2300020020D0020004401400229A048E9
:10D6680040F0B9800BB9F5F797FD082383629D4E0A
:10D678003388002B00F0B580013B9BB29A48338079
:10D68800F7F7D0FC9948F7F74EF933881BB9984952
:10D698009848F5F79FFA984E3388022B00F0A4803B
:10D6A800042B00F0D180012B0FD1944B9A7DD97DAA
:10D6B8000132D2B2914298BF00229A75904B11461E
:10D6C800187AFFF73FFC0223338094F8523013B9DD
:10D6D80094F854300BB38B4F3B889BB2EBB1338833
:10D6E800032B40F0DF803B88D80703D500233B801D
:10D6F800042333803B889BB27BB13B883B889A07E5
:10D7080048BF3B883B88804ADB0748BF3B880023EB
:10D7180013707E4A3B803380137094F8533013B9EA
:10D7280094F855300BB37A4F3B889BB2EBB13388F2
:10D73800032B40F0C5803B88D80703D500233B80E6
:10D74800042333803B889BB27BB13B883B889A0794
:10D7580048BF3B883B886C4ADB0748BF3B880023AF
:10D7680013706A4A3B80338013702B78002B00F0CB
:10D77800DC8100235D482B70F7F74CF86548DFF82B
:10D788008891DFF888A1644DF7F744F894F852308F
:10D7980094F85320002B00F056819346002A00F09D
:10D7A80061819AF80030002B40F0C48099F800B0ED
:10D7B800BBF1000B18BF4FF0010B99F80030012B9B
:10D7C80094BF00230123BBF1000F40F05A819B4610
:10D7D800FFF780F9C4E010228262002B7FF447AF84
:10D7E800CCE640F2E73349E74C4B4D4A5B6A128876
:10D7F8009B1A9BB240F2ED2293427FF666AF494BEB
:10D80800494800271F70F7F755FE3C48F7F79AF884
:10D818000146364802F0C7F83848F7F793F801464A
:10D828003C4802F0C0F8364B187AFFF75DF903233D
:10D838003380374B3D481F80324B1F803C4B0122C1
:10D848001A71F4F75FF940E794F852306BB1274842
:10D858004FF6FF71F5F7DEFB02F03BF92348002194
:10D8680002F06BF97D20F5F7EFFC94F853306BB1BB
:10D8780028484FF6FF71F5F71FFC02F02AF92548F2
:10D88800002102F05AF97D20F5F7DEFC1E4A052337
:10D898003380002313701D4A13701D4A1380194AE0
:10D8A800138012E7052B7FF425AF3B8899077FF596
:10D8B80021AF00203880FFF72BF9144B187019E7B7
:10D8C800052B7FF43FAF3B8899077FF53BAF0023DB
:10D8D80001203B80FFF71CF90B4B187032E700BFA3
:10D8E80000040048C0300020C0050020643000203B
:10D8F8003E14010804000020080D0020A00A0020A2
:10D90800B0300020FE0C0020070D0020060D00207E
:10D91800FC0C002080300020BC2F00200044014077
:10D92800782E0020000D0020A92E0020903F002016
:10D9380094060020012B3FF440AF94F85330002B9D
:10D9480000F08D8095F98D30009395F98C3099F819
:10D9580000209AF800109C48F3F7E2FEFFF7EAF976
:10D9680094F854009AF8001099F8002094F855306B
:10D97800002800F08880002B00F08A8095F98D300F
:10D98800009395F98C309148F3F7FCFE904FBB7DDE
:10D9980085F8A7309AF80030012B94BF00230123A3
:10D9A80085F8A53099F80030012B94BF0023012396
:10D9B80085F8A630874D2B78BBF1000F07D0002BD8
:10D9C80069D0012B6CD0844BB4F84C201A802B788A
:10D9D800022B03D1804B1B8803B92B702A780023B4
:10D9E8000120022A30808AF8003089F8003006D0F9
:10D9F8007A490B701AB9FFF70BF8FEF7E5FF784A7A
:10DA080013880BB9B4F84A30013B9BB2138013B9A1
:10DA18007448F3F7D6FB7348F3F785FB2B78022B92
:10DA280002D07048F3F72EFB6F4B1E78002E5BD0A8
:10DA38006E4B08229A6110229A61F6F72BFD01239A
:10DA480088F800305AE06AB199F80030012B94BF89
:10DA58004FF0000B4FF0010B002B3FF4B9AE94F8D8
:10DA680053007BE79AF80020012A94BF4FF0000B7F
:10DA78004FF0010B002A3FF4ABAE002B7FF45DAFF3
:10DA8800EDE79B4659E71BB1504B01221A727DE71F
:10DA98004E4B0022FAE701222A70554A137092E78A
:10DAA800534A544913780133DBB213700A78AAB980
:10DAB80094F85000834286D34F4890F8723043B9A7
:10DAC8004E4B1B792BB95AB1FEF7A2FF012380F800
:10DAD800723002232B7001230B7074E70520E9E7ED
:10DAE80047490C20FFF7D9BB4448F7F7C5FAF7F7C1
:10DAF800EFFA0128044604D00328A0D007B0BDE8F7
:10DB0800F08F3E48F7F766FA41F28833A7F8DA3023
:10DB1800364B87F8D8401022A7F8DC609A610822B3
:10DB28009A62384B2E709C70E8E794F85630364D60
:10DB3800EBB136493648F9F705FA68B12278354B22
:10DB4800142101FB0233012293F84C30032B04BF4C
:10DB580001232B702E4B1A712D480DF11301F9F783
:10DB680009FA20B19DF81330FBB1012B20D094F8AD
:10DB7800563023B994F85730002B00F0128124480E
:10DB88000DF11301F9F71BFA002857D09DF813304F
:10DB9800033B0F2B52D8DFE803F03F51516E515130
:10DBA800517051768C9A9FA5A1A3FEF753F9DEE731
:10DBB800174805A9F9F731FA0028D8D09DF81400BC
:10DBC800F9F70CFDD3E700BFA72E0020B0300020E6
:10DBD800A00A00208D060020900600207B2E002041
:10DBE800C2300020BC2F0020940A00200004004806
:10DBF8008E0600208C060020E4040020C0050020CA
:10DC08003B1E0108020D0020A62E0020822E0020B7
:10DC1800D015002028030020F6F74CFCA04B1B78F9
:10DC2800022B07D10420FEF7CFFE9E4B032283F878
:10DC3800FA2A03E003219B48F9F7B3FB94F857301D
:10DC4800002B00F0AE8098499848FAF753FD08B1C8
:10DC580001232B70B4F84820944804A9FAF76CFD06
:10DC680000284CD09DF81030042B48D8DFE803F08A
:10DC7800415B5F6393000621DDE78D49A1F1330025
:10DC8800F9F766FBDAE7874F05A907F13300F9F7DB
:10DC980087FC0028D2D09DF81430002BCED0804BC2
:10DCA80018780228CAD1FEF78FFE0C2387F8FA3AB3
:10DCB800C4E77B4B1B78022B05D10320FEF784FEBB
:10DCC800784B0D22B3E77B4B01221A70B6E701218E
:10DCD8007948F3F708FFB1E70221F9E70321F7E7ED
:10DCE8000821F5E76F4B754893F83310F4F738F8C7
:10DCF800A4E76E48FBF798FB714B00221A706B4F34
:10DD08000DF111013846FAF751FD002849D09DF868
:10DD18001130022B43D8002B00F08980664801217E
:10DD2800F3F7E3FE3DE06148FBF7C6FBE7E75F4832
:10DD3800FBF7FAFBE3E7624F3B784BB959480DF123
:10DD48001201F9F76AF918B19DF81200F9F746FCC3
:10DD580054480DF1130205A9F9F7A4F868B19DF824
:10DD6800132005995148FAF775FD3B780133DBB26A
:10DD7800022B88BF00233B70C1E7FEF7FDFE002899
:10DD8800F3D0504B93F82D30013B022BEDD8474888
:10DD9800FAF72AFFE9E74548FBF7F4FBAFE7032B5F
:10DDA8004BD094F8583023B13F494748F4F739F934
:10DDB80008B92B78BBB100232B70424D23783A4920
:10DDC8004248142707FB035393F84D20F3F750F903
:10DDD800237835493E4807FB035595F84A3095F8AE
:10DDE8005620F7F791FB3B4B1B78002B7FF486AE50
:10DDF8003388022B3FF482AE3748FFF7DBF9374808
:10DE0800FFF7B6F83648F3F78AFE2B48F3F756FEC5
:10DE180010B93148FEF7F6FE431E0B2B73D8DFE826
:10DE280003F03B616472152933727266726E97F85B
:10DE380069102248F3F794FFB3E7BA7D1948023A0C
:10DE4800D2B207F11801F9F718F8AAE7144B1878B5
:10DE5800022805D1FEF7B8FD124BFF2283F8FA2AF3
:10DE68001648F3F791FF00283FF448AE114B012202
:10DE78001A7043E60A4B1B78022B01D10320E9E70D
:10DE88000C4B01221A70EBE7F6F714FB044B1B78D6
:10DE9800022BE5D10420DDE7FEF764FCE0E700BFD4
:10DEA8008D060020D0150020822E00209406002028
:10DEB80003160020940A0020A430002084060020C5
:10DEC800B705002028030020D00C0020EC05002016
:10DED800A92E0020000D0020100D0020D0200020C9
:10DEE800903F0020FEF746FCBAE7F4F7D5FF084854
:10DEF800F3F702FEC1B20748F3F732FFB0E7044870
:10DF0800F3F7FAFDACE704283FF499ADA8E700BFA2
:10DF1800A43000208406002008B5FFF78DF9FCE73F
:10DF280038B5254B254A1A60254B264A1A60264BD8
:10DF3800264A1A605A619A62DA63254A1A655A664D
:10DF4800244A9A67244A254B254802F108012832B9
:10DF580000245A6140F2FF12C3E91A427F25214A80
:10DF68001960C3F87022C3F86C42C3F8744AC3F846
:10DF7800785A1D4B036000F58E70FAF71DFA1B4B9B
:10DF88001B4A1A601B482146F3F722F81A4B1B4A12
:10DF9800C3F84C24C3E95545A3F84A44184B40F24A
:10DFA800FF32C3F82426C3F82046164B164A1A60D7
:10DFB800164B174A1A6038BD643000205C1E0108F1
:10DFC80080300020841E0108BC2F0020981501080D
:10DFD800801501088C15010854470108D015002048
:10DFE800940600200000FF074C470108D00C0020D1
:10DFF8006C1F0108EC050020100D00200000FF0137
:10E00800D02000209C30002008470108903F0020C5
:10E018003847010830B59BB0202200210BA803F037
:10E0280067F91822002102A803F062F91C4A136854
:10E0380023F4C06343F400731360136803F4C063EC
:10E048000193019B01224FF40413CDE90823002317
:10E058000A9310210623CDE915134FF40033022447
:10E06800032517934FF0005C4FF0007308A8CDE923
:10E078001345CDE9183C00F045FB08B172B6FEE740
:10E08800CDE90400CDE906004F23214602A8CDE9D9
:10E09800023500F0D1FD08B172B6FEE71BB030BD05
:10E0A80000040058154B07B51A6842F480721A60CC
:10E0B8001A6842F400721A601A6822F480621A60C0
:10E0C80000F0A0F8FFF7A6FF4FF0B043DA6C42F07B
:10E0D8000102DA64DA6C02F001020192019ADA6C48
:10E0E80042F00202DA64DB6C03F002030093009B47
:10E0F80003B05DF804EBFFF70FBF00BF0040005806
:10E108007047FEE7FEE7FEE7FEE7FEE77047704769
:10E118007047F5F79FBC70470D488546FFF7FBFF32
:10E128000C480D490D4A002302E0D458C45004336A
:10E13800C4188C42F9D30A4A0A4C002301E0136040
:10E148000432A242FBD303F00FF9FFF7ABFFFEE75F
:10E158000000012000000020AC0200208C4D0108C6
:10E16800B002002010410020FEE770474FF0B04396
:10E1780010B59A6B4FF0FF329A63D96BDA630024BB
:10E18800996B9C63D96BDC63196C1A64196C1C64F9
:10E19800596C5A64596C5C64996A9A62996A9C626F
:10E1A800D96ADA62D96ADC62196B1A631A6B1C6362
:10E1B800FFF7DBFF204610BD38B5104C2378054625
:10E1C8000BB9012038BD00F08DFA22784FF47A732C
:10E1D800B3FBF2F3B0FBF3F000F074F80446002848
:10E1E800EFD10F2DEDD8024629464FF0FF3000F051
:10E1F80037F8034B20461D60E4E700BF4C020020BF
:10E208005002002010B5032000F018F800F06AFA58
:10E21800064B18600F20FFF7CFFF044618B9FFF729
:10E228006FFF204610BD0124FBE700BF4802002015
:10E23800014B1868704700BF9C3F00200749CA6817
:10E2480022F4E0620302120403F4E063120C1343A5
:10E2580043F0BF6343F40033CB60704700ED00E048
:10E26800164B30B5DC68C4F30224C4F10703251D3E
:10E27800042B28BF0423062D4FF0FF358CBF033C29
:10E28800002405FA03F321EA0303A54022EA050264
:10E29800A340002843EA0203ACBF00F16040084AEB
:10E2A8004FEA0313B8BF00F00F00DBB2AABF00F5B6
:10E2B8006140135480F8003330BD00BF00ED00E02A
:10E2C80014ED00E00138B0F1807F0BD24FF0E0236D
:10E2D800054A5861F02182F823100020072298612E
:10E2E8001A6170470120704700ED00E00A4A53693F
:10E2F80043F4802330B55361EFF3108472B60023E2
:10E30800CD58C5500433B3F5807FF9D11369DB03C9
:10E31800FCD484F3108830BD00400058064B5A697D
:10E32800002ABFBF054A9A6002F188329A60BABFD4
:10E338005869C00F00207047004000582301674506
:10E34800044B5A6942F000425A615869C043C00FF1
:10E35800704700BF0040005870B50546FFF768FFDA
:10E36800124E04463369D90313D43369DA0744BF1C
:10E37800012232614CF2FA32134011D10B4E30694E
:10E3880010F480200BD0FFF753FF001BA842F6D3F0
:10E3980004E0FFF74DFF001BA842E3D3032070BD44
:10E3A800024A1361024A01205360F8E7004000580E
:10E3B800A03F00202DE9F041184D98462B78012BFD
:10E3C80006460C46174626D001232B704FF47A7068
:10E3D80000236B60FFF7C0FFA0B9012E16D1104AC9
:10E3E800536943F0010353612760BFF36F8FC4F88B
:10E3F80004804FF47A70FFF7AFFF094A536923EAA4
:10E408000603536100232B70BDE8F081394620468E
:10E41800FFF76CFFEDE70220F6E700BFA03F002002
:10E4280000400058054A536923F47E7343EAC0004C
:10E4380040F4803040F002005061704700400058BE
:10E448002DE9F041234F3B78012B054688463FD004
:10E4580001233B704FF47A7000237B60FFF77CFF49
:10E46800044688B92B68042B13D11B4A536943F41B
:10E47800803343F0040353614FF47A70FFF76CFF65
:10E488000446154B1A681B6800233B702046BDE8FC
:10E49800F0814FF0FF33C8F800306E68D5E90132DB
:10E4A8001344B3420AD93046FFF7BCFF4FF47A70E1
:10E4B800FFF752FF50B1C8F800600446064A536996
:10E4C80023F47E7323F002035361DAE70136E5E7AC
:10E4D8000224DBE7A03F002000400058024A1368EE
:10E4E80043F480731360704700040058024B1868A7
:10E4F80000F4C060704700BF000400584FF0B043FC
:10E508001868C0F3404070474FF0B0431868C0F334
:10E51800400070474FF0B042536823F47F4343EA0A
:10E528000023536070474FF0B0431868C0F3406051
:10E53800704700007FB54FF0B0432C4AD3F808313C
:10E54800C0F3031003F00F0352F82040284A52F892
:10E558002330B4FBF3F4FFF7C9FF264B054693E8D5
:10E568000700B5F5007F04AB03E9070010D0224B84
:10E578009C4218D303F5B70303F67F539C4229D96D
:10E5880003F5741303F510639C4225D802230BE0AE
:10E598001A4B9C4207D91A4B9C421BD903F53703E7
:10E5A80003F5D853F0E7002304AA02EB830353F8DA
:10E5B8000C4C144D2B6823F0070323432B60FFF703
:10E5C80037FE06462B6803F007039C4206D100205D
:10E5D80004B070BD0123E7E70024EAE7FFF728FE4F
:10E5E800801B0228EED90320F2E700BF0448010887
:10E5F800A447010824140108C0CF6A00BFEA21011A
:10E608003F933402004000584FF0B04310B59A6869
:10E61800D96812F00C0205D00C2A4AD101F0030384
:10E62800012B50D14FF0B0412B480B6813F0080371
:10E6380006D00B6813F0080337D1D1F8941007E01F
:10E648000C68240756BFD1F894300968C3F3032334
:10E6580050F82330002A0CBF184600204FF0B04174
:10E668008A6802F00C020C2A1ED1CA6802F0030262
:10E67800022A2ED0032A06D10B68184A13F4801FE9
:10E68800174B18BF13464FF0B042D068D168D26814
:10E69800C0F306205843C1F302130133B0FBF3F073
:10E6A800530F0133B0FBF3F010BD0B68C3F3031332
:10E6B800CEE7042A0AD0082A05D11B6813F4801370
:10E6C80004D10748CAE700231846C7E703480023D0
:10E6D800C4E7024BD7E700BF044801080024F40050
:10E6E8000048E80108B5FFF78FFF4FF0B043044A30
:10E6F8009B68C3F3031352F82330B0FBF3F008BD53
:10E70800A44701082DE9F0410446002853D04FF0F2
:10E71800B0439D68DE6803689B0605F00C0506F0AB
:10E72800030668D5026A1DB10C2D46D1012E44D1CD
:10E73800002A40D04FF0B043A16A1A68170756BFA5
:10E74800D3F894301B681B0903F0F00399421FD9D2
:10E758000846FFF7EFFE00282DD14FF0B0421368AE
:10E7680043F0080313601368A16A23F0F0030B4316
:10E778001360606AFFF7CEFEFFF7B4FFAB4B18607B
:10E78800AB4B1868FFF718FD002834D0BDE8F081BE
:10E798004FF0B042136843F008031360136823F086
:10E7A800F0030B431360606AFFF7B4FE0846FFF7F7
:10E7B800C1FE0028E0D00120E8E74FF0B043002A6E
:10E7C80054D01A6842F001021A60FFF731FD07467B
:10E7D800FFF79AFE002842D04FF0B042136843F08A
:10E7E800080313601368A16A23F0F0030B43136056
:10E7F800606AFFF78FFE2368D80748D42368990713
:10E8080000F18C8023681E0740F1FA80A3694FF05D
:10E81800B046002B00F0E180D6F89430E16903F0AF
:10E828001002914200F0C48003F00302022AC2D011
:10E83800D80740F1B380D6F8943023F00103C6F826
:10E848009430FFF7F5FC0746D6F89430990740F165
:10E85800A580FFF7EDFCC31B112BF5D904E0FFF7EA
:10E86800E7FCC01B0228B3D903208FE71A6822F0FF
:10E8780001021A60FFF7DCFC0746FFF745FE002897
:10E88800B9D0FFF7D5FCC01B0228F6D9ECE7082D54
:10E8980003D00C2D05D1032E03D16368002BADD115
:10E8A80089E74FF0B043A1681A6822F480120A433E
:10E8B8001A606268B2F5803F10D11A6842F480325B
:10E8C8001A60FFF7B5FC0746FFF718FE002895D138
:10E8D800FFF7AEFCC01B6428F6D9C5E7B2F5041FE4
:10E8E80004D11A6842F400121A60E6E7196821F4A4
:10E8F80080311960196821F400111960002AE0D1EB
:10E90800FFF796FC0746FFF7F9FD00283FF476AFBE
:10E91800FFF78EFCC01B6428F5D9A5E7042D2369F1
:10E9280003D00C2D0ED1022E0CD1002B3FF443AF97
:10E938004FF0B0426169536823F0FE4343EA016334
:10E9480053605FE74FF0B046BBB1336843F4807360
:10E958003360FFF76DFC074633685A0507D57368BF
:10E96800626923F0FE4343EA026373604AE7FFF7F4
:10E978005FFCC31B022BEFD976E7336823F480735F
:10E988003360FFF755FC074633685B057FF53AAF00
:10E99800FFF74EFCC31B022BF6D965E74FF0B042D8
:10E9A800E169D2F8943023F010030B43C2F8943095
:10E9B8004FF0B047D7F8943043F00103C7F89430CC
:10E9C800FFF736FC0646D7F894309A0718D4FFF7B5
:10E9D8002FFC831B112BF6D946E7D6F8943023F089
:10E9E8000103C6F89430FFF723FC0746D6F89430A5
:10E9F8009B0705D5FFF71CFCC31B112BF6D933E782
:10EA08002368580754D50B4F3B68D90514D4FFF732
:10EA180065FDFFF70DFC06463B68DA050CD4FFF7E9
:10EA280007FC831B022BF7D91EE700BF4802002012
:10EA38005002002000040058E3684FF0B046002B55
:10EA480058D023F08003052B02BFD6F8903043F04E
:10EA58000403C6F890304FF0B046FFF7E9FBD6F84C
:10EA6800903043F001030746C6F8903041F28838E9
:10EA7800D6F890309B0705D4FFF7DAFBC31B434554
:10EA8800F6D9F1E6E36823F00403812B1BD1FFF7E5
:10EA9800CFFBD6F8903043F08003C6F89030074695
:10EAA8004FF0B04641F28838D6F89030180504D5B2
:10EAB800E06A00284AD1002068E6FFF7B9FBC01BCE
:10EAC8004045F1D9D0E6FFF7B3FBD6F8903023F0F4
:10EAD8008003C6F8903007464FF0B04641F28838B8
:10EAE800D6F890301905E3D5FFF7A2FBC01B4045C7
:10EAF800F6D9B9E6FFF79CFBD6F8903023F08003EF
:10EB08000746C6F8903041F28838D6F890301A0592
:10EB180016D4FFF78DFBD6F8903023F00103C6F822
:10EB2800903007464FF0B04841F28836D8F8903018
:10EB38009B07BDD5FFF77CFBC31BB342F6D993E611
:10EB4800FFF776FBC01B4045DFD98DE60C2D4ED074
:10EB58004FF0B04302281A6822F080721A6033D14D
:10EB6800FFF766FB0546FFF7DEFC38BBD4E90C313E
:10EB78004FF0B0420B43D0682D4901400B43E16B85
:10EB88000B43216C0B43616C0B43A16B43EA0123DC
:10EB9800D360136843F080731360D36843F08053E5
:10EBA800D360FFF745FB0446FFF7BDFC002882D180
:10EBB800FFF73EFB001B0A28F6D955E6FFF738FB9E
:10EBC800401B0A28CFD94FE6FFF732FB0446FFF770
:10EBD800AAFC30B94FF0B042164BD1680B40D36055
:10EBE800D4E5FFF725FB001B0A28F0D93CE60128ED
:10EBF8003FF4CCAD4FF0B043226BDB6803F0030168
:10EC080091427FF4D8AD616B03F070028A427FF4C1
:10EC1800D2ADA16B03F4FE42B2EB012F7FF4CBAD72
:10EC2800626C03F0604393423FF445AFC3E500BF15
:10EC38008C80C111FCFFFEEE2DE9F0410D46044623
:10EC480010B90120BDE8F081684E336803F007036E
:10EC58008B4216D323689A0727D54FF0B047A2688E
:10EC6800BB6823F0F0031343BB60FFF7E1FA0646E5
:10EC7800BB68DB0319D4FFF7DBFA831B022BF7D938
:10EC880011E0336823F007030B433360FFF7D0FA32
:10EC98000746336803F00703AB42DBD0FFF7C8FA37
:10ECA800C01B0228F5D90320CCE72368580617D5DE
:10ECB8004FF0B0476269D7F8083123F00F0343EAF1
:10ECC8001213C7F80831FFF7B3FA0646D7F8083128
:10ECD800D90305D4FFF7ACFA831B022BF6D9E2E778
:10ECE80023685A0713D54FF0B047E268BB6823F48E
:10ECF800E0631343BB60FFF79BFA0646BB689B03C0
:10ED080005D4FFF795FA831B022BF7D9CBE72368C5
:10ED1800180714D54FF0B0472269BB6823F4605335
:10ED280043EAC203BB60FFF783FA0646BB68590390
:10ED380005D4FFF77DFA831B022BF7D9B3E72368C5
:10ED4800DA070FD4294C236803F00703AB4239D8FC
:10ED5800FFF7C8FC264B1860264BBDE8F041186841
:10ED6800FFF72ABA6268022A1DD1FFF7C7FB0028FD
:10ED78003FF467AF4FF0B04641F28838B36823F0EC
:10ED880003031343B360FFF753FA0746B368626897
:10ED980003F00C03B3EB820FD4D0FFF749FAC01B82
:10EDA8004045F3D97FE7032A02D1FFF7BCFBDEE732
:10EDB80012B9FFF7A9FBDAE74FF0B0431B685B0510
:10EDC800D8D43EE7236823F007032B432360FFF7DB
:10EDD8002FFA0646236803F00703AB42B8D0FFF7C3
:10EDE80027FA801B0228F5D95DE700BF00400058CC
:10EDF800480200205002002030B5046891FAA1F3BF
:10EE0800B3FA83F303255B0005FA03F324EA03034B
:10EE180091FAA1F1B1FA81F149008A401A430260DE
:10EE280030BD0000B0F1904F0BD14FF0B043DA6A1B
:10EE380042F00102DA62DA6A22F00102DA620120A3
:10EE48007047144B984209D14FF0B043DA6A42F048
:10EE58000202DA62DA6A22F00202EFE70E4B984207
:10EE680009D14FF0B043DA6A42F00402DA62DA6A92
:10EE780022F00402E2E7094B984209D14FF0B0436F
:10EE8800DA6A42F08002DA62DA6A22F08002D5E7B2
:10EE9800002070470004004800080048001C004893
:10EEA8002DE9F84F0E460F6897FAA7F54FF0010BBA
:10EEB800B5FA85F54FF0030A4FF00F0837FA05F356
:10EEC80002D10120BDE8F88F0BFA05F43C4053D07D
:10EED800D6F8049021464A46FFF78EFF09F1FF3322
:10EEE800012B19D8B368816894FAA4F2B2FA82F2B5
:10EEF80052000AFA02F221EA020294FAA4F1B1FAE3
:10EF080081F149008B40134383604268F36822EA29
:10EF180004026343134343603369C16894FAA4F25B
:10EF2800B2FA82F252000AFA02F221EA020294FAD2
:10EF3800A4F1B1FA81F149008B401343B9F1020FF2
:10EF4800C36015D1FF2C716918D8026A94FAA4F32A
:10EF5800B3FA83F39B0008FA03F322EA030294FA54
:10EF6800A4F3B3FA83F39B0001FA03F31343036298
:10EF78004A462146FFF740FF01359FE7426A230AC8
:10EF880093FAA3FCBCFA8CFC4FEA8C0C08FA0CFC34
:10EF980022EA0C0293FAA3F3B3FA83F39B00994095
:10EFA80011434162E4E74FF0B0431868C0F30050E2
:10EFB80070474FF0B0431868C0F3802070474FF097
:10EFC800B043D3F89000C0F3400070474FF0B0430F
:10EFD8001868C0F3C00070474FF0B0431868C0F31A
:10EFE800406070474FF0B043044A9B68C3F3031373
:10EFF80052F82330B0FBF3F0704700BFA447010874
:10F008004FF0B043034A9B68C3F3022352F82330FE
:10F01800D8407047E44701084FF0B04238B59168CE
:10F0280001F00C01082950D017D889B3042900F041
:10F038008C80FFF7CBFF46490246002876D1FFF7C0
:10F04800C5FF4FF0B043012816BFD3F894201B68C2
:10F05800C2F3032251F822002AE00C29E9D1D3682F
:10F0680003F00303022B5FD0032B37D0FFF7AEFF6B
:10F07800374C014600284AD1FFF7A8FF012816BFE0
:10F08800D2F894101368C1F3032154F821302CE00E
:10F09800FFF79CFF2E4D044658B9FFF797FF01284C
:10F0A80016BFD2F894401368C4F3032455F824001B
:10F0B80038BDFFF78BFF01280ABF1168D2F89430DA
:10F0C800C1F3031155F82100F2E7FFF76CFF214B5C
:10F0D80001462148012908BF1846E9E7FFF763FF01
:10F0E8001D4A1C4B012818BF13464FF0B042D06888
:10F0F800D168D268C0F306205843C1F30213013324
:10F10800B0FBF3F0530F0133B0FBF3F0D0E7FFF798
:10F118005DFF01280BBF1368D2F89430C3F30313C3
:10F12800002354F82330E0E70A4BDEE7FFF74EFFF1
:10F138004FF0B04301280BBF1B68D3F89430C3F3DA
:10F148000313002351F82300B2E70248B0E700BFD9
:10F15800044801080024F4000048E8014FF0B043D7
:10F1680007B51A6842F001021A601A689207FCD5BE
:10F178001A6822F0F00242F060021A605A6822F41B
:10F188007F425A605A6822F0FE4242F080425A603A
:10F198004FF4E0229A601A6801920199104A0A40D5
:10F1A8000192019A1A60FFF717FF0028FBD14FF070
:10F1B800B0430C4ADA6040F23F3298610192019AFA
:10F1C8001A62D3F8942042F40002C3F89420012074
:10F1D8004FF44032C3F8082103B05DF804FB00BFC8
:10F1E800FFF4CEFE0010042210B54FF0B0440328FF
:10F1F800D4F888302AD11F4A03F0030343F440337C
:10F20800934209D0B3F1031F0DD0013A934211D1B3
:10F21800BDE81040FFF700BFFFF7CBFE01281648F6
:10F2280018BF002010BDFFF7CAFE431E58425841C0
:10F23800C003F7E7FFF7F0FEFFF7D4FEA3680F4A15
:10F24800C3F3C22352F82330D840EBE7034043EA24
:10F2580000400B4B9842DFD0B0F10C1FE3D0043BC9
:10F268009842D5D0FFF7D8FEFFF7BCFEBDE81040A6
:10F27800FFF7C6BE020003000024F400E4470108BB
:10F2880008000C0003685B0670B502462DD4D1E96E
:10F2980000363343CE68056848690C6A33430E6903
:10F2A80033438E6903433343CE6925F47F453343A3
:10F2B80025F0BF0523432B43136053688D6823F45F
:10F2C800706323F0040345EA10401843B5F5006F56
:10F2D80050603EBF536843F480535360B4F5005FF9
:10F2E80001D18B8C1361012000E00020D36923F445
:10F2F8000063D36170BD00001A4A0368904210B5DC
:10F3080002D0B0F1804F09D14C6823F070039042CD
:10F3180043EA040309D0B0F1804F06D0124A904264
:10F3280003D002F58062904203D1CA6823F4407387
:10F33800134303608B68C3620B888362094B98424E
:10F3480007D003F5C053984203D003F58063984271
:10F3580001D10B690363436943F001034361012051
:10F3680010BD00BF002C0140004401400F4B9842E3
:10F378000BD14FF0B0431A6C42F480421A641A6CF5
:10F3880022F480421A6401207047094B98420AD13E
:10F398004FF0B0439A6B42F400329A639A6B22F4AE
:10F3A80000329A63EFE70020704700BF0038014041
:10F3B8000044004038B50368DB0704460D464DD4C9
:10F3C8002A69AB68016813436A691343EA691343FE
:10F3D800234A0A40134303604368EA6823F440530E
:10F3E800134343608368AA6923F44073134383601B
:10F3F8001C4B984220D10320FFF7F6FE2B68F0B192
:10F408006A68E2B10B2B15D8174951F82330E9691E
:10F41800B0FBF3F0B1F5004F4FEA520319D103EBFB
:10F428004003B3FBF2F34FF6F0721A40C3F3420302
:10F438001343E360012003E00C4B984207D00020FF
:10F44800E26A2B8822F00F021343E36238BD0C20D6
:10F45800D2E70344B3FBF2F39BB2EAE70020F5E7F7
:10F46800F369FFEF003801404448010800440040B8
:10F4780010B53024632807D80C703021092808D823
:10F4880030301170187010BD01346438E4B2C0B265
:10F49800F0E701310A38C9B2C0B2EFE730B530241D
:10F4A80042F20F75A84212D80C703021B0F57A7F5D
:10F4B80014D211703022632816D81A703023092804
:10F4C80017D8039A1370049B3030187030BDA0F51C
:10F4D8001C5001341038E4B280B2E3E70131A0F5E2
:10F4E8007A70C9B280B2E1E701326438D2B280B230
:10F4F800E1E701330A38DBB280B2E0E770B5324D9C
:10F50800324E3024A84232D80C70314D314C302163
:10F51800A04230D811703049302288422FD21A7058
:10F528002E4A302390422ED8049A13702C4A302346
:10F5380090422FD8059A1370302342F20F729042EE
:10F548002ED8069A13703023B0F57A7F2ED2079AF8
:10F558001370302363282ED8089A13703023092893
:10F568002DD8099A13700A9B3030187070BD013479
:10F57800E4B23044C6E70131C9B22844C8E70132D1
:10F58800D2B2401AC9E70133A0F57420DBB2A0F566
:10F598001070C7E70133A0F5C330DBB2A038C7E766
:10F5A8000133A0F51C50DBB21038C8E70133DBB2D9
:10F5B800A0F57A70C8E70133DBB26438CAE70133D3
:10F5C800DBB20A38CBE700BFFFC99A3B003665C4F7
:10F5D800001F0AFAFFE0F505809698003F420F00E9
:10F5E8009F86010010B58B1C0C464A1CFFF740FF94
:10F5F8000023E37010BD002810B50C460FDA10F197
:10F60800800F0FD04042C0B22D222346611C03F860
:10F61800032BA21CFFF72CFF0023237110BDC0B2DF
:10F628002022F2E72D228020EFE713B50B1D01936E
:10F63800CB1C00934A1C8B1C0C46FFF72FFF0023A2
:10F64800637102B010BD10B588B001F109030693CB
:10F6580001F108030593CB1D04938B1D03934B1DE8
:10F6680002930B1D0193CB1C00934A1C8B1C0C4668
:10F67800FFF744FF0023A37208B010BD0A2230B57B
:10F6880001231446824207D95A1E12B20A241504CD
:10F6980006D50022CA5430BD01339BB26243F1E75C
:10F6A800B0FBF4F504FB1500303088542846013AC5
:10F6B800EDE7031E10B50C4603DBBDE81040FFF76D
:10F6C800DDBF58420131FFF7D9FF2D23237010BD4C
:10F6D80010B5034C2146FFF785FF204610BD00BF3B
:10F6E800B83F002010B5034C2146FFF784FF2046A1
:10F6F80010BD00BFB83F002010B5034C2146FFF7EE
:10F7080094FF204610BD00BFB83F002010B5034C41
:10F718002146FFF798FF204610BD00BFB83F0020E4
:10F7280013B503688DF807109C680DF107010123D4
:10F73800A04702B010BD07B503688DF807101B6914
:10F7480001220DF10701984703B05DF804FB2DE98C
:10F75800F0411D46036804465B690F461646984704
:10F76800236820461B689847221D39462046FFF724
:10F77800D7FF2DB123682A461B6931462046984792
:10F78800236820465B689847236820469B69BDE844
:10F79800F0410C2118472DE9F0411E460368044644
:10F7A8005B6915460F469847236820461B689847AB
:10F7B800221D39462046FFF7B3FF20460021FFF7F8
:10F7C800BAFF23682046DB683246294698472368F3
:10F7D80020465B68BDE8F04118472DE9F0411F4617
:10F7E800036804465B690D46164698472368204619
:10F7F8001B689847221D20460D21FFF791FF290A13
:10F808002046FFF798FFE9B22046FFF794FF2368E8
:10F8180031463A4620461B699847236820465B686C
:10F828009847236820469B69BDE8F0410C2118479A
:10F8380007B501238DF807200DF10702FFF7CDFF6B
:10F8480003B05DF804FB2DE9F0411F460368044648
:10F858005B690D4616469847236820461B689847FB
:10F86800221D20461D21FFF75BFF290A2046FFF7CE
:10F8780062FFE9B22046FFF75EFF20460021FFF74E
:10F888005AFF23682046DB683A4631469847236882
:10F8980020465B68BDE8F041184707B501230DF124
:10F8A8000702FFF7D0FF9DF8070003B05DF804FBDF
:10F8B8002DE9F0411E46036804465B690F4615466C
:10F8C8009847236820461B689847221D20460E212A
:10F8D800FFF726FF39462046FFF72DFF2368294604
:10F8E800324620461B699847236820465B6898473C
:10F8F800236820469B69BDE8F0410C2118472DE993
:10F90800F0411E46036804465B690F461546984752
:10F91800236820461B689847221D20461E21FFF7B2
:10F92800FFFE39462046FFF706FF20460021FFF775
:10F9380002FF23682046DB68324629469847236839
:10F9480020465B68BDE8F041184710B5002304461F
:10F958001A46C021FFF7FBFE207910BD37B50446D3
:10F968000D468DF80710012380210DF10702FFF7DE
:10F97800EEFE2368012D9B690CBF322140F2DC5159
:10F98800204603B0BDE83040184737B501230C4680
:10F998008DF807100DF107028A210546FFF7D7FEFB
:10F9A800AC7103B030BD07B5042309BA01910DEB62
:10F9B80003028621FFF7CBFE03B05DF804FB07B511
:10F9C80002238DF804108DF805208F2101AAFFF776
:10F9D800BEFE03B05DF804FB37B58DF80630002392
:10F9E8008DF807300423044615468DF804108DF869
:10F9F80005208B210DEB0302FFF7A9FE40F68901D4
:10FA08002046FFF74AFF062D16BF40F0040200F01B
:10FA1800FB02D2B240F6890120468DF80420FFF798
:10FA280007FF03B030BD73B515468DF803300022CB
:10FA38009DF818309DF81C608DF8002004468DF85C
:10FA480001108DF804308C2106236A468DF8025087
:10FA58008DF80560FFF77BFE40F236712046FFF710
:10FA68001CFF5EB100F0FB0240F2367120468DF8B3
:10FA78000020FFF7DDFE657102B070BD40F00402A2
:10FA8800D2B2F1E707B55BBAADF80430BDF8103073
:10FA98005BBAADF8063049BA082352BAADF800107F
:10FAA800ADF8022019466A46FFF751FE03B05DF82B
:10FAB80004FB07B5022301AA1221FFF76CFE9DF88B
:10FAC80004309DF8050000EB032080B203B05DF818
:10FAD80004FB07B5022349BAADF8041001AA194678
:10FAE800FFF735FE03B05DF804FB07B502238DF878
:10FAF80004108DF805208E2101AAFFF728FE03B017
:10FB08005DF804FB13B56FF07F43994228BF19468F
:10FB18000B0C04468DF804300B0A8DF805308DF86F
:10FB2800061001AA03238321FFF711FE236864212D
:10FB38009B692046984702B010BD13B56FF07F430C
:10FB4800994228BF19460B0C04468DF804300B0A5D
:10FB58008DF805308DF8061001AA03238221FFF7DE
:10FB6800F6FD236864219B692046984702B010BDC2
:10FB780037B503230D461446142101AAFFF70BFEDF
:10FB88009DF804305B085B422B809DF90530002B03
:10FB9800B8BF03339B10237003B030BD37B50223C1
:10FBA8000D461446132101AAFFF7F5FD9DF8043010
:10FBB8002B709DF80530237003B030BD10B5436835
:10FBC8000D4A23F07F4323F0FF039342044611D1EB
:10FBD800002240F60211FFF72BFE40F644112046A2
:10FBE800FFF75BFE40F00202D2B240F64411204615
:10FBF800FFF71EFE10BD00BF0001010070B50546ED
:10FC08000E46FFF756FF314604462846FFF761FFC8
:10FC1800A30702D52846FFF7D1FF204670BD07B5D8
:10FC2800002914BF402320238DF807300DF1070267
:10FC380001239321FFF78BFD03B05DF804FB10B59A
:10FC4800002304461A46C121FFF781FD2368204698
:10FC58009B69BDE810404621184708B5FFF775FEB7
:10FC680080B208BD07B50023ADF8043001AA02230D
:10FC78000721FFF76CFD03B05DF804FB07B5130C13
:10FC88008DF8053052BA04238DF80410ADF806201B
:10FC980097210DEB0302FFF75AFD03B05DF804FB53
:10FCA80008B50A4640F6AC01FFF7C2FD08BD10B51D
:10FCB80040F6D8010446FFF7F0FD40F01E02D2B22C
:10FCC80040F6D8012046FFF7B3FD10BD08B50A4637
:10FCD80040F6E701FFF7ACFD08BD000007B5054B8E
:10FCE800019304230DEB03029521FFF730FD03B0C8
:10FCF8005DF804FB0407000107B502238DF8041022
:10FD08008DF80520982101AAFFF721FD03B05DF8C1
:10FD180004FB00000000000013B504461C48B0FBBB
:10FD2800F1F1080C8DF80000080A8DF8010004981C
:10FD38008DF803208DF804308DF80210F0F76CFB75
:10FD480011A3D3E90023F0F70BFDF0F7F1FD030C45
:10FD58008DF8053043BA6A46ADF8063020460823C8
:10FD68008B21FFF7F4FC40F689012046FFF795FD4B
:10FD780040F00402D2B240F6890120468DF80020F6
:10FD8800FFF756FD02B010BD000000008084EE3F72
:10FD98000000093D1FB58DF807309DF818308DF823
:10FDA80008309DF81C308DF809309DF820308DF80A
:10FDB8000A309DF824308DF80B3049BA9DF8283068
:10FDC800ADF804108DF806208DF80C3001AA09232F
:10FDD8008C21FFF7BCFC05B05DF804FB07B50023D8
:10FDE80049BAADF80010ADF8023001936A4608230D
:10FDF8004FF4D861FFF7F1FC03B05DF804FB13B5CD
:10FE080003230C4601AA1421FFF7C5FC9DF8063010
:10FE18005B085B42238002B010BD000038B5044681
:10FE280000F03CFA214605462046F1F775F880B9FE
:10FE3800204600F067F84FF07E51F1F763F840B1C3
:10FE480001F08CFA21230360BDE83840024800F035
:10FE580097B8284638BD00BFDC15010800F060BB24
:10FE680038B5054600F090F8294604462846F1F7CB
:10FE780053F868B900212846F1F726F840B101F097
:10FE88006DFA2123002103600846F0F733FF04468A
:10FE9800204638BD07B51A4A20F000439342014670
:10FEA80005DC002103B05DF804EB00F001B9B3F103
:10FEB800FF4F04DBF0F760FD03B05DF804FB694613
:10FEC80000F0B4FB00F00302012A07D0022A0CD08C
:10FED80082B90199009800F0EBF8EDE701990098D4
:10FEE80000F066F900F10040E6E70199009800F09B
:10FEF800DFF8F7E701990098012200F059F9DBE7EC
:10FF0800D80F493F20F000407047000007B51B4A52
:10FF180020F000439342014606DC0022002103B092
:10FF28005DF804EB00F044B9B3F1FF4F04DBF0F7E0
:10FF380023FD03B05DF804FB694600F077FB00F091
:10FF48000300012808D002280BD090B90199009825
:10FF5800012200F02DF9ECE70199009800F0A8F8CB
:10FF6800E7E701990098012200F022F900F100402A
:10FF7800DFE70199009800F09BF8F7E7D80F493FB1
:10FF8800004870470000C07F20F00042B2F1FF4FE8
:10FF98002DE9F041034604460AD30146F0F7F6FD81
:10FFA80001462046F0F7EAFC04462046BDE8F08109
:10FFB800002AFAD0002806DA0146F0F7DDFC0146EF
:10FFC800F0F798FEF0E710F0FF424FEAE0513DD01D
:10FFD800C3F3160343F40003CA07A1F17F0558BF12
:10FFE8005B0000246D105B00192026464FF08071DD
:08FFF80072189A42DDBF561891
:020000040801F1
:1000000064189A1A1A4601384FEA42034FEA51011E
:10001000F2D1BAB1144E154F30683968D6F8008065
:10002000F0F7AEFC01464046F0F75CFF50B1306897
:1000300039683668F0F7A6FC01463046F0F748FF0D
:1000400068B10234641004F17C5404EBC554B0E789
:100050005B0001321802FBD5013A891ABCE7013472
:1000600024F00104EEE700BF5402002058020020F3
:10007000C0F3C7537F3B162B10B5014614DC002B91
:1000800007DA013300F0004101D141F07E5108460A
:1000900010BD084A1A411042F9D04FF480011941AD
:1000A000014421EA0201F2E7802BF0D1F0F76AFC6B
:1000B0000146ECE7FFFF7F002DE9F04120F000440E
:1000C000B4F1485F0646884603DAF0F73FFF0028A0
:1000D0005CD031463046F0F75DFD4FF07C5105466F
:1000E000F0F758FD2B4907462846F0F753FD2A49FB
:1000F000F0F748FC2946F0F74DFD2849F0F740FCA1
:100100002946F0F747FD2649F0F73CFC2946F0F771
:1001100041FD2449F0F734FC2946F0F73BFD224924
:10012000F0F730FC2946F0F735FD2946F0F732FDAF
:10013000414605463046F0F72DFD01462846F0F7CA
:100140001FFC1A4B9C4205460ADC01463846F0F774
:1001500017FC01464FF07E50F0F712FCBDE8F0812D
:10016000134B9C42CCBF134C04F17F4421464FF00B
:100170007E50F0F705FC214606463846F0F700FCB5
:100180002946F0F7FDFB01463046E5E74FF07E508B
:10019000E4E700BF4ED747ADF6740F317CF29334DD
:1001A000010DD037610BB63AABAA2A3D9999993E19
:1001B0000000483F0000903E2DE9F84320F0004346
:1001C000B3F1485F04460F46914603DAF0F7BEFEEE
:1001D000002835D021462046F0F7DCFC05460146D4
:1001E0002046F0F7D7FC294906462846F0F7D2FC0E
:1001F0002749F0F7C5FB2946F0F7CCFC2549F0F775
:10020000C1FB2946F0F7C6FC2349F0F7B9FB2946A4
:10021000F0F7C0FC2149F0F7B5FB8046B9F1000FBB
:1002200011D101462846F0F7B5FC1D49F0F7A8FBAF
:100230003146F0F7AFFC01462046F0F7A3FB044639
:100240002046BDE8F8834FF07C513846F0F7A2FC19
:10025000414681463046F0F79DFC01464846F0F79E
:100260008FFB2946F0F796FC3946F0F789FB0C49DD
:1002700005463046F0F78EFC01462846F0F782FB33
:1002800001462046F0F77CFBD9E700BFD3C92E2FEB
:10029000342FD7321BEF3836010D50398988083C8E
:1002A000ABAA2A3E2DE9F04720F00048B8F17E5F66
:1002B000044605460CD18C49F0F76CFC8B49054689
:1002C0002046F0F767FC01462846F0F75BFB06E0A6
:1002D00009DD0146F0F754FB0146F0F70FFD044637
:1002E0002046BDE8F087B8F17C5F0BDAB8F1485FD3
:1002F00073DA7F49F0F746FB4FF07E51F0F706FEC8
:100300000028EDD12046FFF701FE01464FF07E5058
:10031000F0F736FB4FF07C51F0F73CFC7549064690
:10032000F0F738FC7449F0F72DFB3146F0F732FC5A
:100330007249F0F725FB3146F0F72CFC7049F0F7D5
:1003400021FB3146F0F726FC6E49F0F719FB3146E8
:10035000F0F720FC6C49F0F715FB3146F0F71AFC7A
:100360006A4981463046F0F715FC6949F0F708FB09
:100370003146F0F70FFC6749F0F704FB3146F0F720
:1003800009FC6549F0F7FCFA3146F0F703FC4FF041
:100390007E51F0F7F7FA82463046FFF7F9FD5F4BE2
:1003A0009845074663DD51464846F0F7A7FC3946B5
:1003B000F0F7F0FB3946F0F7E5FA0146F0F7E2FA1C
:1003C0005749F0F7DFFA01464748F0F7D9FA002D10
:1003D0000446D8BF00F1004482E70146F0F7DAFB9B
:1003E00044490546F0F7D6FB4349F0F7CBFA2946D6
:1003F000F0F7D0FB4149F0F7C3FA2946F0F7CAFB02
:100400003F49F0F7BFFA2946F0F7C4FB3D49F0F742
:10041000B7FA2946F0F7BEFB3B49F0F7B3FA294695
:10042000F0F7B8FB394906462846F0F7B3FB3849E0
:10043000F0F7A6FA2946F0F7ADFB3649F0F7A2FA35
:100440002946F0F7A7FB3449F0F79AFA2946F0F766
:10045000A1FB4FF07E51F0F795FA01463046F0F7D8
:100460004DFC2146F0F796FB014620462DE701465C
:1004700020F47F68F0F786FA514604464846F0F7C4
:100480003DFC01462046F0F785FB28F00F08814629
:1004900041464046F0F77EFB01463046F0F770FAE1
:1004A000414604463846F0F76DFA01462046F0F71B
:1004B00025FC0146F0F766FA01460C48F0F760FAB1
:1004C00001464846F0F75CFA414604464046F0F7DC
:1004D00059FA01461348F0F753FA01462046F0F75F
:1004E0004FFA01460F4870E7DB0FC93F2EBD3BB303
:1004F000CAF2497108EF1138047F4F3A4611243D82
:10050000A80A4E3E90B0A63EABAA2A3E2EC69D3DFE
:100510006133303F2D57014039D119409999793FC6
:100520002EBD3B33DB0F493FF8B521F00046B6F155
:10053000FF4F034605DC20F00042B2F1FF4F0746B3
:1005400004DD1846F0F71EFA034611E0B1F17E5FB4
:1005500003D1BDE8F84000F0CBB98C1704F00204D9
:1005600044EAD07432B9022C4CD0032C00D1294B70
:100570001846F8BD1EB9002F4ADA274BF8E7B6F146
:10058000FF4F0ED1B2F1FF4F04F1FF3405D1022C21
:100590003AD8224B53F82430EAE7022C36D8204BC5
:1005A000F8E7B2F1FF4FE6D0921BB2F1F45F4FEAE9
:1005B000E25017DA002901DA3C3015DB1846F0F773
:1005C0009DFBFFF7A3FC00F093F90346012C0DD02F
:1005D000022C0ED0002CCBD012491846F0F7D2F9DD
:1005E00011490CE0114BF1E70023EFE703F1004361
:1005F000BEE70C491846F0F7C5F901460A48F0F77E
:10060000BFF9A1E7084BB3E7094BB1E70023AFE718
:10061000064BADE7DB0F49C0DB0FC9BF74480108CB
:10062000804801082EBDBB33DB0F4940DB0FC93FBB
:10063000DB0F493F2DE9F04FA04A20F000469642DB
:1006400087B00C46824604DC002308604B6000251E
:100650001AE09B4A96424BDC00289A499A4F26F0B2
:100660000F0623DDF0F78CF9BE42054610D09749FE
:10067000F0F786F9014620602846F0F781F99349A2
:10068000F0F77EF901256060284607B0BDE8F08FDD
:100690008F49F0F775F98F490546F0F771F9014672
:1006A00020602846F0F76CF98A49E9E7F0F76AF923
:1006B000BE4205460ED08549F0F764F90146206038
:1006C0002846F0F75DF98149F0F75CF94FF0FF3506
:1006D0006060D9E77E49F0F755F97E490546F0F7A5
:1006E00051F9014620602846F0F74AF97949EBE7CD
:1006F000794A964200F39180FFF708FC7749074654
:10070000F0F748FA4FF07C51F0F73CF9F0F71EFC97
:100710000546F0F7EBF96B498146F0F73BFA0146E5
:100720003846F0F72DF9694980464846F0F732FA25
:100730001F2D07460CDC6A4A691E26F0FF0352F89B
:100740002120934204D039464046F0F719F90BE0D6
:1007500039464046F0F714F9C0F3C753C3EBD653FC
:10076000082B4FEAE65B01DC206026E0584948464A
:10077000F0F710FA074601464046F0F701F9014646
:1007800006464046F0F7FCF83946F0F7F9F85149CB
:1007900007464846F0F7FEF93946F0F7F1F801460A
:1007A00007463046F0F7ECF8C0F3C753ABEB030B4A
:1007B000BBF1190F16DC2060B04626684046314672
:1007C000F0F7DEF83946F0F7DBF8BAF1000F6060B9
:1007D000BFF65AAF06F1004600F1004026606060A7
:1007E0006D4251E73F494846F0F7D4F907460146C4
:1007F0003046F0F7C5F8014680463046F0F7C0F8BD
:100800003946F0F7BDF8384906464846F0F7C2F9D0
:100810003146F0F7B5F8074695E7B6F1FF4F05DB2F
:100820000146F0F7ADF86060206010E7F715863FED
:10083000A6EBC7563046F0F789FBF0F757F90146AB
:1008400003903046F0F79CF84FF08741F0F7A2F99B
:100850000646F0F77BFBF0F749F9014604900546A0
:100860003046F0F78DF84FF08741F0F793F900210B
:100870000590F0F723FBF0B100212846F0F71EFBAE
:10088000002814BF01230223184A01920222009279
:1008900021463A4603A800F037F9BAF1000F0546A1
:1008A000BFF6F2AE236803F100432360636803F1EF
:1008B0000043636094E70323E6E700BFD80F493F96
:1008C000E3CB1640800FC93FD00FC93F43443537B3
:1008D0000044353708A3852E800F494384F9223F11
:1008E0008C48010800A3852E32318D240C49010863
:1008F0002DE9F04120F00045B5F1A14F04468046B6
:100900000EDBB5F1FF4F04DD0146F0F73BF804467E
:1009100003E0002800F3CE80674C2046BDE8F0815C
:10092000664B9D420EDCB5F1445F08DA6449F0F78E
:1009300029F84FF07E51F0F7E9FA0028EDD14FF099
:10094000FF361CE0FFF7E2FA5E4B9D4204467CDC7A
:10095000A3F5D0039D4267DC0146F0F713F84FF092
:100960007E51F0F70DF84FF0804105462046F0F734
:1009700009F801462846F0F7C1F900260446214649
:100980002046F0F707F901460746F0F703F94E490C
:100990000546F0F7FFF84D49EFF7F4FF2946F0F769
:1009A000F9F84B49EFF7EEFF2946F0F7F3F849491C
:1009B000EFF7E8FF2946F0F7EDF84749EFF7E2FFD8
:1009C0002946F0F7E7F84549EFF7DCFF3946F0F73D
:1009D000E1F8434907462846F0F7DCF84149EFF7CC
:1009E000CFFF2946F0F7D6F83F49EFF7C9FF294670
:1009F000F0F7D0F83D49EFF7C3FF2946F0F7CAF802
:100A00003B49EFF7BDFF2946F0F7C4F801463846E9
:100A1000EFF7B8FF2146F0F7BDF8731C014633D15C
:100A20002046EFF7ADFF72E74FF07E51EFF7A8FFDA
:100A30004FF07E5105462046EFF7A4FF01462846B9
:100A4000F0F75CF90126044699E72A4B9D4214DC35
:100A50004FF07F51EFF794FF4FF07F51054620464E
:100A6000F0F798F84FF07E51EFF78CFF01462846DB
:100A7000F0F744F90226044681E701461E48F0F7E4
:100A80003DF9032604467AE71C4B53F82610EFF78E
:100A900077FF2146EFF774FF194B014653F8260004
:100AA000EFF76EFFB8F1000F0446BFF636AF00F166
:100AB000004432E7134C30E7DB0FC9BFFFFFDF3ED6
:100AC000CAF24971FFFF973FD769853C59DA4B3D20
:100AD000356B883D6E2EBA3D2549123EABAAAA3E23
:100AE00021A215BD6BF16E3D95879D3D388EE33D8E
:100AF000CDCC4C3EFFFF1B40000080BF344C0108B2
:100B0000244C0108DB0FC93F2DE9F04FDBB0029206
:100B10000493649ABB4B059053F822300193049BD5
:100B20000091013B0393029B1A1DC0F29B80DC1EC7
:100B300048BF1C1DE410671CFB000693029B039A30
:100B4000A3EBC707019B03EB0209659BA4EB02081B
:100B50001EAE03EB880A00254FF0000B4D4540F315
:100B60008380049A1EAB03EB82050DF58C7B4FF05E
:100B700000090023019A914540F39E8013460AAA7A
:100B800002EB83030893659BDDF8048003EB840389
:100B900007935AAB03EB88030AAC53F8505C264624
:100BA000C3464FF087490DF58C7ABBF1000F00F377
:100BB00088803946284600F05BFA4FF078510546A8
:100BC000EFF7E8FF00F0A0FA4FF08241EFF7E2FF05
:100BD00001462846EFF7D4FE0546F0F7B7F906467A
:100BE000EFF784FF01462846EFF7CAFE002F814643
:100BF00040F3868008F1FF320AABC7F1080153F8D1
:100C0000225045FA01F31E448B40ED1A0AAB43F81B
:100C10002250C7F107031D41002D7FDD0022013660
:100C20009246904500F3B080002F05DD012F00F0C3
:100C3000BD80022F00F0C580022D6FD149464FF0D4
:100C40007E50EFF79DFE8146BAF1000F66D039461F
:100C50004FF07E5000F00CFA01464846EFF790FE48
:100C600081465BE0002466E718EB050F07D45AF8CD
:100C70002500EFF73BFF46F8040B01356EE75846B9
:100C8000F9E70793059BDAF8001053F82800EFF70F
:100C900081FF01463046EFF775FE079B064608F1D7
:100CA0000108039A9045AAF1040AEADD4BF8046BA7
:100CB00009F1010904355DE7AA461E464FF0000818
:100CC000EFE74FF06E512846EFF764FFF0F73EF97B
:100CD000EFF70CFF49460990EFF75CFF0146284605
:100CE000EFF74EFEF0F732F90BF1FF3B099B46F8A8
:100CF000040B5AF82B101846EFF744FE054654E74C
:100D000006D108F1FF330AAA52F82350ED1183E708
:100D10004FF07C51F0F7F0F8054698BB00214846AB
:100D2000F0F7CCF8002800F0988008F1FF34234653
:100D3000002201998B424CDA002A67D00AAB083FA7
:100D400053F82430002B00F0868039464FF07E5057
:100D500000F08EF9A246814646AF4FF06E58BAF1C8
:100D6000000F80F2AF8027460022002FC0F2D9800A
:100D700046A9254B01EB870B90464FF0000AA4EBE8
:100D80000709C2E0022549E72368BAF1000F08D13C
:100D90001BB1C3F5807323600123013204349A46EA
:100DA0003FE7C3F1FF0323605346F6E708F1FF3244
:100DB0000AAB53F8223003F07F030AA941F822302E
:100DC0003AE708F1FF320AAB53F8223003F03F0351
:100DD000F3E70AA951F82310013B0A43A9E70134BC
:100DE00053F8042D002AFAD0049B1EAA434408F1AC
:100DF000010602EB830544440DF58C79B44208DA10
:100E0000A046C6E6704C0108444C0108089B01242A
:100E1000E6E7079B53F82600EFF768FEAB4628602D
:100E20004FF0000A4FF00008039B9A4504DD49F893
:100E3000268004350136E1E7059B5BF8040953F889
:100E40002A10EFF7A7FE01464046EFF79BFD0AF197
:100E5000010A8046E8E7013C70E7069B029A484693
:100E6000991A00F005F94FF087410446F0F744F86D
:100E700000B34FF06E512046EFF78CFEF0F766F8A6
:100E8000EFF734FE4FF087418146EFF783FE0146CE
:100E90002046EFF775FDF0F759F80AAB08F10104A9
:100EA00043F828004846F0F751F80AAB083743F8F2
:100EB00024004AE72046F0F749F80AAB444643F8D5
:100EC000280042E70AAB53F82A00EFF70FFE494625
:100ED000EFF760FE414647F82A004846EFF75AFE12
:100EE0000AF1FF3A81463AE753F8040B5BF8041B1A
:100EF00003920293EFF74EFE01464046EFF742FDA4
:100F0000DDE9023280460AF1010A01998A4501DCD5
:100F1000CA45E9DD5AAB03EB8909013F49F8A08CCA
:100F200023E7649B022B07DC002B4EDC2ED006F05F
:100F300007005BB0BDE8F08F649B032BF7D10DF188
:100F4000C80B0BEB8407B846A246BAF1000F49DC88
:100F5000A146B9F1010F60DC0020012C76DC329A49
:100F6000339B002D78D100990A604B600A4690604F
:100F7000DDE757F82410EFF705FD013C002CF8DA07
:100F80000DB100F10040009B1860D0E7002032AFA7
:100F9000F4E757F82810EFF7F5FC08F1FF38B8F13F
:100FA000000FF6DAADB100F10043009A014613607C
:100FB0003298EFF7E5FC4FF0010844450BDA0DB12C
:100FC00000F10040009B5860B1E7A046002032AF1E
:100FD000E5E70346E9E757F8041FEFF7D3FC08F10C
:100FE0000108EAE7D8F8003058F8042C02931946B3
:100FF00010460192EFF7C6FC019A01468146104661
:10100000EFF7BEFC029B1946EFF7BCFC48F8040959
:101010000AF1FF3AC8F8009097E757F8043CD7F870
:1010200000A0019351461846EFF7ACFC019B014626
:1010300080461846EFF7A4FC5146EFF7A3FC47F8AB
:10104000040909F1FF39C7F8008082E75BF8241032
:10105000EFF798FC013C80E7009902F1004203F1B0
:1010600000430A604B600A4600F100407FE700BF82
:1010700030F0004238B503460D4604462ED0B2F19A
:10108000FF4F04D30146EFF77DFC034626E010F046
:10109000FF4F18D14FF09841EFF77CFD174A95426A
:1010A00003460CDBC0F3C7520446193A4CF25031E8
:1010B0008D420ADD1249184661F31E0000E0114915
:1010C000EFF768FDE1E7D20DF0E75119FE29F1DCF9
:1010D000002905DD24F0FF4444EAC153184638BD19
:1010E00011F1160F01DA0749E5E701F1190024F0C3
:1010F000FF444FF04C5144EAC050E1E7B03CFFFFE1
:10110000CAF249716042A20D70B5C0F3C7557F3D68
:10111000162D0146044620F0004625DC002D0EDA8F
:101120001649EFF72FFC0021EFF7F0FE28B1002C55
:1011300022DA134B002E18BF1C4621461AE0114E2E
:101140002E41304216D00D49EFF71CFC0021EFF77D
:10115000DDFE0028F1D0002CBEBF4FF400032B4170
:10116000E41824EA0604E8E7B6F1FF4F02D3EFF7EC
:1011700009FC0146084670BD0024DEE7CAF2497149
:10118000000080BFFFFF7F000A22002100F07EB830
:10119000012B2DE9F0478646904601D0242B06D935
:1011A00000F0E0F8162303600020BDE8F087364821
:1011B0000D462A4615F8014B065D16F00806F8D1D3
:1011C0002D2C2ED12C780126951C002B57D0102BBE
:1011D00009D1302C07D12A7802F0DF02582A49D1F0
:1011E0006C781023023506F1004C0CF1FF3C002214
:1011F000BCFBF3F9104603FB19CAA4F13007092F11
:1012000014D83C46A34220DD571C07D0814519D392
:1012100001D1A24516DB00FB0340012215F8014B6A
:10122000EBE72B2C04BF2C78951CCEE7A4F14107EB
:10123000192F01D8373CE5E7A4F16107192F04D82D
:10124000573CDFE74FF0FF32E8E7531C08D1222379
:10125000CEF800306046B8F1000FA6D0691E06E057
:1012600006B14042B8F1000F9FD0002AF6D1C8F86D
:1012700000109AE73024002BB5D10823B3E7302CB7
:10128000A9D00A23AFE700BF7D4C010813460A46E8
:10129000014602480068FFF77BBF00BFA80200209C
:1012A000024B0344587800F0030070477C4C01085F
:1012B000034B1B5C03F00303022B08BF203870476D
:1012C0007D4C0108884210B501EB020402D984422A
:1012D000234607D8431EA14208D011F8012B03F87A
:1012E000012FF8E7024401468A4200D110BD13F8ED
:1012F000014D02F8014DF7E702440346934200D145
:10130000704703F8011BF9E710B50246147813463D
:101310000132002CFAD1013B11F8012B03F8012F07
:10132000002AF9D110BDC9B20346184613F8012BA3
:1013300012B18A42F9D17047002918BF00207047C6
:1013400010B56AB10139841810F8012B11F8013F6A
:101350009A4203D1A04201D0002AF5D1D01A10BD83
:101360001046FCE7014B1868704700BFA802002038
:1013700070B50D4D0D4C641BA4100026A64209D17A
:101380000B4D0C4C00F02EF8641BA4100026A64256
:1013900005D170BD55F8043B98470136EEE755F886
:1013A000043B98470136F2E7804D0108804D010863
:1013B000804D0108884D0108034611F8012B03F800
:1013C000012B002AF9D170470A44914200F1FF3302
:1013D00000D1704710B511F8014B03F8014F91424D
:1013E000F9D110BDF8B500BFF8BC08BC9E467047E7
:0C13F000F8B500BFF8BC08BC9E46704772
:1013FC0000080008005001500250035004500550E2
:10140C0006500750085009500A500B500C500D5004
:10141C00F150F25001F105500000000001000000F5
:10142C00020000006D696E2C00206D572C002057B7
:10143C002C002E00011F136F01130503020B050274
:10144C0000D57FAAFE2B815429FC5683D702A87D98
:10145C0052872DF8AC79D3067BAE04D18550FA2F88
:10146C00A471DB0E5A8F25F08D58F22773A60CD978
:10147C00F623895C08DD77A2DF0AA07521F45E8B68
:10148C009D48E23763B61CC9B461CB1E4A9F35E058
:10149C00CF1AB06531E44E9BE633994C18CD67B248
:1014AC0039EC4693C712B86D10C56FBAEE3B914438
:1014BC006BBE14C19540EA3F42973DE8BC69C31628
:1014CC00EF3A904511C46EBBC613B96C38ED479218
:1014DC00BD68C21743963CE99441EB3E6ABF15C008
:1014EC004B9E34E1B560CA1F62B71DC89C49E336F8
:1014FC0019CC66B3E732984D30E54F9ACE1BB164E8
:10150C0072A70DD88C59F3265B8E24F1A570DA0FD7
:10151C0020F55F8ADE0BA17409DC76A3F722885DC7
:10152C00D603A97C28FD5782FF2A805501D47EABB7
:10153C008451FB2E7AAF05D0AD78D20753862CF9A7
:10154C006162636465666768696A6B6C6D6E6F7007
:10155C007172737475767778797A303132333435B9
:10156C00363738395F232D2E0000000000000000B4
:10157C00000000005B1A00080000000000000000E2
:10158C00671A00080000000000000000431A000861
:10159C006D6C72732E300053657475705374617278
:1015AC007453747834547800536574757053746143
:1015BC0072744D61726B65720021656E6421006DF1
:1015CC004C525301020304006D4C525304030201AC
:1015DC0000656E61626C65642C616E74656E6E6123
:1015EC00312C616E74656E6E61322C723A656E2EA2
:1015FC0020743A616E74312C723A656E2E20743AF6
:10160C00616E7432007472616E73702E2C6D617623
:10161C006C696E6B2C6D61766C6E6B582C6D737087
:10162C005800322E342047487A2C393135204D4819
:10163C007A204643432C383638204D487A2C3433A4
:10164C0033204D487A2C373020636D2048414D2C87
:10165C00383636204D487A20494E00656E61626CF2
:10166C0065642C616E74656E6E61312C616E74658F
:10167C006E6E61322C72656E207461312C72656EE7
:10168C002074613200353020487A2C333120487A6E
:10169C002C313920487A2C464C52432C46534B2C37
:1016AC003139487A377800322E342047487A2C3931
:1016BC003135204643432C383638204D487A2C346B
:1016CC003333204D487A2C373020636D2C38363626
:1016DC0020494E00202F2D2D00202F653100202F6A
:1016EC00653600202F65313100202F653133000D18
:1016FC000A00212120527820706172616D2076657C
:10170C007273696F6E20736D616C6C657220746896
:10171C00616E20547820706172616D2076657273F1
:10172C00696F6E2E20212100212120506C65617380
:10173C006520757067726164652072656365697692
:10174C0065722E20202020202020202020202020E8
:10175C002020202020202020202020212100212199
:10176C0020547820706172616D2076657273696F98
:10177C006E20736D616C6C6572207468616E2052A2
:10178C007820706172616D2076657273696F6E2E50
:10179C0020212100212120506C656173652075701A
:1017AC006772616465205478206D6F64756C652E6A
:1017BC00202020202020202020202020202020201D
:1017CC0020202020202020212100436F6E66696795
:1017DC0049643A003F0020206D696E3A20002020B9
:1017EC006D61783A2000202000203D200020205BF5
:1017FC00612D7A302D39232D2E5F5D002D2028751B
:10180C006E617661696C61626C652900205B0028F1
:10181C00756E6368616E676561626C6529007761DE
:10182C00726E3A207265636569766572206E6F74AC
:10183C0020636F6E6E6563746564002800292C004C
:10184C002C20003B20003B00202054783A204449B7
:10185C005920453737204532322C2076312E332E05
:10186C00303600202052783A20002D2028756E65E5
:10187C0078706563746564206572726F72290020DC
:10188C002063683A20002020665F7265673A20006A
:10189C002020663A2000206B487A00202068656C76
:1018AC00702C20682C203F20202D3E2074686973FA
:1018BC002068656C702070616765002020762020A0
:1018CC002020202020202020202D3E207072696EA8
:1018DC00742064657669636520616E642076657238
:1018EC0073696F6E002020706C2020202020202037
:1018FC002020202D3E206C69737420616C6C20704C
:10190C006172616D6574657273002020706C206368
:10191C0020202020202020202D3E206C6973742054
:10192C00636F6D6D6F6E20706172616D6574657241
:10193C0073002020706C2074782020202020202020
:10194C002D3E206C69737420547820706172616D27
:10195C006574657273002020706C207278202020D2
:10196C00202020202D3E206C69737420527820702A
:10197C006172616D657465727300202070206E61F8
:10198C006D65202020202020202020202D3E206747
:10199C00657420706172616D657465722076616C1E
:1019AC00756500202070206E616D65203D2076618C
:1019BC006C756520202D3E207365742070617261FA
:1019CC006D657465722076616C75650020207020E1
:1019DC006E616D65203D203F2020202020202D3E73
:1019EC002067657420706172616D65746572207614
:1019FC00616C756520616E64206C697374206F6610
:101A0C0020616C6C6F7765642076616C7565730012
:101A1C0020207073746F72652020202020202D3EB2
:101A2C002073746F726520706172616D657465727C
:101A3C0073002020736574636F6E66696769642038
:101A4C002D3E2073656C65637420636F6E666967E9
:101A5C0020696400202062696E64202020202020F0
:101A6C0020202D3E2073746172742062696E64694B
:101A7C006E6700202072656C6F616420202020202E
:101A8C00202D3E2072656C6F616420616C6C20703F
:101A9C006172616D657465722073657474696E67CB
:101AAC007300202073746174732020202020202068
:101ABC002D3E207374617274732073747265616D42
:101ACC00696E672073746174697374696373002041
:101ADC00206C69737466726571732020202D3E2012
:101AEC006C69737473206672657175656E63696574
:101AFC0073207573656420696E2066687373207338
:101B0C006368656D6500202073797374656D626F11
:101B1C006F7420202D3E2063616C6C20737973747C
:101B2C00656D20626F6F746C6F616465720020204C
:101B3C00656D70747920636D64002020696E766128
:101B4C006C696420636D6400202073747265616D30
:101B5C00696E672073746174732073746F70706531
:101B6C0064003E00202074696D656F7574006865B3
:101B7C006C7000706C00706C206300706C2074785A
:101B8C0000706C207278006572723A20696E766112
:101B9C006C696420706172616D65746572206E6130
:101BAC006D65006572723A206E6F2076616C75659A
:101BBC0020737065636966696564006572723A20AA
:101BCC00696E76616C69642076616C756500707302
:101BDC00746F7265002020547820706172616D659D
:101BEC00746572732073746F726564002020706169
